:020000040800F2
:10000000000001203DD801088DD801088DD80108D5
:100010008DD801088DD801088DD801080000000096
:100020000000000000000000000000008DD8010862
:100030008DD80108000000008DD80108FF5C000881
:100040008DD801088DD801088DD801088DD80108F8
:100050008DD801088DD80108415F0008475F00086E
:100060004D5F0008535F0008595F00088DD80108F4
:100070008DD801088DD801088DD801088DD80108C8
:100080008DD801088DD801088DD801088DD80108B8
:10009000000000008DD801085F5F00088DD80108BE
:1000A000395700088DD801084D57000851570008EE
:1000B000655700087957000871F000087DF00008C6
:1000C00089F0000895F000088DD801088DD8010846
:1000D000A96B0008C16B0008DD6B00088DD8010812
:1000E0008DD80108755F00088DD801088DD80108EA
:1000F0008DD8010800000000000000008DD8010824
:10010000A1F00008ADF000087DE401088DD80108D9
:100110008DD801088DD801088DD801088DD8010827
:100120008DD801088DD801088DD801088DD8010817
:080130008DD801088DD80108EB
:1001400081F0004102E000BF83F0004330B54FEA88
:1001500041044FEA430594EA050F08BF90EA020FF5
:100160001FBF54EA000C55EA020C7FEA645C7FEA88
:10017000655C00F0E2804FEA5454D4EB5555B8BFAB
:100180006D420CDD2C4480EA020281EA030382EA1C
:10019000000083EA010180EA020281EA0303362DAE
:1001A00088BF30BD11F0004F4FEA01314FF4801C81
:1001B0004CEA113102D0404261EB410113F0004F93
:1001C0004FEA03334CEA133302D0524263EB43034A
:1001D00094EA050F00F0A780A4F10104D5F1200EE8
:1001E0000DDB02FA0EFC22FA05F2801841F1000143
:1001F00003FA0EF2801843FA05F359410EE0A5F117
:1002000020050EF1200E012A03FA0EFC28BF4CF047
:10021000020C43FA05F3C01851EBE37101F00045FD
:1002200007D54FF0000EDCF1000C7EEB00006EEB0A
:100230000101B1F5801F1BD3B1F5001F0CD3490894
:100240005FEA30004FEA3C0C04F101044FEA4452EB
:1002500012F5800F80F09A80BCF1004F08BF5FEA72
:10026000500C50F1000041EB045141EA050130BD52
:100270005FEA4C0C404141EB0101013C28BFB1F564
:10028000801FE9D291F0000F04BF01460020B1FAAF
:1002900081F308BF2033A3F10B03B3F120020CDA82
:1002A0000C3208DD02F1140CC2F10C0201FA0CF060
:1002B00021FA02F10CE002F11402D8BFC2F1200CC5
:1002C00001FA02F120FA0CFCDCBF41EA0C0190407B
:1002D000E41AA2BF01EB0451294330BD6FEA0404C4
:1002E0001F3C1CDA0C340EDC04F11404C4F12002AF
:1002F00020FA04F001FA02F340EA030021FA04F3C1
:1003000045EA030130BDC4F10C04C4F1200220FA17
:1003100002F001FA04F340EA0300294630BD21FA55
:1003200004F0294630BD94F0000F83F4801306BF1B
:1003300081F480110134013D4EE77FEA645C18BF0F
:100340007FEA655C29D094EA050F08BF90EA020FA6
:1003500005D054EA000C04BF1946104630BD91EA9E
:10036000030F1EBF0021002030BD5FEA545C05D1A1
:100370004000494128BF41F0004130BD14F58004E0
:100380003CBF01F5801130BD01F0004545F0FE4154
:1003900041F470014FF0000030BD7FEA645C1ABF89
:1003A000194610467FEA655C1CBF0B46024650EAC0
:1003B000013406BF52EA033591EA030F41F40021EC
:1003C00030BD00BF90F0000F04BF0021704730B572
:1003D0004FF4806404F132044FF000054FF0000147
:1003E00050E700BF90F0000F04BF0021704730B508
:1003F0004FF4806404F1320410F0004548BF4042DD
:100400004FF000013EE700BF42004FEAE2014FEA31
:1004100031014FEA02701FBF12F07F4393F07F4F0C
:1004200081F06051704732F07F4208BF704793F00F
:100430007F4F04BF41F40021704730B54FF4607422
:1004400001F0004521F000411CE700BF50EA010225
:1004500008BF704730B54FF000050AE050EA0102CE
:1004600008BF704730B511F0004502D5404261EB3E
:1004700041014FF4806404F132045FEA915C3FF47F
:10048000D8AE4FF003025FEADC0C18BF03325FEA1C
:10049000DC0C18BF033202EBDC02C2F1200300FACD
:1004A00003FC20FA02F001FA03FE40EA0E0021FAF2
:1004B00002F11444BDE600BF70B54FF0FF0C4CF4E0
:1004C000E06C1CEA11541DBF1CEA135594EA0C0F92
:1004D00095EA0C0F00F0DEF82C4481EA030621EACD
:1004E0004C5123EA4C5350EA013518BF52EA033508
:1004F00041F4801143F4801338D0A0FB02CE4FF0BA
:100500000005E1FB02E506F00042E0FB03E54FF0E9
:100510000006E1FB03569CF0000F18BF4EF0010EE1
:10052000A4F1FF04B6F5007F64F5407404D25FEADD
:100530004E0E6D4146EB060642EAC62141EA555190
:100540004FEAC52040EA5E504FEACE2EB4F1FD0CD2
:1005500088BFBCF5E06F1ED8BEF1004F08BF5FEA50
:10056000500E50F1000041EB045170BD06F0004602
:1005700046EA010140EA020081EA0301B4EB5C04AF
:10058000C2BFD4EB0C0541EA045170BD41F48011A7
:100590004FF0000E013C00F3AB8014F1360FDEBFCC
:1005A000002001F0004170BDC4F10004203C35DAA8
:1005B0000C341BDC04F11404C4F1200500FA05F32B
:1005C00020FA04F001FA05F240EA020001F00042CC
:1005D00021F0004110EBD37021FA04F642EB060142
:1005E0005EEA430E08BF20EAD37070BDC4F10C046C
:1005F000C4F1200500FA04F320FA05F001FA04F230
:1006000040EA020001F0004110EBD37041F100011B
:100610005EEA430E08BF20EAD37070BDC4F1200526
:1006200000FA05F24EEA020E20FA04F301FA05F28E
:1006300043EA020321FA04F001F0004121FA04F236
:1006400020EA020000EBD3705EEA430E08BF20EA06
:10065000D37070BD94F0000F0FD101F00046400040
:1006600041EB010111F4801F08BF013CF7D041EAC2
:10067000060195F0000F18BF704703F000465200C6
:1006800043EB030313F4801F08BF013DF7D043EA97
:100690000603704794EA0C0F0CEA135518BF95EA4D
:1006A0000C0F0CD050EA410618BF52EA4306D1D1D4
:1006B00081EA030101F000414FF0000070BD50EAF3
:1006C000410606BF1046194652EA430619D094EA7D
:1006D0000C0F02D150EA013613D195EA0C0F05D167
:1006E00052EA03361CBF104619460AD181EA0301BB
:1006F00001F0004141F0FE4141F470014FF0000073
:1007000070BD41F0FE4141F4780170BD70B54FF00D
:10071000FF0C4CF4E06C1CEA11541DBF1CEA13558D
:1007200094EA0C0F95EA0C0F00F0A7F8A4EB05046F
:1007300081EA030E52EA03354FEA013100F0888066
:100740004FEA03334FF0805545EA131343EA12632F
:100750004FEA022245EA111545EA10654FEA0026E4
:100760000EF000419D4208BF964244F1FD0404F59D
:10077000407402D25B084FEA3202B61A65EB0305F9
:100780005B084FEA32024FF480104FF4002CB6EBB6
:10079000020E75EB030E22BFB61A754640EA0C0036
:1007A0005B084FEA3202B6EB020E75EB030E22BF76
:1007B000B61A754640EA5C005B084FEA3202B6EBB7
:1007C000020E75EB030E22BFB61A754640EA9C0076
:1007D0005B084FEA3202B6EB020E75EB030E22BF46
:1007E000B61A754640EADC0055EA060E18D04FEA04
:1007F000051545EA16754FEA06164FEAC30343EAA4
:1008000052734FEAC2025FEA1C1CC0D111F4801F70
:100810000BD141EA00014FF000004FF0004CB6E769
:1008200011F4801F04BF01430020B4F1FD0C88BF08
:10083000BCF5E06F3FF6AFAEB5EB030C04BFB6EB13
:10084000020C5FEA500C50F1000041EB045170BD06
:100850000EF0004E4EEA113114EB5C04C2BFD4EB33
:100860000C0541EA045170BD41F480114FF0000EB7
:10087000013C90E645EA060E8DE60CEA135594EA33
:100880000C0F08BF95EA0C0F3FF43BAF94EA0C0F36
:100890000AD150EA01347FF434AF95EA0C0F7FF4AB
:1008A00025AF104619462CE795EA0C0F06D152EAFF
:1008B00003353FF4FDAE1046194622E750EA4106E3
:1008C00018BF52EA43067FF4C5AE50EA41047FF4F4
:1008D0000DAF52EA43057FF4EBAE12E74FF0FF3C59
:1008E00006E000BF4FF0010C02E000BF4FF0010C2A
:1008F0004DF804CD4FEA410C7FEA6C5C4FEA430CA3
:1009000018BF7FEA6C5C1BD001B050EA410C0CBFF1
:1009100052EA430C91EA030F02BF90EA020F002053
:10092000704710F1000F91EA030F58BF994208BFBA
:1009300090422CBFD8176FEAE37040F00100704777
:100940004FEA410C7FEA6C5C02D150EA013C07D1CE
:100950004FEA430C7FEA6C5CD6D152EA033CD3D019
:100960005DF8040B704700BF8446104662468C4613
:100970001946634600E000BF01B5FFF7B7FF002846
:1009800048BF10F1000F01BD4DF808EDFFF7F4FF6F
:100990000CBF012000205DF808FB00BF4DF808EDFA
:1009A000FFF7EAFF34BF012000205DF808FB00BF1D
:1009B0004DF808EDFFF7E0FF94BF012000205DF83F
:1009C00008FB00BF4DF808EDFFF7CEFF94BF0120F4
:1009D00000205DF808FB00BF4DF808EDFFF7C4FFED
:1009E00034BF012000205DF808FB00BF4FEA410C36
:1009F0007FEA6C5C02D150EA013C0AD14FEA430C19
:100A00007FEA6C5C02D152EA033C02D14FF0000055
:100A100070474FF0010070474FEA410212F5001293
:100A200015D211D56FF47873B3EB625212D94FEA35
:100A3000C12343F0004343EA505311F0004F23FA1F
:100A400002F018BF404270474FF00000704750EA74
:100A5000013005D111F0004008BF6FF00040704731
:100A60004FF00000704700BF4A0011D212F500128B
:100A700011D20DD56FF47873B3EB62520ED44FEAF6
:100A8000C12343F0004343EA505323FA02F0704776
:100A90004FF00000704750EA013002D14FF0FF30B4
:100AA00070474FF0000070474FEA4102B2F1E04357
:100AB00024BFB3F5001CDCF1FE5C0DD901F0004C45
:100AC0004FEAC0024CEA5070B2F1004F40EB830095
:100AD00008BF20F00100704711F0804F21D113F1C1
:100AE0003872BCBF01F00040704741F480114FEAFA
:100AF0005252C2F11802C2F1200C10FA0CF320FA83
:100B000002F018BF40F001004FEAC1234FEAD3239F
:100B100003FA0CFC40EA0C0023FA02F34FEA430309
:100B2000CCE77FEA625307D150EA01331EBF4FF092
:100B3000FE4040F44000704701F0004040F0FE40AD
:100B400040F40000704700BF80F0004002E000BFAA
:100B500081F0004142001FBF5FEA410392EA030FA8
:100B60007FEA226C7FEA236C6AD04FEA1262D2EBF2
:100B70001363C1BFD218414048404140B8BF5B42F7
:100B8000192B88BF704710F0004F40F4000020F090
:100B90007F4018BF404211F0004F41F4000121F0A6
:100BA0007F4118BF494292EA030F3FD0A2F10102F0
:100BB00041FA03FC10EB0C00C3F1200301FA03F12E
:100BC00000F0004302D5494260EB4000B0F5000F51
:100BD00013D3B0F1807F06D340084FEA310102F110
:100BE0000102FE2A51D2B1F1004F40EBC25008BFC2
:100BF00020F0010040EA03007047490040EB00008C
:100C0000013A28BFB0F5000FEDD2B0FA80FCACF18C
:100C1000080CB2EB0C0200FA0CF0AABF00EBC250B9
:100C200052421843BCBFD0401843704792F0000FA7
:100C300081F4000106BF80F400000132013BB5E7FA
:100C40004FEA41037FEA226C18BF7FEA236C21D070
:100C500092EA030F04D092F0000F08BF08467047D5
:100C600090EA010F1CBF0020704712F07F4F04D1A3
:100C7000400028BF40F00040704712F100723CBFB6
:100C800000F50000704700F0004343F0FE4040F4E0
:100C9000000070477FEA226216BF08467FEA23639E
:100CA0000146420206BF5FEA412390EA010F40F489
:100CB000800070474FF0000304E000BF10F00043D5
:100CC00048BF40425FEA000C08BF704743F09643BC
:100CD00001464FF000001CE050EA010208BF7047D7
:100CE0004FF000030AE000BF50EA010208BF70475E
:100CF00011F0004302D5404261EB41015FEA010C73
:100D000002BF84460146002043F0B64308BFA3F16A
:100D10008053A3F50003BCFA8CF2083AA3EBC2534C
:100D200010DB01FA02FC634400FA02FCC2F120026B
:100D3000BCF1004F20FA02F243EB020008BF20F0A2
:100D40000100704702F1200201FA02FCC2F1200208
:100D500050EA4C0021FA02F243EB020008BF20EAFD
:100D6000DC7070474FF0FF0C1CEAD0521EBF1CEA2B
:100D7000D15392EA0C0F93EA0C0F6FD01A4480EA19
:100D8000010C400218BF5FEA41211ED04FF0006302
:100D900043EA501043EA5111A0FB01310CF000402E
:100DA000B1F5000F3EBF490041EAD3715B0040EA54
:100DB000010062F17F02FD2A1DD8B3F1004F40EB24
:100DC000C25008BF20F00100704790F0000F0CF0F7
:100DD000004C08BF49024CEA502040EA51207F3ABB
:100DE000C2BFD2F1FF0340EAC250704740F4000096
:100DF0004FF00003013A5DDC12F1190FDCBF00F087
:100E000000407047C2F10002410021FA02F1C2F134
:100E1000200200FA02FC5FEA310040F1000053EAD0
:100E20004C0308BF20EADC70704792F0000F00F01E
:100E3000004C02BF400010F4000F013AF9D040EA24
:100E40000C0093F0000F01F0004C02BF490011F4B8
:100E5000000F013BF9D041EA0C018FE70CEAD153B6
:100E600092EA0C0F18BF93EA0C0F0AD030F0004C36
:100E700018BF31F0004CD8D180EA010000F00040EA
:100E8000704790F0000F17BF90F0004F084691F0A8
:100E9000000F91F0004F14D092EA0C0F01D14202E2
:100EA0000FD193EA0C0F03D14B0218BF084608D1AB
:100EB00080EA010000F0004040F0FE4040F40000F5
:100EC000704740F0FE4040F4400070474FF0FF0C88
:100ED0001CEAD0521EBF1CEAD15392EA0C0F93EACF
:100EE0000C0F69D0A2EB030280EA010C49024FEA21
:100EF000402037D04FF0805343EA111143EA1013DA
:100F00000CF000408B4238BF5B0042F17D024FF491
:100F1000000C8B4224BF5B1A40EA0C00B3EB510F6C
:100F200024BFA3EB510340EA5C00B3EB910F24BF55
:100F3000A3EB910340EA9C00B3EBD10F24BFA3EBDA
:100F4000D10340EADC001B0118BF5FEA1C1CE0D1A2
:100F5000FD2A3FF650AF8B4240EBC25008BF20F055
:100F6000010070470CF0004C4CEA50207F32C2BFA9
:100F7000D2F1FF0340EAC250704740F400004FF046
:100F80000003013A37E792F0000F00F0004C02BF77
:100F9000400010F4000F013AF9D040EA0C0093F041
:100FA000000F01F0004C02BF490011F4000F013B9B
:100FB000F9D041EA0C0195E70CEAD15392EA0C0F03
:100FC00008D142027FF47DAF93EA0C0F7FF470AF3B
:100FD000084676E793EA0C0F04D14B023FF44CAF7E
:100FE00008466EE730F0004C18BF31F0004CCAD113
:100FF00030F000427FF45CAF31F000437FF43CAF4F
:101000005FE700BF4FF0FF3C06E000BF4FF0010C70
:1010100002E000BF4FF0010C4DF804CD4FEA400252
:101020004FEA41037FEA226C18BF7FEA236C11D09C
:1010300001B052EA530C18BF90EA010F58BFB2EB4F
:10104000030088BFC81738BF6FEAE17018BF40F0CF
:10105000010070477FEA226C02D15FEA402C05D183
:101060007FEA236CE4D15FEA412CE1D05DF8040B08
:10107000704700BF844608466146FFE70FB5FFF79B
:10108000C9FF002848BF10F1000F0FBD4DF808ED53
:10109000FFF7F4FF0CBF012000205DF808FB00BF44
:1010A0004DF808EDFFF7EAFF34BF012000205DF89E
:1010B00008FB00BF4DF808EDFFF7E0FF94BF0120EB
:1010C00000205DF808FB00BF4DF808EDFFF7D2FFE8
:1010D00094BF012000205DF808FB00BF4DF808ED2B
:1010E000FFF7C8FF34BF012000205DF808FB00BFF8
:1010F0004FEA40024FEA41037FEA226C02D15FEAE5
:10110000402C08D17FEA236C02D15FEA412C02D146
:101110004FF0000070474FF0010070474FEA400267
:10112000B2F1FE4F0FD34FF09E03B3EB12620DD915
:101130004FEA002343F0004310F0004F23FA02F07F
:1011400018BF404270474FF00000704712F1610F26
:1011500001D1420205D110F0004008BF6FF00040FD
:1011600070474FF00000704742000ED2B2F1FE4FC0
:101170000BD34FF09E03B3EB126209D44FEA002366
:1011800043F0004323FA02F070474FF0000070472D
:1011900012F1610F01D1420202D14FF0FF307047CE
:1011A0004FF00000704700BF53B94AB9002908BF8B
:1011B00000281CBF4FF0FF314FF0FF3000F00CB89B
:1011C000ADF1080C6DE904CE1CF028FDDDF804E05B
:1011D000DDE9022304B07047704700BF10F8012B0F
:1011E00011F8013B012A28BF9A42F7D0D01A704764
:1011F000034613F8012B002AFBD1181A0138704757
:1012000001F0FF01102A2BDB10F0070F08D010F8B7
:10121000013B013A8B422DD010F0070F42B3F6D1BB
:10122000F0B441EA012141EA014122F007047FF0D4
:1012300000070023F0E80256083C85EA010586EA2B
:10124000010685FA47F5A3FA87F586FA47F6A5FA67
:1012500087F68EB9EED1F0BC01F0FF0102F0070273
:1012600032B110F8013B013A83EA010313B1F8D11E
:101270000020704701387047002D06BF35460338FF
:10128000073815F0010F07D1013015F4807F02BF38
:10129000013015F4C03F0130F0BC0138704700BF89
:1012A00010B5054C237833B9044B13B10448AFF3A0
:1012B00000800123237010BD5003002000000000B7
:1012C0006435020808B5034B1BB103490348AFF36B
:1012D000008008BD000000005403002064350208AF
:1012E00000B59BB04422002109A820F022F9182261
:1012F000002102A820F01DF9144A136823F4C063EA
:1013000043F400731360136803F4C0630193019BFB
:101310002023089301210023B02208A8CDE910134F
:10132000CDE9122301F080FF00B1FEE74F23CDE9A4
:101330000230CDE90400CDE90600022102A802F046
:101340000FFA00B1FEE71BB05DF804FB0004005883
:101350007047000038B5104C237805460BB90120C2
:1013600038BD01F051FF22784FF47A73B3FBF2F3EA
:10137000B0FBF3F000F0C8FC04460028EFD10F2DBD
:10138000EDD8024629464FF0FF3000F06BFC034BCE
:1013900020461D60E4E700BF00000020040000209C
:1013A00010B5032000F04CFC01F02EFF064B186036
:1013B0000020FFF7CFFF044618B9FFF7C9FF20460A
:1013C00010BD0124FBE700BF40000020034A044B8E
:1013D00011681B780B441360704700BF6C0300203A
:1013E00000000020014B1868704700BF6C0300200C
:1013F0008068C0F380007047F7B50023019304466E
:10140000002800F0E980856D25B904F0EFFAE56564
:1014100084F8545023689A68D00040F1A1809A68FB
:10142000D10000F1B480A26D42F01002A265E26D1D
:1014300042F00102E26501251846FFF7D9FFA26DCF
:1014400002F01002024340F0C980A26D206922F42C
:10145000817242F00202A2659A68D2075DD4226BC3
:10146000A67E94F82CC0003A18BF01221703D4E9D5
:1014700002120A43217E42EA8132617E42EAC1328F
:1014800042EA4632002842EA4C02B4BF20F0004152
:101490004FF400113A430A4394F82010012903D174
:1014A000002E76D142F48032616A21B1A66A01F43D
:1014B000E07131430A43D968E66C21F4FE3121F42E
:1014C000FF711143D96094F83C206168012A01F052
:1014D000404C4CEA060609D1D4E910273A4332437E
:1014E000A66C324342EA0C0242F001061F693E4AF2
:1014F0003A4032431A6121F00042B2F1804F0CD0E1
:10150000B1F1004F09D0394ED6F8082701F4701117
:1015100022F470120A43C6F808275A69666BA16B59
:1015200022F0070232435A615A6922F0700242EAFD
:1015300001125A61002835D19A6A62F00F029A624C
:101540005B6903F007039E423CD10023E365A36D72
:1015500023F0030343F00103A365284603B0F0BD65
:101560009A68234922F0104222F0170242F080527A
:101570009A60204A1268B2FBF1F2013252000192E5
:10158000019A002A3FF44BAF019A013AF7E7002590
:1015900052E7A16D41F02001A165E16D41F001012B
:1015A000E16581E7B0F5001FCAD19A6AE269013AA4
:1015B00092006FF00F0102F01C0201FA02F2216E9C
:1015C0000A43BCE7A36D23F0120343F01003A365A5
:1015D000E36D43F00103E3650125BEE7A36D43F02E
:1015E0001003A365F8E700BF02FCFF1F00200140C5
:1015F000400D030040000020F8B54569082D044661
:101600000E460AD00368DB68D80705D5A36D43F002
:101610002003A3650120F8BD0425FFF7E3FE07467C
:1016200023681A682A4220D0A26D42F40072A26593
:10163000DA6812F4406F14D1A27E92B91A681207C8
:101640000FD51846FFF7D4FE20BB5A6822F00C02D3
:101650005A60A26D22F4807222F0010242F001026F
:10166000A265227EFAB10020D5E7711CD9D0FFF720
:10167000B9FEC01BB04201D8002ED1D123681B682F
:101680002B40CDD1A26D84F8543042F00402A26503
:101690000320C0E7A26D42F02002A265E26D42F095
:1016A0000102E265DDE70C221A60DCE70368186CD2
:1016B00070470000F7B50023019390F85430012BD8
:1016C000044600F0C08005680269012380F85430A8
:1016D0002846FFF78DFE002840F0AF8048680B6871
:1016E000022822F004027ED0B2F1004FC3F3110EA3
:1016F00035D1AA6A42EA0E02AA628A68686902EAD9
:10170000032222F07C4222F0FF0220EA03210A4356
:10171000002B6A611DDA4D4A4D4DD2F80817AB42D5
:1017200001F0E07043D10D0213D4D2F8083723F052
:10173000E073034343F40003C2F80837454B1A68CB
:10174000454BB2FBF3F20C2302FB03330193019BE5
:1017500053BB0020002384F8543003B0F0BD226E48
:1017600000F01F074FF00F0C0CFA07FC6FEA0C0695
:1017700022EA0C0CBEF1000F11D1C3F38462BA400F
:1017800042EA0C0222668008E26901309042B4D835
:10179000A86AC3F38362BA4006403243ACE793FAC7
:1017A000A3F2B2FA82F2EAE7019B013BCEE72B4DAE
:1017B000AB420BD1C901CCD4D2F8083723F0E07387
:1017C000034343F08073C2F80837C2E7244DAB42AD
:1017D000BFD14B02BDD4D2F8083723F0E0730343E6
:1017E00043F48003EFE7B2F1004F01BFAA6AC3F3ED
:1017F00011018A43AA62002BABDA154813498342D0
:10180000D1F8082709D1D1F8083702F0A07223F0E7
:10181000E0731A43C1F808279BE71048834204D1BC
:10182000D1F8083702F44002F1E70D48834290D125
:10183000D1F8083702F0C072E9E7A26D42F0200249
:10184000A265184686E7022087E700BF0020014016
:10185000001000B040000020400D0300004000B820
:10186000002000B4806D7047026838B50446104609
:10187000FFF7BEFD08B9002038BD9368990707D46B
:10188000936823F0004323F0170343F010039360A1
:10189000FFF7A8FD054623689B685B07EBD5FFF7BC
:1018A000A1FD401B0228F6D923689B685A07F2D590
:1018B000A36D43F01003A365E36D43F00103E365FB
:1018C0000120D9E773B50023026801939368DD070F
:1018D000044602D5002002B070BD9168214B194228
:1018E00009D0A36D43F01003A365E36D43F001033A
:1018F000E3650120EFE7936823F0004323F017032B
:1019000043F001039360184BD3F8083718021CD436
:10191000637E012BDED0FFF765FD144E054622687D
:101920001368DB07D6D49368D9075FBF9368334049
:1019300043F001039360FFF755FD401B0228EED9E9
:1019400023681B68DA07EAD4CBE7094B094A1B680E
:10195000B3FBF2F301330193019B002BD8D0019B21
:10196000013BF8E71700008000200140E8FFFF7FFF
:1019700040000020400D030038B504460068FFF722
:1019800037FD054620BB94F85430012B20D00123AD
:1019900084F854302046FFF795FFB0B9A36D226854
:1019A00023F4706323F0010343F48073A3651C23C5
:1019B000E065136084F85400936823F0004323F03B
:1019C000170343F00403936038BD84F85450FBE7D9
:1019D0000220F9E738B503689A680446900704D4F2
:1019E0009A68D10703D4002038BD9B68FBE79A684A
:1019F00002F00502012A19D19A6822F0004222F071
:101A0000170242F002029A6003221A60FFF7EAFC12
:101A1000054623689B68DB07E5D5FFF7E3FC401B21
:101A20000228F6D923689B68DA07F2D5A36D43F044
:101A30001003A365E36D43F00103E3650120D3E7E1
:101A400070B5044600284BD0836D43F002038365D4
:101A5000FFF70AFF054668B92046FFF7BBFF0546BA
:101A600008B90123A3652268936823F0104323F08B
:101A70001703936023685A6822F4677222F0030206
:101A80005A6040F29F321A60D968164A0A40DA60FA
:101A90005A6922F007025A6100269A6A9E621A6AFF
:101AA00002F0F0221A625A6A02F0F0225A62DA6AEE
:101AB00002F0F022DA621A6922F040421A610A4A00
:101AC000D2F8083723F0FE73C2F80837204603F037
:101AD000ADFFE6652666A66584F85460284670BDAD
:101AE0000125FBE700023E830020014010B590F87D
:101AF0005430012B044615D0012380F85430FFF7F1
:101B0000B3FE58B92046FFF765FF38B9A36D23F43B
:101B1000807323F0010343F00103A365002384F8DD
:101B2000543010BD0220FCE7F7B50023019390F874
:101B30005430012B04467FD0012380F85430FFF746
:101B400049FF23689A6812F00102054607D0A36D89
:101B500043F01003A365002384F854302DE0A16DF9
:101B6000364F21F4817141F00201A165DE68D96828
:101B700026F4FF4626F07C0621F40041360421F0CD
:101B80000301360CD96008209968394041F00041C2
:101B900099609968002913DA01990131019101993D
:101BA000B1F52E3FF5D3A36D23F0120343F01003DC
:101BB000A365002384F854300125284603B0F0BD06
:101BC000D3F8B410013801F07F010A44DCD19968E0
:101BD0001A48014041F001019960D3F8B41021F096
:101BE0007F0141EAD202C3F8B4209A68024042F071
:101BF00002029A60FFF7F6FB074623689A68D2074D
:101C000008D4DA683243DA60A36D23F0030343F0AB
:101C100001039FE7FFF7E6FBC01B0228EDD923680D
:101C20009B68D907E9D5A36D43F01003A365E36D65
:101C300043F00103E365BFE70225BEE7E8FFFF7F4E
:101C40000749CA6822F4E0620302120403F4E06365
:101C5000120C134343F0BF6343F40033CB6070476F
:101C600000ED00E0164B30B5DC68C4F30224C4F18B
:101C70000703251D042B28BF0423062D4FF0FF3535
:101C80008CBF033C002405FA03F321EA0303A540BB
:101C900022EA0502A340002843EA0203ACBF00F198
:101CA0006040084A4FEA0313B8BF00F00F00DBB2F0
:101CB000AABF00F56140135480F8003330BD00BF67
:101CC00000ED00E014ED00E0002807DB044A4109C4
:101CD000012300F01F00834042F82130704700BF0D
:101CE00000E100E000280CDB4309064900F01F007A
:101CF00020330122824041F82320BFF34F8FBFF3EE
:101D00006F8F704700E100E00138B0F1807F0BD2A7
:101D10004FF0E023054A5861F02182F8231000209B
:101D2000072298611A6170470120704700ED00E0BA
:101D30000028A1BF43094033054A52F82330A3BF0E
:101D400000F01F0023FA00F000F0010000207047AF
:101D500000E100E0002808DB4309044900F01F000F
:101D600001226033824041F82320704700E100E007
:101D7000704708B5FFF7FCFF08BD704710B5044673
:101D800008B9012010BD437F03F0FF0213B90277A9
:101D9000FFF7F3FF022363772379E3B92368134A3C
:101DA0005A619A6822F018029A6062792368D2B95F
:101DB0004FF0FF321A619A68616922F060020A43AB
:101DC0009A609A68A16922F080020A439A6001230E
:101DD00063770020D6E7D4E90212204600F008F825
:101DE0000028E2D0CDE72269E4E700BFB71DC104B7
:101DF000CB0710B50CD51F23013B1CD321FA03F4EC
:101E0000E407F9D5102A12D004D83AB1082A10D024
:101E100001200BE0182AFBD1062BF9D8006841619C
:101E2000836823F0180313438360002010BD072B41
:101E3000F3E70F2BF1E7102AEAD0E9D8002AE7D11F
:101E4000ECE710B5044640B10223037103F0A0FD96
:101E5000002020616071207110BD0120FCE710B5E9
:101E600004680122236801F0100102FA01F123EA5B
:101E7000010323600271002010BD034640B190F8B9
:101E80002520022A06D00422C263002280F82420E2
:101E9000012070470268806C116821F00E0111600A
:101EA000016821F480710160116821F00101116065
:101EB000D3E9100202F01C0101228A404260D3E9FA
:101EC000132151605A6D32B1116821F48071116093
:101ED000D3E9162151600122002083F8252083F8E0
:101EE0002400704708B590F82530022B03D0042356
:101EF000C363012008BD03681A6822F00E021A604D
:101F00001A6822F001021A60826C136823F480734D
:101F10001360D0E9101303F01C02012393404B60BF
:101F2000D0E913325A60436D33B11A6822F48072DB
:101F30001A60D0E916325A60012380F82530002358
:101F400080F82430836B03B198470020D2E790F8E3
:101F5000250070470A4A536943F4802330B5536122
:101F6000EFF3108472B60023CD58C5500433B3F597
:101F7000807FF9D11369DB03FCD484F3108830BD72
:101F800000400058064B5A69002ABFBF054A9A60B4
:101F900002F188329A60BABF5869C00F00207047BA
:101FA0000040005823016745044B5A6942F0004243
:101FB0005A615869C043C00F704700BF00400058C5
:101FC00070B50546FFF70EFA124E04463369D90381
:101FD00013D43369DA0744BF012232614CF2FA327A
:101FE000134011D10B4E306910F480200BD0FFF755
:101FF000F9F9001BA842F6D304E0FFF7F3F9001B40
:10200000A842E3D3032070BD024A1361024A0120B3
:102010005360F8E700400058700300202DE9F041BC
:10202000184D98462B78012B06460C46174626D0AD
:1020300001232B704FF47A7000236B60FFF7C0FF11
:10204000A0B9012E16D1104A536943F00103536120
:102050002760BFF36F8FC4F804804FF47A70FFF7E6
:10206000AFFF094A536923EA0603536100232B702B
:10207000BDE8F08139462046FFF76CFFEDE702200E
:10208000F6E700BF7003002000400058054A53697E
:1020900023F47E7343EAC00040F4803040F0020035
:1020A00050617047004000582DE9F041234F3B78C4
:1020B000012B054688463FD001233B704FF47A70D0
:1020C00000237B60FFF77CFF044688B92B68042B54
:1020D00013D11B4A536943F4803343F00403536123
:1020E0004FF47A70FFF76CFF0446154B1A681B68B3
:1020F00000233B702046BDE8F0814FF0FF33C8F865
:1021000000306E68D5E901321344B3420AD9304633
:10211000FFF7BCFF4FF47A70FFF752FF50B1C8F8D9
:1021200000600446064A536923F47E7323F00203D9
:102130005361DAE70136E5E70224DBE770030020AC
:10214000004000582DE9F04F564C00234FF00F0887
:102150000A6832FA03F501D1BDE8F08F012505FACE
:1021600003F919EA020275D04E68032706F0030549
:102170004FEA430E07FA0EFC6F1E012F6FEA0C0C9C
:102180006AD8876807EA0C0ACF6807FA0EF747EAA9
:102190000A078760476827EA0909C6F300179F40C6
:1021A00047EA09074760C76807EA0C098F6807FA1A
:1021B0000EF747EA0907022DC76059D0076805FAEC
:1021C0000EF507EA0C073D4316F4403F056041D089
:1021D00023F0030707F1804707F5803703F0030C6E
:1021E000BD684FEA8C0C4FF0070E0EFA0CFEB0F1F2
:1021F000904F25EA0E0E51D02B4DA84250D005F538
:102200008065A84214BF0725022505FA0CF545EAAA
:102210000E05BD602568D74316F4801F0CBF3D40F6
:1022200015432560656816F4001F0CBF3D4015433B
:102230006560D4F8805016F4803F0CBF3D401543D4
:10224000C4F88050D4F88450B60354BF3D401543C1
:10225000C4F8845001337BE7032DAFD0C76807EA89
:102260000C098F6807FA0EF747EA0907C760A5E768
:102270004FEAD30900EB890903F0070AD9F8207067
:102280004FEA8A0A08FA0AFB27EA0B0B0F6907FADA
:102290000AF747EA0B07C9F820708FE70025B4E773
:1022A0000125B2E70008005800040048044AD1683C
:1022B000014208B502D0D06003F02CFE08BD00BF7B
:1022C0000008005803689A69910744BF00229A6287
:1022D0009A69D2075EBF9A6942F001029A6170471B
:1022E00030B5039D04682B4343EA0243064A606805
:1022F000C1F309010B4342EA555223F0004320EA9F
:1023000002000343636030BDFF63FF0370B5426B9F
:102310001F4CA2420BB201F0010501F002041DD0D6
:102320001C4EB2421AD01C4EB24217D0002BACBF8A
:102330000023B8230DB143F0F2030CB143F0F403D2
:10234000102902D143F0900303E0202901D143F08A
:10235000200301680A6813430B6070BD002BACBFFB
:102360000023B8230DB143F0F2030CB143F0F403A2
:102370001029E7D0202902D143F06003E9E7064C99
:10238000A242E6D0402908BF43F04003E1E700BF86
:10239000B92A0008B12D00089529000811F00103A1
:1023A00007D090F8413003F02803282B14BFF22304
:1023B00042238A0709D590F8412002F02802282AF2
:1023C0000CBF43F0440343F0F4030A0401680A68B5
:1023D00048BF43F0B80322EA03030B60704770471D
:1023E00010B5044698B10268242380F84130136880
:1023F00023F001031360FFF7F2FF0020606484F80C
:10240000400084F84100206384F8420010BD0120A0
:10241000FCE70000F8B51F4690F8413003F02803B0
:10242000282B04460E46154601D00120F8BD01B107
:102430001AB94FF400736364F7E748F20101FFF73C
:10244000ADFF90F84030012B40D0012380F84030A0
:1024500090F841302A2B14D10221FFF79FFF036827
:102460001A6810040DD51A68E06B22F400421A6055
:1024700038B1174B8363FFF735FD10B1E06B836B09
:102480009847292384F8413020682023002284F8CB
:1024900042306264436823F4004343606585638D82
:1024A0002385E7620B4B6363836981696662C903B5
:1024B00003D51B0744BF0823C361204684F840208E
:1024C00048F20101FFF722FF0020AFE70220ADE74D
:1024D000B92F0008A72E0008F8B51F4690F8413024
:1024E00003F02803282B04460E46154601D0012090
:1024F000F8BD01B11AB94FF400736364F7E748F20D
:102500000201FFF74BFF90F84030012B3FD090F8CD
:1025100041300121292B80F8401013D1FFF73EFFF5
:1025200003681A6850040DD51A68A06B22F4804223
:102530001A6038B1174B8363FFF7D4FC10B1A06B5E
:10254000836B98472A2384F8413020682023002297
:1025500084F842306264436823F400434360658535
:10256000638D2385E7620C4B6363836981696662CF
:10257000C90303D41B0744BF0823C361204684F862
:10258000402048F20201FFF7C1FE0020B0E7022020
:10259000AEE700BFB92F0008A72E000808B590F8D5
:1025A0004120202A0AD1282280F84120044A42638F
:1025B0004FF40041FFF7AAFE002008BD0220FCE70F
:1025C000A72E00080268436B9169126803B118478F
:1025D00070477047704738B5002580F8425090F832
:1025E0004130212B4FF0200380F841300AD11123D4
:1025F000036345630121FFF7D1FE80F84050FFF7E8
:10260000E8FF38BD1223036345630221FFF7C6FECE
:1026100080F84050FFF7DEFFF3E708B503681A685B
:10262000002180F84210510415D51A6822F4804226
:102630001A6090F84130292B13D1282380F84130BB
:10264000212303630121FFF7A9FE002380F8403016
:102650000CF004FD08BD1204EBD51A6822F4004208
:10266000E6E790F841302A2BF4D1282380F8413056
:10267000222303630221FFF791FE002380F84030FC
:102680000CF0D9FCE6E790F8412002F02802282A55
:10269000F8B5036834D19E69C2689D699968DF689E
:1026A0002D0C022AC6F3004605F0FE051FD185EA6F
:1026B000D11515F00605C1F309020ED1816C013167
:1026C0008164816C022907D108218564D96180F871
:1026D000405031460CF062FCF8BD4FF40041FFF76A
:1026E0005DFE002380F8403007F0FE02F1E74FF472
:1026F0000041FFF753FE002380F840302A46E8E708
:102700000822DA61002380F84030E5E708B5164B6F
:10271000C362202200230363436380F8412080F8D2
:1027200042304B0712D503685A6A436A1A70436AEB
:1027300001334362038D4BB1013B0385438D013B64
:102740009BB24385436C43F00403436448F20301A6
:10275000FFF724FE03681022DA61002380F840307E
:102760000CF054FC08BD00BF0000FFFF704770472D
:10277000704790F84120602A08B54FF0000208D158
:10278000202180F8411080F840200263FFF7F0FF1D
:1027900008BD026380F840200CF064FCF8E70000FC
:1027A00070B500223D4D90F8413080F84220C5625E
:1027B0004285426C283B0A43022B044642642AD8D5
:1027C0000321FFF7EBFD282380F84130344BA06B49
:1027D0006363236B002841D0112B01D0212B3DD105
:1027E00023681A68510442BF1A6822F480421A60B2
:1027F000FFF7ADFB01282CD0A06B2A4B836300238D
:1028000084F84030FFF76EFB002845D0A06B836B47
:10281000BDE87040184748F20301FFF7BFFDFFF71E
:1028200051FD90F84130602B11D0202380F84130C9
:1028300003689A6995060AD59A69D00605D51022CB
:10284000DA61626C42F0040262642022DA610023E1
:10285000BDE72046BDE87040FFF78BBFE06B002866
:10286000F7D0122B01D0222BF3D123681A6812045F
:1028700042BF1A6822F400421A60FFF768FB012881
:10288000E7D0E06B074B8363002384F84030FFF709
:1028900029FB08B1E06BBAE770BD00BF0000FFFF85
:1028A000A72E0008B92F000873B505682023EB6137
:1028B00090F84130212B04460E4635D10121FFF717
:1028C0006DFD112323636B6823F0FF7323F48B33B7
:1028D00023F4FF7323F001036B6000236363F206AC
:1028E000A3F58033E36205D51023EB61636C43F0FD
:1028F0000403636494F84130602B05D1730741BF32
:102900006B6ADBB20193019B2046FFF7DBFC636C33
:1029100094F84120602A00D07BB1616C204602B05F
:10292000BDE87040FFF73CBF90F84130222BCAD180
:102930000221FFF733FD1223C4E794F84120212A36
:1029400012D1202284F84120236394F8422084F895
:102950004030402A84F8423003D1FFF707FF02B02D
:1029600070BDFFF736FEFAE794F84120222AF6D12F
:10297000202284F84120236394F8422084F84030D8
:10298000402A84F8423002D1FFF7F1FEE7E7FFF773
:1029900021FEE4E713B590F84030012B044600F027
:1029A0008580012380F84030CB0612D5D30610D5A0
:1029B00003681022DA61436C43F00403436420216E
:1029C000FFF7A4FCFFF77EFC002084F8400002B073
:1029D00010BD880708D5930706D52368226D9A6233
:1029E0004FF0FF332365EFE7080633D5530631D5A3
:1029F00010212046FFF78AFC638D9BB233B3638DB1
:102A00009BB2FF2B18D90023FF22E16C2285009393
:102A10004FF0807389B2FFF763FC638D228D9B1AA0
:102A20009BB2638594F841202368222A1A6832D128
:102A300042F400421A60C7E7628DE16C92B2002353
:102A400022850093D2B24FF00073E3E74021FFF7F5
:102A5000A7FEB9E7480621D553061FD594F84110C3
:102A6000134A144B222918BF1346628D92B2FF2AD3
:102A700008D9FF22E16C228500934FF0807389B260
:102A80002046C8E7628DE16C92B222850093D2B2F3
:102A90004FF00073F3E742F48042CBE7880693D50A
:102AA000930691D52046FFF7FFFE8DE702208EE7C3
:102AB000002000800024008073B590F84030012B86
:102AC000044678D0012380F84030CB0612D5D606D4
:102AD00010D503681022DA61436C43F004034364A9
:102AE0002021FFF713FCFFF7EDFB002084F84000E6
:102AF00002B070BD0D0641D550063FD525682B6844
:102B000023F040032B60638D9BB25BB36968638DD8
:102B10009BB2FF2BC1F309011AD9FF2323854FF084
:102B200080730022268D009294F828202046FFF71B
:102B3000D7FB638D9B1B9BB2638594F84130222B9E
:102B40002B680CBF43F4004343F480432B60CCE775
:102B5000638D2385E36A13F5803F14BFE36A4FF06A
:102B60000073DEE76B689A0103D42046FFF733FD5C
:102B7000BBE740212046FFF713FEB6E74B0612D510
:102B8000560610D5638D9BB2002BF2D123685A688C
:102B90009501AAD4E26A12F5803FE6D15A6842F460
:102BA00080425A60A1E788069FD593069DD52046AE
:102BB000FFF77AFE99E702209AE7036899691A6895
:102BC00010B4CC0508D5140606D5446C44F00104B5
:102BD00044644FF48074DC614C0508D5140606D5B6
:102BE000446C44F0080444644FF48064DC6189055B
:102BF00008D5120606D5426C42F0020242644FF438
:102C00000072DA61416C11F00B0F02D010BCFFF7BB
:102C1000C7BD10BC704700002DE9F8430568D5F822
:102C20000090D0F82C8090F8417007F0F70720232F
:102C3000212F04460E46EB6164D148F20101FFF7F3
:102C4000ADFB27636B6843F400436B606B6823F054
:102C5000FF7323F48B3323F4FF7323F001036B60C2
:102C60002046FFF72FFB19F4804F50D02B6823F438
:102C700080432B60A36B1BB11B685B689BB26385B1
:102C800072070FD5636A6A6A1A70636A01336362F6
:102C9000238D2BB1013B2385638D013B9BB2638563
:102CA00026F00406638D9BB21BB1636C43F00403F2
:102CB0006364F30611D519F0100F0ED0638D9BB22B
:102CC000002B3ED194F84130282B29D1B8F1007F58
:102CD00026D131462046FFF719FD002384F8423003
:102CE000656C6363002D3BD0616C2046FFF758FD97
:102CF00094F84130282B45D131462046BDE8F843B1
:102D0000FFF704BD222F9DD148F2020197E719F485
:102D1000004FB5D02B6823F400432B60E36BAAE788
:102D200094F841202368292A4FF01002DA61D4D1A7
:102D300018F5803FD1D02046FFF7C4FAFFF76DFCAD
:102D4000CBE723681022DA61636C43F00403636409
:102D500038F08073C1D1616C2046FFF721FDBCE7DC
:102D6000E36A13F5803F0FD02046FFF756FC0F4B68
:102D7000E362202384F8413084F8405025632046E4
:102D80000CF044F9BDE8F88394F8413084F84050E1
:102D9000222B4FF0200384F841302046256302D1D6
:102DA0000CF049F9EEE70CF059F9EBE70000FFFFF2
:102DB00070B590F84060C56A012E04460B4670D08D
:102DC000012680F840608E0607D5960605D5FFF7E8
:102DD00023FF002084F8400070BDD80659D5D106E5
:102DE00057D512F4404F50D0D4E90E10E0B921B1BC
:102DF000520402D50A6852680AB323681022DA61C5
:102E0000636C43F00403636494F8413035F08072DE
:102E1000DBB2DED1213B092B30D8DFE803F02D34C3
:102E20002F2F2F2F2F2F2D341604E0D50068406848
:102E30000028DCD119B1500444BF0A68526894F8E4
:102E40004120282A07D1B5F1007F04D11946204638
:102E5000FFF75CFCBDE794F841202368292A4FF076
:102E60001002DA61B5D115F5803FB2D02046FFF7E8
:102E700029FAFFF7D2FBACE721232363616C2046DC
:102E8000FFF78EFCA5E72223F7E723681022DA611B
:102E90009FE719079DD513079BD52046FFF7F3FB46
:102EA00097E7022098E770B590F84060C56A012E58
:102EB00004460B467ED0012680F840608E0607D57A
:102EC000960605D5FFF7A8FE002084F8400070BDE7
:102ED000D90630D5D6062ED5628D92B2E2B994F8D5
:102EE0004120282A07D1B5F1007F04D11946204698
:102EF000FFF70CFCE8E794F841202368292A4FF0FB
:102F00001002DA61E0D115F5803FDDD02046FFF7F1
:102F1000D9F9FFF782FBD7E723681022DA61636CE7
:102F200043F00403636435F08073CDD1616C2046B7
:102F3000FFF736FCC8E758071BD5510719D5638D35
:102F40009BB26BB123685A6A636A1A70636A013371
:102F50006362238D013B2385638D013B9BB26385B7
:102F6000638D9BB2002BAFD115F5803FACD02046CE
:102F7000CFE71E0705D5100703D52046FFF783FBD3
:102F8000A2E79907A0D593079ED5638D9BB26BB13D
:102F9000636A226813F8011B91626362638D013BCF
:102FA0009BB26385238D013B23858DE735F08073CC
:102FB0008AD1DCE702208AE7806A836B0BB10022AA
:102FC0009A63C36B0BB100229A63FFF7D2BB000078
:102FD000024A136843F4807313607047000400587A
:102FE000024B186800F4C060704700BF000400582E
:102FF000024A936823F4004393607047000400582A
:10300000054A136843F007031360044A136943F049
:103010000403136130BF70470004005800ED00E066
:103020004FF0B0431868C0F3404070474FF0B043D2
:103030001868C0F3400070474FF0B042536823F463
:103040007F4343EA0023536070474FF0B043186852
:10305000C0F34060704700007FB54FF0B0432C4A8A
:10306000D3F80831C0F3031003F00F0352F82040E7
:10307000284A52F82330B4FBF3F4FFF7B1FF264B94
:10308000054693E80700B5F5007F04AB03E90700A8
:1030900010D0224B9C4218D303F5B70303F67F539D
:1030A0009C4229D903F5741303F510639C4225D87B
:1030B00002230BE01A4B9C4207D91A4B9C421BD9A6
:1030C00003F5370303F5D853F0E7002304AA02EB16
:1030D000830353F80C4C144D2B6823F00703234350
:1030E0002B60FEF77FF906462B6803F007039C422E
:1030F00006D1002004B070BD0123E7E70024EAE711
:10310000FEF770F9801B0228EED90320F2E700BF1A
:10311000383B0208983B020880350208C0CF6A009D
:10312000BFEA21013F933402004000584FF0B04302
:1031300010B59A68D96812F00C0205D00C2A4AD151
:1031400001F00303012B51D14FF0B0412B480B6824
:1031500013F0080306D00B6813F0080337D1D1F839
:10316000941007E00C68240756BFD1F89430096822
:10317000C3F3032350F82330002A0CBF1846002065
:103180004FF0B0418A6802F00C020C2A1ED1CA68C6
:1031900002F00302022A2ED0032A06D10B68184A35
:1031A00013F4801F174B18BF13464FF0B042D0687E
:1031B000D168D268C0F306205843C1F3021301332B
:1031C000B0FBF3F0530F0133B0FBF3F010BD0B680D
:1031D000C3F30313CEE7042A05D0082A06D11B68DF
:1031E00013F4801305D006480023C9E700231846CE
:1031F000C6E70448C4E7024BD7E700BF383B0208E4
:103200000024F4000048E80108B5FFF78FFF4FF0F5
:10321000B043044A9B68C3F3031352F82330B0FB56
:10322000F3F008BD983B02082DE9F0410446002860
:1032300053D04FF0B0439D68DE680368990605F0EF
:103240000C0506F0030668D5026A1DB10C2D46D1A7
:10325000012E44D1002A40D04FF0B043A16A1A6831
:10326000120756BFD3F894301B681B0903F0F00314
:1032700099421FD90846FFF7EFFE00282DD14FF0E5
:10328000B042136843F0080313601368A16A23F087
:10329000F0030B431360606AFFF7CEFEFFF7B4FF45
:1032A000AC4B1860AC4B1868FEF754F8002834D0CB
:1032B000BDE8F0814FF0B042136843F0080313609B
:1032C000136823F0F0030B431360606AFFF7B4FE4A
:1032D0000846FFF7C1FE0028E0D00120E8E74FF0E4
:1032E000B043002A54D01A6842F001021A60FEF777
:1032F00079F80746FFF79AFE002842D04FF0B04217
:10330000136843F0080313601368A16A23F0F00305
:103310000B431360606AFFF78FFE2368DF0748D412
:103320002368980700F1A18023681E0740F1FC8004
:10333000A3694FF0B046002B00F0E380D6F894303C
:10334000E16903F01002914200F0C68003F003022D
:10335000022AC2D0D80740F1B580D6F8943023F0C5
:103360000103C6F89430FEF73DF80746D6F89430CE
:10337000990740F1A780FEF735F8C31B112BF5D94B
:1033800004E0FEF72FF8C01B0228B3D903208FE713
:103390001A6822F001021A60FEF724F80746FFF7C8
:1033A00045FE0028B9D0FEF71DF8C01B0228F6D94B
:1033B000ECE7082D626803D00C2D1AD1032E18D12A
:1033C000002A8AD09907AFD523694FF0B046002B69
:1033D00067D0336843F480733360FEF703F8074621
:1033E00033685A0555D4FDF7FDFFC31B022BF7D9EF
:1033F000CCE74FF0B043A068196821F48011014375
:10340000B2F5803F196010D11A6842F480321A6018
:10341000FDF7E8FF0746FFF703FE002880D1FDF720
:10342000E1FFC01B6428F6D9B0E7B2F5041F04D150
:103430001A6842F400121A60E6E7196821F4803134
:103440001960196821F400111960002AE0D1FDF714
:10345000C9FF0746FFF7E4FD00283FF461AFFDF721
:10346000C1FFC01B6428F5D990E7042D03D00C2DB3
:10347000AAD1022EA8D12369002B3FF42EAF4FF022
:10348000B0426169536823F0FE4343EA016353602D
:103490004AE77368626923F0FE4343EA026373609C
:1034A00042E7336823F480733360FDF79BFF0746E0
:1034B00033685B057FF538AFFDF794FFC31B022B24
:1034C000F6D963E74FF0B042E169D2F8943023F0C7
:1034D00010030B43C2F894304FF0B047D7F8943044
:1034E00043F00103C7F89430FDF77CFF0646D7F898
:1034F00094309A0718D4FDF775FF831B112BF6D96A
:1035000044E7D6F8943023F00103C6F89430FDF771
:1035100069FF0746D6F894309B0705D5FDF762FF93
:10352000C31B112BF6D931E72368580754D50B4F2D
:103530003B68D90514D4FFF74BFDFDF753FF064652
:103540003B68DA050CD4FDF74DFF831B022BF7D93E
:103550001CE700BF400000200400002000040058C9
:10356000E3684FF0B046002B58D023F08003052BC2
:1035700002BFD6F8903043F00403C6F890304FF005
:10358000B046FDF72FFFD6F8903043F00103074611
:10359000C6F8903041F28838D6F890309B0705D4B1
:1035A000FDF720FFC31B4345F6D9EFE6E36823F0A0
:1035B0000403812B1BD1FDF715FFD6F8903043F0A3
:1035C0008003C6F8903007464FF0B04641F2883885
:1035D000D6F89030180504D5E36A002B4AD10020B4
:1035E00066E6FDF7FFFEC01B4045F1D9CEE6FDF7CC
:1035F000F9FED6F8903023F08003C6F890300746E5
:103600004FF0B04641F28838D6F890301905E3D52E
:10361000FDF7E8FEC01B4045F6D9B7E6FDF7E2FE30
:10362000D6F8903023F080030746C6F8903041F278
:103630008838D6F890301A0516D4FDF7D3FED6F8A0
:10364000903023F00103C6F8903007464FF0B048A1
:1036500041F28836D8F890309B07BDD5FDF7C2FE01
:10366000C31BB342F6D991E6FDF7BCFEC01B404533
:10367000DFD98BE60C2D4ED0022B4FF0B0431A68E9
:1036800022F080721A6033D1FDF7ACFE0546FFF7D9
:10369000DCFC38BBD4E90C314FF0B0420B43D068AE
:1036A0002D4901400B43E16B0B43216C0B43616CD3
:1036B0000B43A16B43EA0123D360136843F080738B
:1036C0001360D36843F08053D360FDF78BFE04464C
:1036D000FFF7BBFC002882D1FDF784FE001B0A28FF
:1036E000F6D953E6FDF77EFE401B0A28CFD94DE6FA
:1036F000FDF778FE0446FFF7A8FC30B94FF0B04262
:10370000164BD1680B40D36069E7FDF76BFE001BD9
:103710000A28F0D93AE6012B3FF4DFAD4FF0B04371
:10372000D868236B00F003029A427FF4D6AD626B37
:1037300000F0700393427FF4D0ADA26B00F4FE431F
:10374000B3EB022F7FF4C9AD636C00F06040C01A88
:1037500018BF0120ACE500BF8C80C111FCFFFEEE5C
:103760002DE9F0410D46044610B90120BDE8F08175
:10377000684E336803F007038B4216D323689A0719
:1037800027D54FF0B047A268BB6823F0F00313437E
:10379000BB60FDF727FE0646BB68DB0319D4FDF7C7
:1037A00021FE831B022BF7D911E0336823F00703B6
:1037B0000B433360FDF716FE0746336803F007033B
:1037C000AB42DBD0FDF70EFEC01B0228F5D903206B
:1037D000CCE72368580617D54FF0B0476269D7F891
:1037E000083123F00F0343EA1213C7F80831FDF73D
:1037F000F9FD0646D7F80831D90305D4FDF7F2FDE7
:10380000831B022BF6D9E2E723685A0713D54FF042
:10381000B047E268BB6823F4E0631343BB60FDF785
:10382000E1FD0646BB689B0305D4FDF7DBFD831B6A
:10383000022BF7D9CBE72368180714D54FF0B04710
:103840002269BB6823F4605343EAC203BB60FDF7FF
:10385000C9FD0646BB68590305D4FDF7C3FD831BAC
:10386000022BF7D9B3E72368DA070FD4294C236872
:1038700003F00703AB4239D8FFF7C6FC264B1860AC
:10388000264BBDE8F0411868FDF764BD6268022A66
:103890001DD1FFF7C5FB00283FF467AF4FF0B046DE
:1038A00041F28838B36823F003031343B360FDF794
:1038B00099FD0746B368626803F00C03B3EB820F0F
:1038C000D4D0FDF78FFDC01B4045F3D97FE7032A15
:1038D00002D1FFF7BAFBDEE712B9FFF7A7FBDAE781
:1038E0004FF0B0431B685B05D8D43EE7236823F054
:1038F00007032B432360FDF775FD0646236803F09D
:103900000703AB42B8D0FDF76DFD801B0228F5D947
:103910005DE700BF00400058400000200400002088
:1039200008B5FFF703FC4FF0B043054AD3F8083160
:1039300003F00F0352F82330B0FBF3F008BD00BFD3
:10394000983B020808B5FFF75FFC4FF0B043044A0C
:103950009B68C3F3022352F82330D84008BD00BF50
:10396000783B020808B5FFF74FFC4FF0B043044A1C
:103970009B68C3F3C22352F82330D84008BD00BF70
:10398000783B020810B5D8B1D1B14F234FF0B04207
:103990000360936803F00C04446003F0F004846057
:1039A00003F4E06403F46053C4600361D2F80831A7
:1039B0001B01DBB24361034B1B6803F007030B6081
:1039C00010BD00BF00400058704770B50446002885
:1039D00066D0436A002B5FD14268B2F5827F00D087
:1039E000C3610023A36294F85D3003F0FF0223B9A2
:1039F00084F85C202046FFF7E7FF2268E068A668AD
:103A0000A169022384F85D30136823F0400313603A
:103A1000B0F5E06F4FF000038ABF1D464FF48055AC
:103A2000B0F5706F18BFA362636806F4044603F430
:103A300082733343266906F002063343666906F053
:103A40000106334301F400763343E66906F0380695
:103A50003343266A06F080063343A66A06F400560E
:103A600033431360666B636A06F0080603F01003C5
:103A700000F470603343090C034301F004010B436D
:103A80002B435360D36923F40063D36100200123E7
:103A9000206684F85D3070BD0023C0E90433A0E7E0
:103AA0000120F8E7704710B5044680B10268022390
:103AB00080F85D30136823F040031360FFF7F2FFD6
:103AC0000020206684F85C0084F85D0010BD0120B1
:103AD000FCE7022310B580F83D300368196A41F213
:103AE00011121142044608D1196A40F244421142AF
:103AF00002BF1A6822F001021A60204602F0FBFCA5
:103B0000002084F8480084F83C0084F83E0084F8E3
:103B10003F0084F8400084F8410084F8420084F8B3
:103B2000430084F8440084F8450084F8460084F893
:103B3000470084F83D0010BD90F83D30012B17D1AF
:103B400002230C4A80F83D300368934202D0B3F15F
:103B5000804F07D19968084A0A40062A06D0B2F574
:103B6000803F03D01A6842F001021A6000207047BB
:103B700001207047002C0140070001000368196A0A
:103B800041F21112114208D1196A40F24442114225
:103B900002BF1A6822F001021A60012380F83D304A
:103BA000002070470368DA6822F00102DA60196ABF
:103BB00041F21112114208D1196A40F244421142F5
:103BC00002BF1A6822F001021A60012380F83D301A
:103BD0000020704790F83C20012A03464FF0020075
:103BE00009D01A6883F83D0051610020012283F852
:103BF0003D2083F83C00704770477047036870B5FC
:103C0000DD681E69B20704460DD5A9070BD56FF014
:103C100002021A61012202779B699A0774D001F0AF
:103C200052FE00232377730710D568070ED523684B
:103C30006FF004021A61022222779B6913F4407F1D
:103C4000204667D001F03FFE0023237731070FD5D0
:103C50002A070DD523686FF008021A610422227723
:103C6000DB699B0720465BD001F02DFE0023237704
:103C7000F00610D5E9060ED523686FF010021A6120
:103C800008222277DB6913F4407F20464ED001F0F2
:103C90001AFE00232377F20708D5EB0706D5236821
:103CA0006FF001021A61204601F0EAFD300608D5E6
:103CB000290606D523686FF080021A61204600F0BD
:103CC00002FAF20508D52B0606D523686FF4807238
:103CD0001A61204600F0F8F9700608D5690606D585
:103CE00023686FF040021A612046FFF786FFB20694
:103CF00022D5AB0620D523686FF0200220461A613A
:103D0000BDE8704000F0DEB901F0DBFD2046FFF7B2
:103D100073FF86E701F0D5FD2046FFF76DFF93E7BF
:103D200001F0CFFD2046FFF767FF9FE701F0C9FDD7
:103D30002046FFF761FFACE770BD00001B4A036837
:103D4000904202D0B0F1804F08D14A6823F070034E
:103D50001343CA6823F44073134306E0144A9042A5
:103D6000F7D002F580629042F3D04A6923F08003D5
:103D7000134303608B68C3620B6883620B4B9842EA
:103D800007D003F5C053984203D003F580639842EF
:103D900001D10B690363012343610369DB0742BF60
:103DA000036923F001030361704700BF002C014049
:103DB0000044014010B5044650B390F83D3003F084
:103DC000FF021BB980F83C2002F06EFB0223206842
:103DD00084F83D30211DFFF7B1FF012384F84830FE
:103DE000002084F83E3084F83F3084F8403084F876
:103DF000413084F8423084F8433084F8443084F809
:103E0000453084F8463084F8473084F83D3010BDA2
:103E10000120FCE7036A01F01F0110B501248C406A
:103E200023EA04030362036A8A401A43026210BD54
:103E3000082908B525D00AD8A9B1042919D090F8C5
:103E40004330012B13D1022380F843302CE00C299E
:103E50001FD01029F3D190F84230012B07D1022353
:103E600080F8423020E090F83E30012B19D001203C
:103E700043E090F83F30012BF9D1022380F83F3026
:103E800012E090F84030012BF1D1022380F840304D
:103E90000AE090F84130012BE9D1022380F841304B
:103EA00002E0022380F83E3000680122FFF7B2FFF3
:103EB000124B984214D003F5C05398420BD003F52F
:103EC0008063984207D0B0F1804F0DD0036843F073
:103ED0000103036010E0436C43F400434364F5E7DF
:103EE000436C43F4004343648268054B1340062B44
:103EF00002D0B3F5803FE9D1002008BD002C01407D
:103F000007000100FFF794BF082910B503465AD0F7
:103F100010D809B3042946D093F8434093F84720BA
:103F2000012CE0B2D2B26FD1012A3BD1022283F838
:103F3000432065E00C2956D01029EDD190F842407D
:103F400093F84720012CE0B2D2B25DD1012A29D1E9
:103F5000022283F8422053E090F83E4093F8442038
:103F6000012CE0B2D2B24FD1012A1BD1022283F838
:103F70003E2083F8442018680122FFF74BFF234BB3
:103F8000984202D0B0F1804F07D18268204B134095
:103F9000062B06D0B3F5803F03D0036843F001033E
:103FA0000360002010BD90F83F4093F84520012C9D
:103FB000E0B2D2B228D1012AF4D1022283F83F2004
:103FC00083F84520D7E790F8404093F84620012C2D
:103FD000E0B2D2B218D1012AE4D1022283F8402003
:103FE00083F84620C7E790F8414093F84720012C1A
:103FF000E0B2D2B208D1012AD4D1022283F8412002
:10400000022283F84720B6E70120CBE7002C0140CD
:1040100007000100036A01F01F0110B504248C4061
:1040200023EA04030362036A8A401A43026210BD52
:1040300008B529B990F84430012B1DD0012039E092
:10404000042907D190F84530012BF7D1022380F8DD
:10405000453014E0082907D090F84730012BEDD106
:10406000022380F847300AE090F84630012BE5D172
:10407000022380F8463002E0022380F844300068D2
:104080000422FFF7C7FF436C43F4004343640A4B29
:10409000984202D0B0F1804F07D18268074B13409D
:1040A000062B06D0B3F5803F03D0036843F001032D
:1040B0000360002008BD00BF002C01400700010084
:1040C000FFF7B6BF704770477047000010B5026831
:1040D00052E8003F23F4907342E80031026800295F
:1040E000F5D10F4C02F1080353E8003F234002F1E1
:1040F000080C4CE800310029F4D1C36E012B07D124
:1041000052E8003F23F0100342E800310029F7D1C4
:104110002023C0F88C300023C366436710BD00BF66
:10412000FEFFFFEF026852E8003F23F0800342E801
:10413000003102680029F5D152E8003F43F0400306
:1041400042E800310029F7D17047D0F88820212AB1
:10415000034611D1B0F8562092B20AB9FFF7E2BF78
:10416000026D016812F8010B88621A65B3F85620D7
:10417000013A92B2A3F856207047D0F88820212A3D
:10418000034613D1B0F8562092B20AB9FFF7CABF5E
:104190001A6D006832F8021BC1F3080181621A65CA
:1041A000B3F85620013A92B2A3F856207047D0F8DF
:1041B0008830212B10B51BD1B0F86A20C2B1B0F8FD
:1041C0005610036889B2A1B903F1080252E8002F22
:1041D00022F4000203F1080040E800210029F3D195
:1041E00053E8002F42F0400243E800210029F7D1B4
:1041F00010BDD96909060AD5016D11F8014B9C6201
:10420000B0F856300165013B9BB2A0F85630013A38
:1042100092B2D3E7D0F88830212B10B51BD1B0F87B
:104220006A20C2B1B0F85610036889B2A1B903F18F
:10423000080252E8002F22F4000203F1080040E8CF
:1042400000210029F3D153E8002F42F0400243E857
:1042500000210029F7D110BDD96909060CD5016DDF
:1042600031F8024BC4F308049C62B0F85630016583
:10427000013B9BB2A0F85630013A92B2D1E77047A9
:10428000D0F88830202B10B544D1002944D0002A22
:1042900042D0A0F85620A0F85420426E01650023B9
:1042A000C0F89030B2F1005F4FF02103C0F88830C1
:1042B0000268836819D1B3F5805F14D10469174B84
:1042C0001749002C08BF0B46836702F1080353E827
:1042D000003F43F4000302F1080040E800310029E8
:1042E000F3D1002010BD0D4BEEE7B3F5805F0FD189
:1042F00004690C4B0C49002C08BF0B46836752E83D
:10430000003F43F0800342E800310029F7D1E8E79D
:10431000044BF3E70220E5E70120E3E7AF410008A3
:10432000154200084B4100087B41000808B5806A2F
:104330000023A0F85E30A0F8563002F011FC08BD52
:10434000704700000368D9691A682DE9F04140F60A
:104350000F0631429D68044610D18E0640F19780C9
:1043600002F0200605F080573E4300F09080436F36
:10437000002B00F08580BDE8F0411847AB4EAC48FB
:104380002E401040304300F08280CF0709D5D00581
:1043900007D501201862D4F8900040F00100C4F85D
:1043A00090008F0709D5E80707D502201862D4F8D6
:1043B000900040F00400C4F890004F0709D5E807CA
:1043C00007D504201862D4F8900040F00200C4F829
:1043D00090000F070BD502F02000304307D00820D3
:1043E0001862D4F8900040F00800C4F890000E0560
:1043F0000AD5500108D54FF400601862D4F8903007
:1044000043F02003C4F89030D4F89030002B37D01C
:104410008B0609D502F0200205F080552A4303D00F
:10442000636F0BB1204698472668D4F89020B36894
:1044300002F0280203F0400353EA0205204621D08F
:10444000FFF744FEB3685F0617D5226802F1080340
:1044500053E8003F23F04003083242E800310029CE
:10446000F3D1D4F8800040B1724B8363FDF73AFD7D
:1044700030B1D4F88000836B7DE7204602F070FBFA
:10448000BDE8F08102F06CFBC4F89050F8E7E06EF4
:10449000012840F08980CE0640F18680D00640F1A8
:1044A000838010221A629A6851064BD5D4F8802076
:1044B00011684A6892B2002AE2D0B4F85C009042D7
:1044C000DED9A4F85E200A6892062FD453E8002FA4
:1044D00022F4807243E800210029F7D103F1080299
:1044E00052E8002F22F0010203F1080040E8002109
:1044F0000029F3D103F1080252E8002F22F0400214
:1045000003F1080040E800210029F3D12022C4F87B
:104510008C20E16653E8002F22F0100243E80021CE
:104520000029F7D1D4F88000FDF7A7FC0223236708
:10453000B4F85E30B4F85C10C91A89B22046FFF7AF
:10454000FFFE9DE7B4F85E20B4F85E00B4F85C109E
:1045500080B292B2002893D0891A89B200298FD0F4
:1045600053E8002F22F4907243E800200028F7D18E
:10457000314D03F1080252E8002F2A4003F10806EA
:1045800046E800200028F4D12022C4F88C2060677F
:10459000E06653E8002F22F0100243E800200028D4
:1045A000F7D102232367C9E7CF0209D56E0207D5E9
:1045B0004FF4801220461A62BDE8F04102F01ABBA7
:1045C00008060BD502F0800005F40005284305D04D
:1045D000A36F002B3FF454AF2046CCE64F0611D515
:1045E00056060FD553E8002F22F0400243E8002181
:1045F0000029F7D12023C4F88830A167204602F0B3
:10460000ABFA3DE70D0206D5500004D52046BDE8C3
:10461000F04100F032BECB017FF532AF002ABFF689
:104620002FAF2046BDE8F04100F026BE010000108B
:10463000200100042D430008FEFFFFEFD0F88C207E
:10464000B0F86010222A08B5036855D15B6A826D04
:104650000B401370836D01338365B0F85E30013B0E
:104660009BB2A0F85E30B0F85E309BB2002B42D116
:10467000026852E8003F23F4907342E80031036877
:104680000029F5D103F1080252E8002F22F00102BF
:1046900003F1080C4CE800210029F3D12022C0F8D6
:1046A0008C20184A41679342016705D1C26E012AE6
:1046B0000ED002F04DFA1EE05A681102F6D553E80A
:1046C000002F22F0806243E800210029F7D1EDE7B6
:1046D0000022C26653E8002F22F0100243E80021B6
:1046E0000029F7D1DA69B0F85C10D20644BF102275
:1046F0001A62FFF725FE08BD9A6942F008029A6126
:10470000F9E700BF00800040D0F88C20B0F86010BE
:10471000222A08B5036852D15A6A1140826D22F8E4
:10472000021B8265B0F85E20013A92B2A0F85E20CA
:10473000B0F85E2092B2002A40D153E8002F22F454
:10474000907243E800210029F7D103F1080252E8F2
:10475000002F22F0010203F1080C4CE8002100298F
:10476000F3D12022C0F88C20174A41679342016799
:1047700005D1C26E012A0ED002F0EAF91EE05A6895
:104780001102F6D553E8002F22F0806243E80021A1
:104790000029F7D1EDE70022C26653E8002F22F08E
:1047A000100243E800210029F7D1DA69B0F85C1063
:1047B000D20644BF10221A62FFF7C2FD08BD9A69F3
:1047C00042F008029A61F9E7008000402DE9F84FB5
:1047D0000368B0F86060D3F81CB01F689D68D0F81B
:1047E0008C20222A044640F0B980B0F8683043B1EA
:1047F000DFF87491DFF874A14FF000081BF0200F70
:1048000020D1B4F85E309BB2D3B1B4F868209A429C
:1048100016D9226802F1080353E8003F23F08053C1
:10482000083242E8003122680029F2D1504B636718
:1048300052E8003F43F0200342E800310029F7D15D
:10484000BDE8F88F2368A26D5B6A33401370A36DD7
:104850000133A365B4F85E30013B9BB2A4F85E302F
:104860002368D3F81CB01BF0070F2ED01BF0010FEC
:1048700009D0F90507D501221A62D4F8902042F038
:104880000102C4F890201BF0020F09D0EA0707D5F7
:1048900002221A62D4F8902042F00402C4F8902058
:1048A0001BF0040F09D0E80707D504221A62D4F8D8
:1048B000903043F00203C4F89030D4F8903023B124
:1048C000204602F04DF9C4F89080B4F85E309BB2F7
:1048D000002B93D1226852E8003F23F4807342E812
:1048E000003123680029F5D103F1080252E8002FB6
:1048F00002EA090203F1080040E800210029F3D18F
:1049000020225345C4F88C20616721670AD05A6879
:10491000110207D553E8002F22F0806243E80021FE
:104920000029F7D1E26E012A14D10022E26653E891
:10493000002F22F0100243E800210029F7D1DA69A4
:10494000B4F85C10D20644BF10221A622046FFF76A
:10495000F7FC53E7204602F0FBF84FE79A6942F074
:1049600008029A616CE700BFFEFFFFEF0080004085
:104970003D4600082DE9F84F0368B0F86060D3F8B1
:104980001CB01F689D68D0F88C20222A044640F095
:10499000B780B0F8683043B1DFF87091DFF870A1EC
:1049A0004FF000081BF0200F20D1B4F85E309BB20E
:1049B000D3B1B4F868209A4216D9226802F10803EC
:1049C00053E8003F23F08053083242E80031226868
:1049D0000029F2D14F4B636752E8003F43F02003B8
:1049E00042E800310029F7D1BDE8F88F2368A26DB5
:1049F000596A314022F8021BA265B4F85E20013AE0
:104A000092B2A4F85E20D3F81CB01BF0070F2ED092
:104A10001BF0010F09D0F90507D501221A62D4F85D
:104A2000902042F00102C4F890201BF0020F09D040
:104A3000EA0707D502221A62D4F8902042F0040255
:104A4000C4F890201BF0040F09D0E80707D5042212
:104A50001A62D4F8903043F00203C4F89030D4F8CE
:104A6000903023B1204602F07BF8C4F89080B4F86F
:104A70005E309BB2002B95D1226852E8003F23F4B0
:104A8000807342E8003123680029F5D103F1080260
:104A900052E8002F02EA090203F1080040E8002171
:104AA0000029F3D120225345C4F88C206167216787
:104AB0000AD05A68110207D553E8002F22F080620D
:104AC00043E800210029F7D1E26E012A14D1002227
:104AD000E26653E8002F22F0100243E8002100298B
:104AE000F7D1DA69B4F85C10D20644BF10221A621A
:104AF0002046FFF725FC55E7204602F029F851E74C
:104B00009A6942F008029A616EE700BFFEFFFFEF6C
:104B1000008000400947000810B590F88430012B50
:104B20001ED0012380F884302423C0F88830026826
:104B300052E8003F23F00C0342E800340168002CE7
:104B4000F5D151E8002F42F0080241E80023002B84
:104B5000F7D12022C0F8882080F88430184610BD94
:104B60000220FCE710B590F88430012B1ED0012301
:104B700080F884302423C0F88830026852E8003F6F
:104B800023F00C0342E800340168002CF5D151E811
:104B9000002F42F0040241E80023002BF7D120222D
:104BA000C0F8882080F88430184610BD0220FCE749
:104BB000D0F88820D0F88C001043704738B50446F0
:104BC00003682169A2681D68C0690A4361690A43D4
:104BD0007549024329400A431A605A68E16822F481
:104BE00040520A435A60714AA16993421CBF226A2B
:104BF00011439A6822F06E4222F430620A439A60AE
:104C0000DA6A616A22F00F020A43DA62684A934262
:104C100017D14FF0B043674AD3F8883003F003034D
:104C200043F4403393425BD0B3F1031F21D0013AE8
:104C3000934274D0B0F5004F40F0B080FEF792FE82
:104C400031E05D4A934231D14FF0B0435B49D3F834
:104C5000883003F00C0343F440228A4240D005D848
:104C6000E3B1574B9A425AD0012062E0B2F10C1FD7
:104C7000FAD1B0F5004F37D04FF400406368616A55
:104C8000504A32F81120B0FBF2F000EB5300B0FBB9
:104C9000F3F04FF6EF73A0F1100274E0B0F5004F9F
:104CA00077D1FEF74FFE002842D01DE03F4A9342E5
:104CB000DAD14FF0B043D3F8883003F44063B3F552
:104CC000006F3DD006D883B3B3F5806FCCD1FEF72B
:104CD0002DFA2CE0B3F5406FC6D14FF4004030E020
:104CE000B0F5004F3848C9D16268616A354B33F876
:104CF0001130B0FBF3F0530803EB4003B3FBF2F3C6
:104D00004FF6EF72A3F110019142ADD823F00F02DC
:104D1000216892B2C3F342031343CB6008E0B0F5BD
:104D2000004F3ED1FEF702FABDE7FEF70BFE40B999
:104D300000204FF00113A3660023C4E91D3338BDE2
:104D4000214865681F4B626A05EB450133F8122064
:104D5000B0FBF2F3994287D8B3EB053F84D8002328
:104D60001946FCF721FA090241EA10616B080002BA
:104D7000C0182A464FF0000341F10001FCF714FA75
:104D8000124BA0F540729A423FF66EAF2368D8608E
:104D9000CEE7FEF7D7FD0028CAD06FE7FEF7E2FDA9
:104DA000F9E7FEF7C3F9F6E7F369FFCF00800040AB
:104DB00000380140020003000044004008000C00DD
:104DC00004000C003C3A02080024F400FFFC0F0031
:104DD000836A1A0710B506D50168846B4A6822F405
:104DE000004222434A60DC0706D50168C46A4A686B
:104DF00022F4003222434A60990706D50168046B09
:104E00004A6822F4803222434A605A0706D5016874
:104E1000446B4A6822F4802222434A60DC0606D5AD
:104E20000168C46B8A6822F4805222438A60990622
:104E300006D50168046C8A6822F4005222438A6015
:104E40005A060FD50168446C4A6822F48012224346
:104E5000B4F5801F4A6005D14A68846C22F4C00210
:104E600022434A601B0606D50268C16C536823F4CE
:104E700000230B43536010BD2DE9F843DDF820906B
:104E800005460E46174698462A68D36936EA030354
:104E90000CBF01230023BB4201D0002029E0B9F15F
:104EA000FF3FF2D0FCF79EFAA0EB080048452C68C3
:104EB00002D8B9F1000F1ED154E8003F23F4D0739B
:104EC00044E80032002AF7D104F1080353E8003F18
:104ED00023F0010304F1080141E80032002AF3D174
:104EE0002023C5F88830C5F88C30002385F884303D
:104EF0000320BDE8F88323685A07C5D5802EC3D0A8
:104F0000402EC1D0E3691B05BED54FF40063236278
:104F100054E8003F23F4D07344E80032002AF7D16C
:104F200004F1080353E8003F23F0010304F10801F2
:104F300041E80032002AF3D12023C5F88830C5F8B3
:104F40008C30C5F89030D0E72DE9F7439846D0F87B
:104F50008830202B04460E46174643D1002943D003
:104F6000002A41D021230025C0F89050C0F8883095
:104F7000FCF738FAA368A4F85470B3F5805F814653
:104F8000A4F8567003D123690BB935461E46B4F810
:104F90005620CDF8008092B24B4642B940212046BF
:104FA000FFF76AFF48B92023C4F8883006E00022E2
:104FB00080212046FFF760FF18B1032003B0BDE851
:104FC000F08322685EB935F8023BC3F308039362AD
:104FD000B4F85620013A92B2A4F85620D7E716F852
:104FE000013BF4E70220E9E70120E7E773B5044657
:104FF0000026C0F89060FCF7F5F923681B681A07D3
:10500000054619D423681B685B070AD56FF07E43F9
:10501000009300222B464FF480012046FFF72CFF1F
:10502000B0B900202023C4F8883084F88400C4F884
:105030008C30E06620670CE06FF07E4300933246D0
:1050400003464FF400112046FFF716FF0028D9D081
:10505000032002B070BD10B5044650B3D0F88830BC
:105060001BB980F88430FFF70AF922682423C4F8BA
:105070008830136823F001031360A36A13B120463C
:10508000FFF7A6FE2046FFF799FD012811D02368FF
:105090005A6822F490425A609A6822F02A029A6072
:1050A0001A6842F0010220461A60BDE81040FFF77E
:1050B0009DBF012010BD10B5044670B3D0F88830F4
:1050C0001BB980F88430FFF7DAF822682423C4F88B
:1050D0008830136823F001031360A36A13B12046DC
:1050E000FFF776FE2046FFF769FD012815D02368FB
:1050F0005A6822F490425A609A6822F022029A601A
:105100009A6842F008029A601A6842F0010220464A
:105110001A60BDE81040FFF769BF012010BD000014
:1051200030B581658168A0F85C200023B1F5805F0F
:10513000A0F85E20436731D10369002B40F2FF13D2
:1051400018BFFF23A0F860300023C0F8903022235E
:10515000C0F88C30016801F1080353E8003F43F0C8
:105160000103083141E800340368002CF2D1456E98
:1051700084680169B5F1005F35D1B0F86850954297
:1051800031D8B4F5805F29D1C1B1264A426753E8CE
:10519000002F42F4807243E8002121E029B903691D
:1051A000002B14BF7F23FF23CCE7B1F1805FC9D16F
:1051B0000369002B14BF3F237F23C3E71A4A4267CA
:1051C00003F1080252E8002F42F0805203F1080078
:1051D00040E800210029F3D1002030BD114A426788
:1051E0000029D4D1ECE7B4F5805F16D151B10F4A54
:1051F000426753E8002F42F4907243E800210029EF
:10520000F7D1E9E70A4A426753E8002F42F020024B
:1052100043E800210029F7D1DEE7044A426700296C
:10522000F2D0E6E7CD470008754900083D46000882
:1052300009470008D0F88C30202B30B415D1B9B113
:10524000B2B100230468C3660A4B9C420AD063686B
:105250001B0207D554E8003F43F0806344E8003563
:10526000002DF7D130BCFFF75BBF022030BC704788
:105270000120FBE7008000407047704790F88430C1
:10528000012B0FD0012380F88430016851E8002FF2
:1052900042F0020241E80023002BF6D180F884306E
:1052A000184670470220704790F88430012B0FD0C9
:1052B000012380F88430016851E8002F22F00202B7
:1052C00041E80023002BF6D180F88430184670475F
:1052D00002207047836810B504462BB103220146B3
:1052E00098470023C4E9023310BD836810B5044613
:1052F00013B1032201469847204610BD10B504465D
:1053000050F8103FDA6822F00102DA60DA6822F021
:105310000202DA60DA6822F00402DA60DA6822F067
:105320000802DA60DA6822F01002DA60FEF726FC82
:105330002269136823F001031360012384F84E30BF
:1053400084F84F3084F8503084F8513084F852306B
:1053500084F8533084F8543084F8553084F856304B
:1053600084F8573010BD4B1E032B00D9FEE789008F
:10537000081F70470139435C13F0100004D0022964
:1053800016D80C4A32F81100DB0712D503290FD8C2
:10539000DFE801F00205080B40F00100704740F023
:1053A0001000704740F48070704740F480507047A0
:1053B000FEE770475C3A02080139032900D9FEE78D
:1053C000014B585C704700BF583A02080139032965
:1053D00000D9FEE7014B585C704700BF543A020801
:1053E0002DE9F04104460E46FFF7BDFF04EB061819
:1053F00008F16408054631462046FFF7DDFFD8F87E
:1054000008302BB12369C2431A61DA680243DA60BB
:10541000771E04EB47039B880B2B49D8DFE803F08A
:1054200051181818060618184A4A4A2AE35DDE067B
:1054300004D5294604F11000FEF742FEE35DD807CB
:1054400036D5294604F11000BDE8F041FEF75ABDFB
:10545000E35DD90604D5294604F11000FEF7E8FD06
:10546000E35DDA0724D5294604F11000BDE8F041D8
:10547000FEF7DEBC294604F11000FEF745FD31467B
:105480002046FFF7A3FF2569014606462046FFF7A1
:1054900071FF2B6A1843D8F80830286243B13146AF
:1054A0002046FFF789FFC3432B61EB681843E86090
:1054B000BDE8F081294604F11000BDE8F041FEF797
:1054C00023BD23691B68DB07F2D404F11000BDE89B
:1054D000F041FEF731BB70B501250446861C294614
:1054E00036F8023F23B129462046FFF779FF002115
:1054F0000135052DF4D1E36E3BB123696FF0010254
:105500001A61DA6842F00102DA6049B123691B6866
:10551000DB0705D404F11000BDE87040FEF70CBBBA
:1055200070BD01211030FEF755BB0369186800F00B
:105530000100704710B502460C46FFF7F6FF80B930
:10554000CB68DB070ED5CB6823F00103CB60104698
:10555000FFF7E7FF6FF001032361E36843F0010306
:10556000E36010BDBDE810401046FFF7DABF000051
:105570000B4B98420BD0B0F1804F0AD003F5C053CB
:10558000984208D003F58063984206D0FEE70020D9
:10559000704701207047022070470320704700BF0A
:1055A000002C0140024670B5044652F8100FFFF778
:1055B000DFFF0546104600F009FF094A002342F8C4
:1055C000253004F16406E36004F1B405B54204D06B
:1055D000103D2846FFF789FEF8E7204670BD00BF62
:1055E0008803002070B504460846FFF7C1FF25690F
:1055F00005B1FEE7204B216104F10C0243F82020A5
:1056000004F110060E23C4E917353046C4E90C55E1
:10561000C4E90E55C4E9105584F82C50A56484F8EB
:105620004C5084F84D50E46000F0A4FE04F1640096
:10563000FFF750FE04F17400FFF74CFE04F1840004
:10564000FFF748FE04F19400FFF744FE04F1A400C4
:10565000FFF740FEC4E900554FF6FF73C4E9065357
:105660008023C4E90855A5606561A3623046BDE8A2
:105670007040FEF79FBB00BF8803002010B588B0C4
:1056800018220446002102A81BF053FF002301A9A1
:1056900002A80193FEF776F9206900F03DFF01288A
:1056A00002D002280FD0FEE7059CFEF74BF9B4F5B7
:1056B000C06F05D00BD824F48074B4F5806F00D18E
:1056C000400008B010BD069CFEF74CF9EFE7B4F5BA
:1056D000E06FF4E7012A38B505460C460BD0022AE4
:1056E00016D004B1013C29692846CC62EC61BDE8C2
:1056F0003840FFF71FBFFFF7C1FF084BB0FBF3F0C7
:1057000044432A69230C93620133B4FBF3F4E8E7C2
:10571000FFF7B4FFB0FBF4F4F3E700BF40420F0023
:1057200010B500F110042046FEF73CFA2046BDE813
:105730001040FEF7CEB90000034B186810B10430DA
:10574000FEF75CBA704700BF88030020FFF7F4BF84
:10575000034B586810B10430FEF750BA704700BFD1
:1057600088030020034B986810B10430FEF746BA56
:10577000704700BF88030020034BD86810B1043085
:10578000FEF73CBA704700BF880300200022C0E942
:105790000022C0E902227047F8B504460E4600F127
:1057A000640500F1B40728461035FFF7EFFFBD424E
:1057B000F9D10023204623613146FFF713FF20462D
:1057C000F8BD38B50023C0E90033C0E902338B6867
:1057D00004460D462BB102229847EB68E360AB68A4
:1057E000A360204638BD30B587B002AD04462846D8
:1057F000FFF7E7FF95E803006B4683E8030094E8B2
:10580000030085E8030093E80300049BA268A360FB
:10581000059B049284E80300E268E3602846059251
:10582000FFF763FD07B030BD38B504460D46E36EA3
:1058300064301BB1BDE83840FFF7D5BFFFF7D3FF99
:10584000AB683BB123696FF001021A61DA6842F07C
:105850000102DA6038BD826810B50AB918F03CFB65
:10586000BDE81040C368184708B500B9FEE700F06E
:105870007FFD0068C36E13B16430FFF7ECFF08BD15
:10588000FFF7F2BF10B500B9FEE7037F013B072B1E
:1058900010D8DFE803F004140F100F0F0F120124CB
:1058A00000F066FD240100686434204483680BB175
:1058B000FFF7D1FF10BD0324F2E70424F0E7022430
:1058C000EEE7FFF7DFBFFFF7DDBF1AF0E5BB1AF029
:1058D000E3BB1AF0E9BB4FF0B04382B0DA6C02438D
:1058E000DA64DB6C03400193019B02B07047000057
:1058F00008B5032818D8DFE800F002080D120120CF
:10590000FFF7E9FF4FF0904008BD0220FFF7E3FFEB
:105910000648F9E70420FFF7DEFF0548F4E780209A
:10592000FFF7D9FF0348EFE70020EDE70004004848
:1059300000080048001C004808B5064900F0E0FCDB
:10594000C0F3C430112800D9FEE7034B53F8200000
:1059500008BD00BF38390208703A0208A0F580502F
:105960000138022800D9FEE7014B53F820007047A8
:10597000643A020808B5054900F0C2FCC0F3C4301F
:10598000012800D0FEE7002008BD00BF2039020832
:105990000268094B9A420DD14FF0B0439A6B42F026
:1059A00000529A639A6B22F000529A639A6D22F029
:1059B00000529A65704700BF0074004010B50A4954
:1059C00086B0044600F07AFC019050B12046FFF703
:1059D000D1FF014628B901A8FCF741FA01A8FCF75C
:1059E00030FA06B010BD00BF203902084FF0B043B6
:1059F00082B01A6E42F400721A661A6E02F40072D5
:105A00000192019AD3F8882042F04052C3F88820CE
:105A1000044B1868C30403D4034902B000F036BC39
:105A200002B0704718000020383902084FF0B04328
:105A30001A6C42F400721A641A6C22F400721A642E
:105A40001A6C42F400721A641A6C22F400721A641E
:105A50001A6E22F400721A6670470000F0B59FB00B
:105A6000054664220E4605A800211BF062FD0023B6
:105A7000EA04CDE902330493ADF80230019340F11A
:105A8000AC8041F203039D4200F2A7805D4B059379
:105A90002846FFF763FF07270446082E00F0AE8074
:105AA0000A2E00F0AD80062E0CBF182300234FF005
:105AB0000042CDE906230023CDE908320422CDE9D6
:105AC0000E330A92ADF82C3001228DF82E308DF86D
:105AD00034308DF840308DF8503018931B93199363
:105AE0008DF86830484B0C9205A84FF48052CDE9F0
:105AF000112713971D60FBF77FFC002879D1012C3B
:105B0000029435D0414B9C4232D0414B9C422FD025
:105B1000404B9C422CD0404B9C4229D03F4B9C4256
:105B200026D03F4B9C4223D03E4B9C4220D03E4B44
:105B30009C421DD03D4B9C421AD03D4B9C4217D0FD
:105B400003F104239C4213D03A4A24F000439342C9
:105B50000ED0394A93420BD0384A934208D0384A83
:105B6000944205D0374A944202D0374A934240D1FA
:105B7000012302A905A8CDE90337FBF79BFD002807
:105B800037D105A8FBF7D0FF002832D105A8FBF7D5
:105B9000F3FE70BB0A2105A8FBF72EFD48BB05A844
:105BA000FBF760FE830505D505A8FBF77FFD80B2F6
:105BB000ADF8020005A8FBF799FFD0B905A8FBF7DF
:105BC0003FFFB0B9214AD2F8083723F0E073C2F89A
:105BD0000837BDF8020080B20CE01D49284600F0ED
:105BE0006DFB01A905902846FFF7A6FE059B04461C
:105BF00013B900201FB0F0BD03274EE7102356E76E
:105C0000082354E70024014018000020020000048B
:105C1000040000080800000C100000102000001410
:105C2000400000188000001C000100200002002439
:105C3000000400280010003000200034004000382C
:105C40000080003C000001400000024400200140B0
:105C500038390208F8B51449144E074600F02EFBF7
:105C6000FFF786FC56F82030044673B9B420FFF7DE
:105C70002CFE0D490546384600F020FB014628461B
:105C8000FFF78AFD56F824301D6056F824301C6852
:105C900044B12046FFF786FC2046B421BDE8F84019
:105CA000FFF717BEF8BD00BF3C380208880300208C
:105CB00037B5FBF797FB4FF0E0250446AB6900933F
:105CC000FBF790FBAB6901936969844201F1010123
:105CD0004FF47A7308D0019A8A1A5A43B2FBF1F250
:105CE00003FB002003B030BD009A8A1A5A43B2FB6E
:105CF000F1F203FB0420F5E7FBF774BB704708B52E
:105D0000FBF764FBFCF735F8FFF7F8FF08BD10B5AB
:105D100094B048220021044602A81BF00AFCFDF7BB
:105D200057F94FF0B0439A6D42F480629A659A6DCC
:105D300002F480620192019A032C11D8DFE804F08A
:105D40000219283DD3F8942042F00102C3F89420B0
:105D5000D3F894309C0703D40823029301230893BB
:105D6000029B002B36D002A8FDF75EFA002831D046
:105D7000FEE71A6842F480721A601B685905EFD476
:105D8000022302934FF480724023CDE90623E7E714
:105D9000D3F8902042F00102C3F89020D3F890206D
:105DA0009407DDD4D3F8902022F01802C3F8902095
:105DB0000423029381230593D2E71A6842F48032C8
:105DC0001A601B6899035EBF01224FF48033CDE94E
:105DD0000223C5E714B010BD70474FF0B04382B046
:105DE0001A6D42F400221A651A6D02F40022019223
:105DF000019A9A6C42F480529A649B6C03F480532B
:105E00000093009B02B070470C4BD3F8FC20D201EA
:105E10005EBFD3F8FC2042F08072C3F8FC20084B30
:105E200000225A601A6842F001021A6000BF00BFE7
:105E300000BF5868B0FA80F04009704700ED00E0FC
:105E4000001000E008B5FFF7C8FFFFF7DDFFFBF724
:105E5000A7FAFFF7C1FFFBF743FABDE80840014886
:105E6000FBF78CBF1C000020012A02D1016000203A
:105E70007047022A05D0032AF9D0002AF7D1026020
:105E8000F5E70B680360F2E7036818470023C0E9F1
:105E90000033C0E90233704770B50024012904F1D2
:105EA00001032CD1184DE4B2142161436E18F3683C
:105EB0003BB1043129440322084698470023C6E930
:105EC0000333142363430022E8560F4B93F9001069
:105ED000814201D1D968A9B90132102A03F1140312
:105EE000F4D10A4A0A49D2F8803051F8241023EA42
:105EF0000103BDE87040C2F88030FBF7F3BE4908EB
:105F00001C46CBE770BD00BF980300200008005876
:105F1000B83A02080023012803F101020AD1142231
:105F2000DBB25343054A181D1044816829B11A4455
:105F30001369184740081346EDE77047980300209F
:105F40000120FCF7B3B90220FCF7B0B90420FCF73C
:105F5000ADB90820FCF7AAB91020FCF7A7B938B5ED
:105F600005242025A8B2FCF7A1F9013C4FEA45051C
:105F7000F8D138BD38B506244FF48065A8B2FCF7D7
:105F800095F9013C4FEA4505F8D138BD2DE9F041BE
:105F900016468CB00A460024012A04F1010543D1BB
:105FA000E4B26200CDE90713C168DFF884800323FF
:105FB00093400B40D34003F0030303AD099307A9BB
:105FC00002230A93FCF7BEF81423314628465C43AB
:105FD000FFF7F7FB95E8030008EB040301AA04337D
:105FE00082E8030093E8030085E8030092E80300D9
:105FF000271D83E803004744059BBA68BB60069BE6
:1060000005922846FA68FB600692FFF76EF918F9C8
:10601000040000220621FBF725FE18F90400FBF717
:1060200053FE0CB0BDE8F08152082C46B4E700BF27
:1060300098030020344A104608B5062300F8043BB4
:10604000FFF724FF072302F118001375FFF71EFF67
:10605000082302F12C0082F82830FFF717FF0923EC
:1060600002F1400082F83C30FFF710FF0A2302F1F2
:10607000540082F850301621FFF708FF02F1680043
:1060800082F86410FFF702FF02F17C0082F87810BA
:10609000FFF7FCFE02F1900082F88C10FFF7F6FE8D
:1060A00002F1A40082F8A010FFF7F0FE02F1B800A0
:1060B00082F8B4102921FFF7E9FE02F1CC0082F842
:1060C000C810FFF7E3FE02F1E00082F8DC10FFF7F2
:1060D000DDFE02F1F40082F8F010FFF7D7FE02F5C2
:1060E000847082F80411FFF7D1FE02F58E7082F8F9
:1060F0001811FFF7CBFEBDE8084002F5987082F852
:106100002C11FFF7C3BE00BF9803002038B5054C23
:10611000A4F5A075143C201DFFF7E7F8AC42F9D1B7
:1061200038BD00BFD804002030B591FAA1F391FA30
:10613000A1F1B3FA83F3C4685B000325B1FA81F1DE
:1061400005FA03F3490024EA03038A401A43C260B4
:1061500030BD431C04D00C3151F80C3C5A1C01D109
:1061600000207047834201F10C01F5D101207047F6
:10617000F8B5471C06460D4600D1FEE700F00F02B9
:10618000414BC0F3031053F82240FFF7B1FB94FAE0
:10619000A4F3B3FA83F3876803225B0002FA03F3E4
:1061A00094FAA4F2B2FA82F227EA03075200032318
:1061B00093403B4305F007018360032903D8DFE8E0
:1061C00001F05F032C61FEE7012394FAA4F2B2FA16
:1061D00082F206685200032707FA02F226EA020654
:1061E00094FAA4F2B2FA82F2520093400139334396
:1061F0000129036005D843682A074CBF2343A34302
:106200004360C5F30112012A02D0022A18BF0022FE
:106210002146BDE8F840FFF787BFC5F306227F2A75
:1062200001D10223D1E7360716D5230A93FAA3F644
:10623000B6FA86F6476A93FAA3F3B6004FF00F0C4E
:10624000B3FA83F30CFA06F69B0027EA060602FA75
:1062500003F333434362E4E794FAA4F3B3FA83F31A
:10626000066A9B000F2707FA03F326EA030694FA4F
:10627000A4F3B3FA83F39B009A4032430262D0E75F
:106280000023A2E70323A0E7F83A0208431C06D143
:106290007047834202D18968FFF76ABF0C310B68EF
:1062A0005A1CF6D1FEE70B685A1C01D1002070473A
:1062B000834201D1486870470C31F4E7431C01D098
:1062C000FFF7F1BF002070474B6813B94FF0FF3064
:1062D0007047834201D1086870470C31F4E708B178
:1062E000FFF7F2BF4FF0FF30704703460868421CCB
:1062F00000D17047984201D1886870470C31F5E7AA
:10630000431C01D0FFF7F1BF704703468B4208469C
:1063100004D01BB100290CBF1846002070470000B4
:106320004FF0B0431A6842F061021A604FF4E02265
:106330009A6061221A60064ADA6000229A6140F28D
:106340003F321A62034B4FF000629A60704700BF01
:106350000001042200ED00E04FF0B04382B01A6E5D
:1063600002431A661B6E03400193019B02B0704703
:10637000043870470368124A934282B004D14FF444
:10638000006002B0FFF7E8BFB3F1804F0CD14FF0CF
:10639000B0439A6D42F001029A659B6D03F00103D0
:1063A0000193019B02B07047064A934202D14FF419
:1063B0000030E6E7044A9342F4D14FF48020E0E74E
:1063C000002C014000440140004801400368134A8A
:1063D000934206D14FF0B042136E23F4006313666C
:1063E0007047B3F1804F06D14FF0B042936D23F068
:1063F0000103936570470A4A934205D14FF0B042BA
:10640000136E23F40033EAE7064A9342E8D14FF0D3
:10641000B042136E23F48023E1E700BF002C01405B
:106420000044014000480140431C10D00C4B9842EE
:1064300010D007D8B0F1804F0ED0A3F5C0539842CA
:106440000CD0FEE7074B9842FBD11D2070476FF040
:106450000D0070471C2070471B20704718207047A4
:106460000044014000480140431C10D00C4B9842AE
:1064700010D007D8B0F1804F0ED0A3F5C05398428A
:106480000CD0FEE7074B9842FBD11D2070476FF000
:106490000D0070471C2070471B2070471A20704762
:1064A000004401400048014038B50446FFF762FF50
:1064B0002068FFF7B9FFD4E91312FBF7D3FB20687C
:1064C000FFF7B2FFFBF700FC22681046FFF7CCFF96
:1064D00005461046FFF7A8FF85420BD02846D4E9B1
:1064E0001312FBF7BFFB2068FFF7BEFFBDE8384083
:1064F000FBF7EABB38BD10B5FFF768FF044600683C
:10650000FFF792FFFBF7EEFB2068FFF7ADFFBDE85A
:106510001040FBF7E7BB0000431C10D00A4B984229
:106520000BD003D8B0F1804F0BD0FEE7074B984259
:1065300003D003F580639842F7D102207047002012
:1065400070470120704700BF002C0140004401400B
:106550004FF0B042D2F8883023F440630343C2F8CE
:10656000883070472DE9F04F89B0CDE9012304460A
:10657000129BD0F8A00003938B46B449FFF79EFE10
:10658000B3498246D4F8A400FFF798FEB149064605
:10659000D4F8A800FFF792FEAF490746D4F8AC0044
:1065A000FFF78CFEAA498046D4F8A000FFF786FECC
:1065B000A6498146D4F8A400FFF780FE0546BAF14B
:1065C000000F03D1B9F1000F00F03A81D4F8A430E4
:1065D000013303D016B9002D00F03281D4F8A83071
:1065E000013302D0002F00F02B81D4F8AC300133FE
:1065F00003D0B8F1000F00F0238131465046FFF779
:1066000084FE206020B929464846FFF77EFE2060C0
:1066100039462068FFF779FE41462060FFF775FE96
:106620002060002800F00C818C4B984240F0A18043
:106630004FF0B0431A6C42F480421A641A6C22F490
:1066400080421A641A6E42F480421A661B6E03F48A
:1066500080430593059B2423A4F8B030BAF1000FC2
:1066600000F0BA807949D4F8A000FFF70FFE26B1F8
:106670007749D4F8A400FFF709FE4FF00009002F76
:1066800000F0BC807349D4F8A800FFF7FFFD4FF479
:10669000807AB8F1000F06D06F49D4F8AC004AF404
:1066A000007AFFF7F3FD94F8B1206D4B94F9B00038
:1066B000C4F83C90271D43F822702368C4E9013BCD
:1066C000019BE360039B2361029B63610C23002217
:1066D000C4E9063A0823E362226262620121FBF701
:1066E000C1FAD4F800805F4B984538D1BBF5165FEE
:1066F000384600F28580FEF7C1FD3846002E00F0D6
:106700009380FEF7A8FC002800F09A800220FFF793
:10671000FEFA4FF0B043D3F890309B0700F1A6800B
:106720004FF0B04322681B68590500F1D5802268FC
:106730004C4B9A4202D10020FFF70AFF16B9002DF8
:1067400000F0BB803846FEF786FC002878D022682F
:10675000444B9A4203D14FF48060FFF7F9FE16B91B
:10676000002D00F0B380384609B0BDE8F04FFEF7C9
:1067700072BC3D4B984215D14FF0B0439A6B42F436
:1067800000329A639A6B22F400329A639A6D42F453
:1067900000329A659B6D03F400330693069B40F22A
:1067A000251359E72F4B98427FF458AF4FF0B04371
:1067B000DA6B42F00102DA63DA6B22F00102DA638B
:1067C000DA6D42F00102DA65DB6D03F00103079335
:1067D000079B40F226233FE7B9F1000F3FF44DAF8E
:1067E0001B49D4F8A000FFF751FD25B11749D4F893
:1067F000A400FFF74BFD4FF4004940E7BA4648E7D5
:10680000FEF752FD3846AEB1FEF725FCC0B14FF0A1
:10681000B0431A682368500589D5434562D14FF4C7
:106820000060FFF795FE5AE0002D7FF46AAFFEF797
:1068300042FC68E73DB9FEF73EFC00287FF470AFEC
:1068400009B0BDE8F08FFEF706FCF6E70038020855
:10685000C43702087C37020840370208003801407C
:10686000D804002000800040004400402268234BF0
:106870009A4203D14FF44060FFF76AFE3846002E7B
:10688000E1D1002DDFD1FEF716FC0028D8D04FF063
:10689000B04322681B685B057FF549AF174B9A42EE
:1068A000BDD03846FEF707FC0028C9D02268134B3C
:1068B0009A4202D10020FFF74BFE3846FEF7FBFB61
:1068C0000028BDD022680D4B9A4212D0384609B03C
:1068D000BDE8F04FFEF7EFBB084B9A429FD00EB9D0
:1068E000002DDED03846FEF7B6FB00287FF41FAF40
:1068F000A6E74FF48060FFF72BFEE7E7008000403B
:1069000010B4019C18B1019410BCFFF72BBE10BC51
:1069100070470000094B13B59C6809492046FFF7F2
:10692000CDFC48B107480023C0F8A0401A460093A8
:106930004FF41651FFF716FE02B010BDD43902080D
:10694000003802084400002008B5074B90F8B12039
:1069500053F82200FEF72CF900F02200A0F12203E8
:106960005842584108BD00BFD804002008B5074B65
:1069700090F8B12053F82200FEF71AF900F0210038
:10698000A0F121035842584108BD00BFD80400209F
:106990002DE9F0472B4C06460D46FAF723FD94F8F7
:1069A000B130022B074613D894F8B120264B53F888
:1069B0002240A4F104084046FFF7D8FFD0BB4FF4B3
:1069C0007A73AAB231462046FEF7BEFA40B908E013
:1069D0001E4B1F49D3F808804046FFF76FFC18BBD9
:1069E00000252846BDE8F0875AF8233043B994F8CB
:1069F000B1300133DBB2022B84F8B130F4D90CE0B2
:106A000049464046FFF75AFC94F8B1205AF8223024
:106A10001B688342EBD1022AC6D9FFF77BFF94F8AB
:106A2000B130022BC0D9DBE7DFF81CA0DFF82090E3
:106A30000023E0E7FAF7D6FCC01BB0F57A7FBAD3A3
:106A4000CEE700BF44000020D8040020D43902085B
:106A50000038020870B50E46054610B94FF0FF30F9
:106A600070BDFFF771FF04460028F7D129460122C7
:106A700011F8B23F337095F8B100034B53F8200082
:106A8000FEF7D8FB2046EBE7D804002038B50D46CA
:106A90000446C0B1FFF758FFA8B994F9B000C4F894
:106AA0009850FBF71FF994F8B100074B04F1B201BD
:106AB00053F820000122FEF7BDFB94F9B000BDE8B9
:106AC0003840FBF701B938BDD804002038B5154669
:106AD0000446C8B1C0F89C1090F9B000FBF702F969
:106AE000D4F8B830B4F8C21094F8B10013FA81F1B8
:106AF000064BAAB253F82000FDF7C2FB94F9B00090
:106B0000BDE83840FBF7E0B838BD00BFD80400202E
:106B100050B1D0F8A430013306D190F8B120034B26
:106B200053F82200FDF7F8BF704700BFD8040020DB
:106B300050B1D0F8A430013306D190F8B120034B06
:106B400053F82200FEF70EB8704700BFD8040020AB
:106B5000D0F8943004381847D0F8983004381847E3
:106B600010B5044650F80439DA69D1070CD5012272
:106B70001A62FFF7E9FEB0B904F1AE012046012226
:106B8000BDE81040FEF756BBDA69920701D5022234
:106B9000EEE7DA69510701D50422E9E7DA6912075D
:106BA000E7D50822E4E710BD08B52420FBF7D2F8AA
:106BB000024B1868BDE80840FDF7C4BBD8040020AC
:106BC00008B52520FBF7C6F8034B586818B1BDE897
:106BD0000840FDF7B7BB08BDD804002008B5262043
:106BE000FBF7B8F8024B9868BDE80840FDF7AABB70
:106BF000D8040020012200F1AE01FEF71BBB00000B
:106C00000A490346086810B50344EFF3088293422B
:106C100005D9074B0C221A604FF0FF3010BD054A12
:106C2000054C121B9342F4D20B60F7E70C010020D5
:106C30008C39002000000120000400004FF0FF30DC
:106C400070474FF400534B6000207047012070479D
:106C50000020704700207047FEE70000024B16221C
:106C60001A604FF0FF3070478C39002001207047C8
:106C70000048704780EE3600704770477047704795
:106C80007047704770477047D0F8F000704790F831
:106C90006E01704790F81B02003818BF0120704742
:106CA00090F86F314FF47A605843704790F8630161
:106CB0007047000000487047D83B02080048704702
:106CC000D83B020800487047EA3B0208004870477A
:106CD000EA3B020800487047F63B0208004870474C
:106CE000F63B020880F8E810704780F820107047E3
:106CF0006830704760387047704702460023F0B52F
:106D0000D0F8A45E02F509761846A027AB4200DB56
:106D1000F0BD07FB03F491F800C0345DA44502BF49
:106D200000F6F604013042F824300133EEE70000AB
:106D3000084A0023C2E90433D360426EA0F85830F9
:106D4000C0E90E33C0E90C33C2F80C35C2F808357F
:106D5000704700BF202F0020A0F1C800FFF7E8BF58
:106D600002F6F60250F82230002B10DBD0F8A42EE9
:106D700093420CDAA02202FB030000F2862300F209
:106D8000A62053F8042B41F8042B8342F9D1704715
:106D90002DE9F041054605F5005488464FF4FA61A7
:106DA00017461E4603F022F89DF81830079984F81C
:106DB000D5334EF660235943C4F8C403C4F8CC83DA
:106DC000C4F8D07384F8D46301F5FA61284603F05F
:106DD0000DF8C4F8C803BDE8F081A0F1C800FFF7C2
:106DE000D7BF000010B590F83E11044621B1044B06
:106DF000594302F0FBFF0146C4F8E01010BD00BF8C
:106E0000C0D40100A0F1C800FFF7ECBF10B590F8A6
:106E10003F11044621B1044B594302F0E7FF0146FC
:106E2000C4F8E41010BD00BF80EE3600A0F1C80029
:106E3000FFF7ECBF7FB50A4A034608465169049143
:106E4000D96B0391996B0291596B01911B6B009364
:106E5000D2E9032303491AF081FA07B05DF804FB75
:106E6000202F0020FF3B0208A0F1C800FFF7E2BF7F
:106E700010B5C06D104C036886B01B68984701467A
:106E800004A80EF0E9FA9DF810309DF813200B4984
:106E900003F5FA6303939DF8113002939DF81230C5
:106EA00001939DF81530009320469DF814301AF098
:106EB00055FA204606B010BDE4040020603C0208EC
:106EC00070B5D0F840510C46284600211646FAF716
:106ED000F1F8D8B921460E48F9F73AFE014628469E
:106EE00017F0F6FBF9F790FA0A4B0022F9F72CF9A4
:106EF000044630460D46F9F765FA02460B46204631
:106F00002946F9F7D9FAF9F787FD70BD0020FCE7AB
:106F10009A99593F0000F03F02F6F60238B550F852
:106F20002240002C054616DBD0F8A42E944212DA3B
:106F3000A022544304F246209DF8142004992844CA
:106F400004F0E1F82C4484F84502E86D03681B68FE
:106F50009847C4F8AC02002038BD38B500F580551C
:106F60000446B5F86C31A5F81C36002100F5D65062
:106F7000A5F822161C220C3004F5D5541AF0D9FAC3
:106F800004340123C5F8C84A85F81C3B38BDA0F17C
:106F9000C800FFF7E2BF2DE9F04307468DB08846F1
:106FA000914641F624357C1941464A4620461AF05E
:106FB00096FA0146A0B92C2201A81AF0BAFA01A843
:106FC00003F0CDF901AE23460BAA344603CC94421C
:106FD00018605960264603F10803F6D122781A702A
:106FE0002C3542F2BC339D42DDD10DB0BDE8F083BB
:106FF000A0F1C800FFF7CFBF014807F0CEBC00BF2B
:10700000202F0020A0F1C800FFF7F6BF01480EF0C6
:107010005CBB00BF34310020A0F1C800FFF7F6BF11
:10702000D0F8CC1000F58B500022083007F054B88F
:10703000A0F1C800FFF7F4BF07B5D0F8CC3000933B
:107040000A46044B04490193684606F00DFD03B05F
:107050005DF804FB42DB02087C3C0208A0F1C8009A
:10706000FFF7EABF0249D0F8CC000EF068BB00BFC2
:10707000823C0208A0F1C800F4E700BFD0F8CC10B1
:1070800000F6A86006F05CBBA0F1C800F6E710B4FB
:10709000044600F5D7500C3039B1024604F58B5048
:1070A000012310BC083006F0E5BD10BC10221AF018
:1070B00040BAA0F1C800FFF7EABF0B7813F0030352
:1070C00010B500F5805409D100F58B50012208302D
:1070D00006F0F6FDC4F8E80A002010BD012B07D128
:1070E00094F8F835DB0703D400F5AF501430F1E71E
:1070F0000020EFE7036810B55C6A50F8042C516A71
:107100008C4201D8036010BD40F80429F5E7F0B5C2
:107110004C1E04EBD474641091424FEA81050CDDDF
:1071200050F824105E6A4F6AB74206D94151611E79
:1071300001EBD17521466C10EEE74351F0BDF0B57F
:10714000541E04EBD4740E4665106FF0404CA942F7
:1071500015DBD4070ED4023A02EBD272B1EB620F08
:1071600008D14C1C620000EBC40454F8044C40F8F5
:107170002140511E3246BDE8F040FFF7C8BF4C1C0D
:10718000640004EB0C0E50F82E7050F824E07F6A77
:10719000DEF824E0BE4588BF04F1FF3450F82470C7
:1071A00040F821702146D2E7F0B5541E04EBD474A8
:1071B0000E4665106FF0404CA94215DBD4070ED483
:1071C000023A02EBD272B1EB620F08D14C1C6200A2
:1071D00000EBC40454F8044C40F82140511E3246E0
:1071E000BDE8F040FFF793BF4C1C640004EB0C0EAD
:1071F00050F82E7050F824E07F6ADEF824E0BE4597
:1072000088BF04F1FF3450F8247040F82170214603
:10721000D2E7036810B55C6A50F8042C516A8C42BE
:1072200001D8036010BD40F80429F5E7F0B5541EFD
:1072300004EBD47466106FF0404C0C46B44225DB6E
:10724000D5070ED4023A02EBD272B4EB620F08D12A
:10725000621C550000EBC20252F8042C40F82420B6
:107260006C1E621E02EBD2725210A1424FEA8405DC
:1072700021DA50F822405E6A676AB7421BD2445155
:10728000541E04EBD47514466A10EEE7651C6D00BD
:1072900005EB0C0E50F82E7050F825E07F6ADEF8F2
:1072A00024E0BE4538BF05F1FF3550F8257040F8A1
:1072B00024702C46C2E74351F0BD036810B55C6AE8
:1072C00050F8042C516A8C4201D3036010BD40F881
:1072D0000429F5E7F0B5541E04EBD47466106FF082
:1072E000404C0C46B44227DBD5070ED4023A02EBE1
:1072F000D272B4EB620F08D1621C550000EBC202DF
:1073000052F8042C40F824206C1E621E02EBD2724C
:107310005210A1424FEA840524DA50F8224093F932
:10732000286094F92870B7421CDD4451541E04EBC8
:10733000D47514466A10ECE7651C6D0005EB0C0E65
:1073400050F82E7050F825E097F928709EF928E043
:10735000BE45C8BF05F1FF3550F8257040F82470D0
:107360002C46BFE74351F0BD10B5036850F8042C1C
:1073700093F9284092F928108C4201DC036010BD7B
:1073800040F80429F2E7F0B5541E04EBD4746610FB
:107390006FF0404C0C46B44227DBD5070ED4023ABE
:1073A00002EBD272B4EB620F08D1621C550000EB05
:1073B000C20252F8042C40F824206C1E621E02EB1C
:1073C000D2725210A1424FEA840524DA50F82240CA
:1073D00093F9286094F92870B7421CDA4451541E7E
:1073E00004EBD47514466A10ECE7651C6D0005EBE0
:1073F0000C0E50F82E7050F825E097F928709EF981
:1074000028E0BE45B8BF05F1FF3550F8257040F8BB
:1074100024702C46BFE74351F0BD10B5036850F807
:10742000042C93F9284092F928108C4201DB036068
:1074300010BD40F80429F2E78842134604D00A1A26
:107440000146981A1AF05BB870478842F8B50446AE
:107450000D4602D00430854200D1F8BD06462368AF
:1074600056F8047B93F9283097F928209A4207DAD6
:10747000014632462046FFF7DFFF27603046EAE745
:10748000FFF7CBFFFAE78842F8B504460D4602D075
:107490000430854200D1F8BD0646236856F8047BC7
:1074A00093F9283097F928209A4207DD01463246A1
:1074B0002046FFF7C1FF27603046EAE7FFF754FF99
:1074C000FAE78842F8B504460D4602D004308542FA
:1074D00000D1F8BD0646236856F8047B5B6A7A6AD9
:1074E0009A4207D2014632462046FFF7A5FF2760A1
:1074F0003046ECE7FFF7E1FEFAE78842F8B50446CC
:107500000D4602D00430854200D1F8BD06462368FE
:1075100056F8047B5B6A7A6A9A4207D9014632467A
:107520002046FFF789FF27603046ECE7FFF771FE42
:10753000FAE78842F8B504460D4602D00430854289
:1075400000D1F8BD0646236856F8047B5B6A7A6A68
:107550009A4207D9014632462046FFF76DFF276061
:107560003046ECE7FFF7C6FDFAE78B889A0903F08F
:107570003F0310B502FB033304464A88006D52FAFC
:1075800083F1036802319B689847F9F793FBD4F8BD
:107590004411F9F7E7FBF9F7E7FD00EB8000421C27
:1075A0000021206EBDE8104003F008BE00F003008B
:1075B000023801288CBF00200120704780F00200B3
:1075C000C0F3400070478B889A0903F03F0310B561
:1075D00002FB033304464A88006D52FA83F10368C4
:1075E00002319B689847F9F765FBD4F85811F9F711
:1075F000B9FBF9F7B9FD00EB8000421C0021206EB9
:10760000BDE8104003F0DABD2DE9F84F04460D4601
:107610001746994600F10408291B40291CDD4FEA52
:10762000A10ADFB9AAF10206761054F826305246B4
:1076300031462046FFF783FD5EB1013EF5E755F880
:10764000043D22682A602A1B921000212046FFF781
:1076500076FD2B1B042BF2DCBDE8F88FC910D4F8A3
:1076600004A054F82100DAF824B0D0F824E055F84A
:1076700004CC2368DCF82420F34546462AD99645F5
:1076800021D9206044F821302B462268D2F824E02A
:1076900031460868426A72450E4601F10401F8D885
:1076A000191F0B4651F80429D2F824C0E645F8D832
:1076B0009E4217D3013F29464B463A463046FFF7D4
:1076C000A3FF3546A8E7934506D9C4F800C045F89E
:1076D000043CD9E7934502D9C4E900A3D4E7964511
:1076E000CFD9F2E746F8042B1860CEE72DE9F84F22
:1076F00004460D461746994600F10408291B402907
:1077000019DD8E10CFB9B11E491054F82130324620
:107710002046FFF78BFD59B10139F6E755F8043DD6
:1077200022682A602A1B921000212046FFF77EFD66
:107730002B1B042BF2DCBDE8F88FC910D4F804A091
:1077400054F82100DAF824B0D0F824E055F804CC3D
:107750002368DCF82420F34546462AD2964521D2F8
:10776000206044F821302B462268D2F824E03146CC
:107770000868426A72450E4601F10401F8D3191FE8
:107780000B4651F80429D2F824C0E645F8D39E42AE
:1077900017D3013F29464B463A463046FFF7A6FF2E
:1077A0003546ABE7934506D2C4F800C045F8043C23
:1077B000D9E7934502D2C4E900A3D4E79645CFD2D6
:1077C000F2E746F8042B1860CEE72DE9F84F04469F
:1077D0000D461746994600F10408291B402919DD7A
:1077E0008E10CFB9B11E491054F8213032462046D0
:1077F000FFF770FD59B10139F6E755F8043D2268ED
:107800002A602A1B921000212046FFF763FD2B1BE4
:10781000042BF2DCBDE8F88FC910D4F804A054F8AA
:1078200021009AF928B090F928E055F804CC236893
:107830009CF92820F34546462BDD964522DD206045
:1078400044F821302B46226892F928C0324611684C
:1078500091F928006045164602F10402F7DC1A1F70
:10786000134652F8040990F928E0E645F8DB9E42F9
:1078700017D3013F29464B463A463046FFF7A5FF4E
:107880003546AAE7934506DDC4F800C045F8043C38
:10789000D8E7934502DDC4E900A3D3E79645CEDDE2
:1078A000F2E746F8040B1960CDE72DE9F84F0446DE
:1078B0000D461746994600F10408291B402919DD99
:1078C0008E10CFB9B11E491054F8213032462046EF
:1078D000FFF759FD59B10139F6E755F8043D226823
:1078E0002A602A1B921000212046FFF74CFD2B1B1B
:1078F000042BF2DCBDE8F88FC910D4F804A054F8CA
:1079000021009AF928B090F928E055F804CC2368B2
:107910009CF92820F34546462BDA964522DA20606A
:1079200044F821302B46226892F928C0324611686B
:1079300091F928006045164602F10402F7DB1A1F90
:10794000134652F8040990F928E0E645F8DC9E4217
:1079500017D3013F29464B463A463046FFF7A5FF6D
:107960003546AAE7934506DAC4F800C045F8043C5A
:10797000D8E7934502DAC4E900A3D3E79645CEDA07
:10798000F2E746F8040B1960CDE72DE9F84F0446FD
:107990000D461746994600F10408291B40291CDDB5
:1079A0004FEAA10ADFB9AAF10206761054F8263090
:1079B000524631462046FFF7F7FB5EB1013EF5E740
:1079C00055F8043D22682A602A1B921000212046A7
:1079D000FFF7EAFB2B1B042BF2DCBDE8F88FC91084
:1079E000D4F804A054F82100DAF824B0D0F824E048
:1079F00055F804CC2368DCF82420F34546462AD900
:107A0000964521D9206044F821302B462268D2F8CF
:107A100024E031460868426A72450E4601F10401CD
:107A2000F8D8191F0B4651F80429D2F824C0E645AE
:107A3000F8D89E4217D3013F29464B463A46304676
:107A4000FFF7A3FF3546A8E7934506D9C4F800C061
:107A500045F8043CD9E7934502D9C4E900A3D4E72B
:107A60009645CFD9F2E746F8042B1860CEE7000020
:107A70002DE9F04F00F5D95300F50E52BBB0814609
:107A80000F4604333C320025596A31B13AA901EB63
:107A90008501013541F8C83C2DB22C339342F3D116
:107AA00008AE06EB8508B0454FEA850414D0A21055
:107AB000B2FA82F2C2F11F024FF0000352004146B7
:107AC0003046FFF762FF402C23DD18A93046FFF750
:107AD00030FD18ACA04517D1DFF88CB03C464FF014
:107AE00000084FF00A0A454502DDE31B852B15DD32
:107AF000BC4204D120461D4919F053FE0634002330
:107B000023703BB0BDE8F08F2046FFF7F3FA043452
:107B1000E0E741463046FFF70CFDDDE756F8281058
:107B2000B8F1000F01D004F801AB042205A80391BD
:107B300003F056FBD9F85C0003681B68984703996B
:107B40004B6A91F928200092C31A05AA594620468B
:107B500019F004FC23461C4613F8012B002AFAD125
:107B600008F10108BFE700BF8E3C0208973C0208FD
:107B7000A0F1C800FFF77CBF036810B51B6804467E
:107B800098476368834228BF581C606010BD2DE988
:107B9000F041044640689DF818701D460368DB6B91
:107BA00016469847606803682946D3F8E830984736
:107BB000606803683146D3F8E43098473946606816
:107BC00000220AF090FC606884F824500368082DB5
:107BD0001B6EBDE8F0418CBF102120211847406882
:107BE00003681B6F1847406803685B6F1847000005
:107BF0002DE9F0430346006DDFF85880D3E9049582
:107C0000036885B01B6A0E46984704464046FFF756
:107C1000E6FF07464046FFF7E6FF80463846F9F79D
:107C20007DFA07B240464FF47A73B5FBF3F5B9FB22
:107C3000F3F303950293F8F7E7FB24B2CDE90001D3
:107C40003B4605492246304619F088FB05B0BDE8A1
:107C5000F08300BF202F00209E3C0208A0F1C80046
:107C6000FFF7C6BF0000000038B50C2015F022FE5B
:107C700008250024C02015F03BFE013D0444F9D145
:107C80002046F8F79FFB0AA3D3E90023F8F714FC7A
:107C900000224FF07F53F8F70FFC074B0022F8F754
:107CA0000BFCF8F7E1FE80B238BD00BFAFF30080F7
:107CB0000000000000E5C0400000303F2DE9F34126
:107CC000466DC76CB0F858800D480C46FFF7CCFFE6
:107CD000336805461B68304698473B6806465B6933
:107CE000384698470749CDE900802A4620464FF498
:107CF0007A73B6FBF3F319F031FB02B0BDE8F08103
:107D000004310020F23C0208A0F1C800FFF7D6BF02
:107D1000D0E9003213448B4209D9438901339BB225
:107D200043810089984234BF00200120704701231D
:107D300001604381184670472DE9F84F00F5D95589
:107D4000043500F50E5A07460C46914698462E46D5
:107D50000AF13C0A4FF0FF3B20223146204619F041
:107D6000BEFB30B3736A5B4538BF354606F12C065F
:107D700038BF9B465645EFD12B4604F120022068C0
:107D800061681E4603C6083494423346F7D1F86D45
:107D9000C5F8209003681B6898474FF081416862DE
:107DA0004046F8F7DFFFF9F7B9F985F82800BDE894
:107DB000F88F3546E0E7F0B51F468B8816469A06E1
:107DC0008DB005460C4627D10A78092302F003023C
:107DD000D340DB0703D5CB880BB90B89E3B19DF802
:107DE0004C201299684603F080FB9DF801309BB14E
:107DF0009DF8003003F00F03022B0DD194F902011E
:107E0000F8F75CFF4FF07A51F8F7ACFF3A460346BB
:107E100031462846FFF790FF0DB0F0BDF0B591F860
:107E20004A3003F0F002802A8BB005460C4621D17F
:107E30004B88052B1CD990F83D31CBB9504E4FF4EF
:107E40007A72D6E904010023F9F7AEF9B16801446A
:107E500005F5D7501C30FFF75BFF48B1618894F8F7
:107E60004B30E26C092903F004034ED8002B53D1A8
:107E70000BB0F0BD902AFBD14A88052AF8D903F04F
:107E80000F03022BF4D1252AF2D900F58056D6F83B
:107E9000143B002B6FD0D6F8181B01F09BFF002875
:107EA00069D1E36CD6F8142B9A42E1D16A4604F109
:107EB000500304F1700C174618685968164603C63B
:107EC000083363453246F7D1202205F16801384670
:107ED00019F005FB0028CBD094F90201284EF8F7E1
:107EE000EDFE4FF07A51F8F73DFF4FF47A720446F9
:107EF0000023D6E90401F9F757F9B2682346024492
:107F000039462846FFF718FFB2E7216D002BAFD0A6
:107F1000D5F898318B42ABD3922194F84A308DF842
:107F2000001094F802118DF80110CDF8022003F032
:107F3000010305F168020DF1060105F1880052F810
:107F4000044B41F8044B8242F9D1002B0CBF26228E
:107F50000E226946284602F039FD0446002887D0E3
:107F60002B6801461B6C284698472146820028460C
:107F700003F08CF87CE70023C6F8143B78E700BFD9
:107F8000002F00202DE9F047089E9DF82480994697
:107F9000337804468A461746BBB304F594713046DD
:107FA000F9F71CF900285FD103260022514604F599
:107FB000087003F075FBD0F884304B4505465BD262
:107FC000C0F88490E06D03681B68984795F82030EE
:107FD000C5F8880023F00303334385F820303A4680
:107FE00005F1620307F1200152F8040B43F8040B7A
:107FF0008A42F9D18EB141F28831204601F0F6FE75
:1080000004F58053C3F8200B07E0202200F5087028
:1080100003F02CFB05460028BFD0B8F1000F02D0BA
:10802000FF2385F82130E06DFFF7A6FD0023C4F89B
:10803000480FA4F84C3F95F82030206E03F003035E
:10804000DA1E5342534184F84E3F95F8203084F8AD
:108050004F3F036804221B6804F5756198470223AB
:1080600084F8543F0D2008E0304604F5A471F9F778
:10807000B5F80646002898D00020BDE8F08700003B
:10808000F7B51D4F04461646D7E904011D464FF4C7
:108090007A720023F9F788F8B968014404F5D850DA
:1080A0000830FFF735FE28B32A7804F580502946BA
:1080B00002F03F0280F8402011F8013B9B09013398
:1080C0005A4380F8413019F074FBE06DC4F8486FF2
:1080D00003681B6898470023C4F84C0F04F58B50C5
:1080E0000093AC22012304F57561083005F09CFF74
:1080F0000830C0B203B0F0BD002F0020F8B51E4F0D
:1081000004461646D7E904011D464FF47A7200234F
:10811000F9F74AF8B968014404F5D8500830FFF778
:10812000F7FD38B32A7804F58050294602F03F0263
:1081300080F8402011F8013B9B0901335A4380F835
:10814000413019F036FBE06DC4F8486F03681B68D6
:10815000984704F575650949C4F84C0F04F5D073C8
:1081600004F1F402284619F0F9F82846F9F740F826
:108170000830C0B2F8BD00BF002F0020333D020818
:10818000F8B51B4F04461646D7E904011D464FF4C7
:108190007A720023F9F708F8B968014404F5D85059
:1081A0000830FFF7B5FD10B32A7804F58050294652
:1081B00002F03F0280F8402011F8013B9B09013397
:1081C0005A4380F8413019F0F4FAE06DC4F8486F72
:1081D00003681B689847002384F8503F94F83D31AA
:1081E000C4F84C0F13B1802384F8503F0920F8BD28
:1081F000002F00202DE9F04FC0F8482F1A78012AEF
:10820000DBB0044661D1BA48BA4DFFF72DFDADF899
:10821000A000E06C03685B699847ADF8A200206D90
:1082200003681B6A9847ADF8A4002846FFF7D7FCFF
:10823000F8F774FFEB682A932B69ADF8A6004FF4AA
:108240007A72D4E936012B934FF47A762369B3FB23
:10825000F6F32C930023F8F7A7FF236B2E93636BA1
:108260002F93A36B3093E36B2D9031932846B4F892
:108270005830ADF8C830FFF7B6FC4FF08141F8F741
:1082800071FDF8F74BFF636EADF8CA00D3F808250F
:10829000D3F80C35ADF8CE306369B3FBF6F3349305
:1082A0006B69ADF8CC20359328AA04F64C7436AD32
:1082B000134603CBAB42206061601A4604F1080408
:1082C000F6D13C205BB0BDE8F08F032A21D100F548
:1082D0000E563C3630460DF01DF98548FFF7C4FCBC
:1082E000F8F7E8FC8449F8F7F1FD01210246304631
:1082F0000DF0B8F930460DF010F9054630460DF096
:108300000EF92A46014604F64C7019F052FA281D5F
:10831000D8E7052A2BD191F8202002F00302032A86
:1083200040F04F815A789B781A4340F04A8100F51B
:1083300009710423D4F8A45EAA421846C2DAAD2B10
:10834000C0D891F8200078B103F648700E68265026
:1083500025188888A880981D54FA80F091F820503C
:1083600080F8485F0733DBB20132A031E2E7062A2A
:1083700040F014815D78002D40F0238193F8068051
:108380009A78B3F803700492B8F1200F5A7900F587
:108390000E5100F5D95328BF4FF0200804333C316B
:1083A000586A30B15AA800EB8500013540F8C83C46
:1083B0002DB22C338B42F3D1002A44D128AE06EBE8
:1083C0008509B1454FEA850A16D04FEAAA02B2FAEA
:1083D00082F2C2F11F024FF00003520049463046BC
:1083E000FFF712F9BAF1400F28DD304638A9FFF740
:1083F00084F838AEB1451CD108F1050A07AB4FF03F
:10840000000B5FFA8AFA03EB0806D946049B4B453A
:1084100002DDBD4200F39F80A4F84C5FA4F84E9F9C
:108420005A4607A904F5756019F0C3F90BF1080065
:1084300048E73046FEF7EDFE0436DBE749463046B6
:10844000FFF75BF8D8E7012A27D128AE06EB8509AC
:10845000B1454FEA850ACFD04FEAAA02B2FA82F2BA
:10846000C2F11F024FF00003520049463046FFF7A9
:108470003DF9BAF1400F0BDD304638A9FFF721F87E
:1084800038AEB145B8D03046FEF717FF0436F8E7EE
:1084900049463046FFF715F8AEE7022A2ED128AE3E
:1084A00006EB8509B1454FEA850AA5D04FEAAA0235
:1084B000B2FA82F2C2F11F024FF0000352004946A5
:1084C0003046FFF782F9BAF1400F0BDD304638A98C
:1084D000FEF7D9FF38AEB1458ED03046FEF744FFE7
:1084E0000436F8E749463046FEF7CDFF84E700BF83
:1084F00004310020202F002000007A44032A7FF45A
:108500007BAF28AE06EB8509B1454FEA850A3FF4FB
:1085100073AF4FEAAA02B2FA82F2C2F11F024FF021
:108520000003520049463046FFF7BFF9BAF1400F49
:108530000CDD304638A9FEF788FF38AEB1453FF470
:108540005BAF3046FEF769FF0436F7E74946304631
:10855000FEF77BFF50E70BEB0A03822B05933FF7F7
:108560005BAFE06D28AB026853F827B01268904704
:10857000DBF824205946831A4246A6EB08000393F1
:1085800019F017F9039B3360059B9BF82820327183
:1085900009F10109564401379B4637E7072A10D1F4
:1085A00000F5D07300F64C75074A0849009300F1B6
:1085B000F403284618F0D2FE2846F8F719FE0430D6
:1085C00080E600207EE600BFD83B0208303D02086E
:1085D00010B588B004466A46022100F6A86003F090
:1085E000E3FB6A46034604F16801204602F04EF8B8
:1085F00008B010BD10B5D1F8CC10044601230DF021
:1086000088F8204610BD00002DE9F04FCFB0054698
:108610000C46164601462D4A06A89946FFF7EAFF82
:1086200006A80DF0DEF9002847D02B68284F5B69BB
:1086300028469847014606A814F02AFE2078254BC4
:10864000C0F3830AFEF7B2FF002818BF1F46286D4B
:10865000B4F802B00368DB6B98478046286D036866
:108660009B6B98471C4905464846F8F77BFBF8F793
:1086700055FD04902846F8F751FD03904046F8F761
:108680004DFD5346CDE901B032461449009706A886
:1086900014F02BFE227840F20713C2F38302D3407A
:1086A000DB070DD594F84A3094F84B200C4906A806
:1086B00014F01BFE06A80DF04CF94FB0BDE8F08F8A
:1086C000084906A814F011FEF4E700BF823C020836
:1086D00098DF0208393D020800007A443B3D020859
:1086E000843D020841DB020810B490F8E84014B160
:1086F00010BCFFF789BF10BC7047000070B5CAB04E
:1087000005460C46164601461D4A02A8FFF772FFB1
:1087100002A80DF066F960B32B6828465B6998479C
:10872000014602A814F0B4FD20781649164AC0F399
:108730008303FEF73BFF002818BF0A46618802A8A2
:10874000CDE900213246114914F0CFFD227840F2E4
:108750000713C2F38302D340DB070CD594F84A30E9
:1087600094F84B200A4902A814F0BFFD02A80DF0AE
:10877000F0F84AB070BD074902A814F0B6FDF5E75D
:10878000823C0208393D020898DF0208953D020844
:10879000843D020841DB020890F8E8300BB1FFF796
:1087A000ADBF704770B5CAB004460D4616460146C7
:1087B000134A02A8FFF71EFF02A80DF012F9E0B15C
:1087C000236820465B699847014602A814F060FDC3
:1087D00028780C490C4AC0F38303FEF7E7FE002813
:1087E00018BF0A46698802A8CDE900210749324628
:1087F00014F07BFD02A80DF0ACF84AB070BD00BFCC
:10880000823C0208393D020898DF0208C63D020892
:1088100090F8E8300BB1FFF7C5BF70472DE9F8437A
:108820008C88A309013390465FFA83F904F03F0472
:1088300001F10A05002600F168073CB918F80900A3
:10884000B0428CBF00200120BDE8F8834A4639467B
:10885000284618F044FE08B90136F6B2013CE4B2ED
:108860004D44EAE770B590F83D410546002C47D1EC
:108870000B781846FEF7A2FE00283FD08A8895F8AC
:10888000686102F03F0296423AD903F00306012ED6
:1088900003D195F86961964232D9C3F38303042B5F
:1088A00019D195F86A3193422AD905F58053D3F846
:1088B000E83AABB195F81A3263B1012B1CD0114ADA
:1088C0001148022B08BF02462846FFF7A7FF80F099
:1088D0000100C0B270BD2BB995F86B419442E4D849
:1088E0001846F7E7072B02D195F86C31DBE7012B2F
:1088F000DBD195F86D31D6E7044AE5E70120E9E7D9
:108900000020E7E7100100201401002018010020DA
:1089100030B585B004464FF49063006EADF8043076
:108920000368042204F580551B680DF10601984781
:10893000DDF80630C5F8143B4EF66021204601F004
:1089400055FA01A9C5F8180B0A2200252046CDF8D2
:108950000A5002F03BF8014618B12A46204602F0C0
:1089600095FB05B030BD00002DE9F04704464020DE
:108970001E461546DDF824800F46FCF7A6FF202191
:10898000814605F0F9FC874B236033686665C4E9CE
:1089900013950025C4E904551B6865603046984767
:1089A000012384F82C30804BA364804B2360089B08
:1089B00023660A9BA4F85850C4E90605C4E9095582
:1089C000C4E9105525626366C4F85C8004F1680050
:1089D00001F0D4FC764B236004F50979E833C4F840
:1089E000C83004F508764D4604F6A46A2846A0353A
:1089F00001F0B5FC5545F9D14FF4486200214846D5
:108A000018F097FDC4F8B47EC4F8C06E04F1C80332
:108A100004F5805604F58B5004F582570025C4F800
:108A2000B03E0437634BC4F8B83E083004F1F00997
:108A3000C4F8A45EC4F8A88E3946C4F8AC9EC4F845
:108A4000BC0EC6F8645105F063F804F5B050394621
:108A5000183005F05DF87823C6F8003B04F5D957C7
:108A60000423C6F8FC5AC6F8085BB4221F4404F578
:108A70000E55C6F8043BC6F80C2BC6F8103BB8469A
:108A80003C35404608F12C0801F069FC4545F8D119
:108A9000B42128460CF02BFD002200230025C4E958
:108AA000362304F50053C4E93855C4F8D05029469C
:108AB000C6F8205B40F69802C3E9F155384684F8C1
:108AC000E85086F81C5B18F034FD29464FF4987284
:108AD000484618F02EFD4FF07E53C4F8F0304FF0AA
:108AE0007C53C4F84431344BC4F8583104F1F400D9
:108AF0003249202205F032FD00230022C4E946233A
:108B0000C4E9482304F594702D49102205F026FD90
:108B10002C4BC4F838314FF4A163A4F8603114230E
:108B200084F83C3142F60173A4F83E31264BC4F878
:108B30006431264BC4F868314FF4FA7240F60803EA
:108B4000A4F86C31A4F8722101234FF4E13284F8C7
:108B50007031C4F8782184F87C3104F27D101C490E
:108B600084F86E5184F81B5284F87451102205F079
:108B7000F5FC022384F8943104F5D750002384F8DF
:108B80008E51C4F89051C4F89C311022C6F8145B81
:108B9000C6F8185B29460C3018F0CBFC2046BDE81F
:108BA000F08700BF5843020880EE3600FC430208FD
:108BB000DC3E0208E02E00209A99993EFE3D020814
:108BC0009F4802088D67594400007A4240400808D7
:108BD0000F3E020837B504460D4601F0FDFC29465C
:108BE000C4F8CC5004F6A86004F58B5504F0ECFEF4
:108BF0000835D4F8CC1004F1680204F5087002F0CE
:108C0000ABFCD4F8CC100022284604F0A9FF28467B
:108C100005F061F9014630B104F5D75201230C3259
:108C2000284605F027F894F86131009394F86031F4
:108C3000D4F86421D4F838110A48FEF7A8FF94F953
:108C40003C11084805F0A9FE23682046D3F89C3063
:108C500098472368D3F8A030204603B0BDE83040E1
:108C6000184700BF202F00202DE9F04385B00546AE
:108C700008469DF83090884614461E4605F0A8FB2D
:108C8000074640B14B4632462146284605B0BDE86E
:108C9000F04301F0B0BE2146404605F0E5FBCDF8BB
:108CA0000090ADF80C00334603AA21462846ADF8E3
:108CB0000E7001F0CDFE05B0BDE8F083F0B51F46A3
:108CC00000F580530D46D3F8E81A87B004461646DF
:108CD00089B10B887BB100F58B50012302AA0830C3
:108CE00004F0C8FF00280FDC3B46324629462046E8
:108CF00001F081FE0FE03B4632462946204607B090
:108D0000BDE8F04001F077BE009733462A4602A93D
:108D10002046FFF7A9FF07B0F0BD2DE9F0430E464E
:108D20000978C1F3830185B0072905461F4691469E
:108D3000DDE90C3057D1002405F5805819681C5422
:108D4000FF2088F840001879441E1E2C2FD9307857
:108D5000FEF734FC04330190009328460B46394655
:108D6000FFF710F9044600283DD03078FEF726FCC6
:108D700005F64873002845D0CDE90234012301935C
:108D8000337900934A4606F10A033946284601F032
:108D900023FD014638B3B3889B090133DBB24FF49E
:108DA0009672284605B0BDE8F043FFF787BF01285B
:108DB0000AD13078FEF7FAFBA8B10A4605333946E6
:108DC0002846FFF75DF9CDE702280AD13078FEF793
:108DD000EDFB40B10A46053339462846FFF78EF9C8
:108DE000C0E7032802D005B0BDE8F0833078FEF775
:108DF000DDFB0028F7D00A46053339462846FFF741
:108E0000BFF9AFE798F94020002ACDE900343A468F
:108E10004B464FF00101284602DA01F0F1FCB8E7B9
:108E200001F0EEFC98F8412098F940300146002806
:108E3000D9D0013A03F03F0343EA82134FF496720C
:108E40000C92DBB24246284605B0BDE8F04301F083
:108E500030BE73B50D4604461646FFF7B9FB014612
:108E600068B176B194F819020130C0B20A4604F52F
:108E7000D75100902B460C312046FFF7F5FE02B08B
:108E800070BD2A46204602B0BDE8704002F0FEB830
:108E9000A0F1C800FFF7DDBF2DE9F04700F58057CE
:108EA0001E4697F81C3B8AB00546884614464BBBC5
:108EB000144612F8013B202BFAD02046F8F798F917
:108EC000042808D9A3787C2B05D123883380A37884
:108ED000B370033403367B490822204618F0FFFAAA
:108EE0008146002840F0A38008342021204618F055
:108EF00028FB00286ED1744930460AB0BDE8F0471F
:108F000018F04FBC104605F038FBF8B923469846D8
:108F1000994613F8012B202AF9D0A8EB04044F46F8
:108F200019F8010B04F008FE0028F8D13B780BB1CA
:108F300038704F46B94617F8013BDBB9631E062B64
:108F40001BD9002333700AB0BDE8F08707F5C36171
:108F50004FF4966207F5B47018F02BFCB7F8722145
:108F60005A490023304687F81C3B0AB0BDE8F04759
:108F700018F0F4B9462BDDD1E0E798F80030002B6B
:108F8000DFD005EB840404F58054D4F8C47A002FB4
:108F9000D7D005F58B504146083004F0C1FE05F5E9
:108FA000B0553A881835074660B1038841462846CF
:108FB00004F0E6FE0028C4D037B13B790371C4F851
:108FC000C80ABEE70346F1E799F80030463B18BFF0
:108FD0000123F3E7824622460AF8019BAAEB040329
:108FE000402BA8BF402303EBD3734FEA63084146ED
:108FF00002A802F02DF9C0B1504617F049F8C0B2EE
:109000000090434602AA05F1680105F5087002F0D8
:1090100097FB40B141F28831284600F0E7FE2C4929
:10902000C7F8200B68E72B4966E72B4964E7B8F1DE
:10903000000F29D129492046F8F7D0F8074618BB78
:1090400027492848DFF8A090DFF89880DFF89CA037
:1090500014F038F905F50974D5F8A43E9F42BFF61F
:1090600070AF94F8202062B14946404614F03DF9B3
:1090700021464046202202F0CDF85146404614F0E9
:1090800034F90137A034E7E719491222204618F0D5
:1090900026FA60B9113414F8013F202BFBD00BB134
:1090A000144929E72846FFF733FC134924E73346E0
:1090B0002246414605F6A8600AB0BDE8F04703F035
:1090C0008DBF00BF303E0208393E0208193E02083B
:1090D0004A3E02084D3E0208623E0208733E020804
:1090E0007B3E0208C0350020803E020841DB0208BA
:1090F000863E0208993E0208C13E02082DE9F04F63
:1091000003F6F603B5B050F823700E46002F3E99D3
:109110000491DDE93F9B0446C0F2F080D0F8A43E04
:109120009F4280F2EB80A0257D4300F5087305F196
:10913000040805939844002A5ED14719D9F800A085
:10914000D7F8A832534580F0D980ABF104030093DF
:10915000524609F104034146FFF74CF881460028C6
:1091600000F0CC80C7F8A8A2E06D03681B689847A0
:10917000C7F8AC023078FEF721FA04F64873E0B184
:10918000CDE9023901230193337900934146049AD2
:1091900006F10A03204601F01FFB0146002800F0FB
:1091A000AD80B3889B090133DBB24FF49672204641
:1091B00035B0BDE8F04FFFF781BDCDE900390121A1
:1091C000049B4246204601F01BFB0146002800F0AC
:1091D000958097F84532FF2BE3D04FF4967005F158
:1091E00026023E9004F5087010440246204635B031
:1091F000BDE8F04F01F05DBC022A7FD1BBF1050F45
:109200007CD9431993F8442202F00302032A75D152
:1092100099F80420D9F800A09108072A07916DD881
:10922000D3F8A8220592524568D8C3F8A8A2C06D09
:109230000693026812689047069B0799C3F8AC0230
:10924000002309F80B3009F1050B19BB5846F7F755
:10925000CFFF2023CDE900834A46431D042109A8FE
:1092600002F038F8099B0A930AA90422204601F06B
:10927000F2FA014670B1A02303FB074393F845328D
:10928000FF2B3ED1B3889B090133DBB2C8222046B5
:10929000FFF714FD059B53453ED100238DF82D307B
:1092A0000DF12D00F7F7A4FF814638B3E06DFEF70E
:1092B00063FC042350458DF82C3009F1050308BFE9
:1092C0000AF1010001930AAB0A9000930221049B6A
:1092D0004246204601F094FA014678B1A02303FBF0
:1092E000074797F84532FF2B1ED1B3889B090133FE
:1092F000DBB24FF416722046FFF7E0FC35B0BDE854
:10930000F08FC82005F12602009004F50870024491
:10931000204601F0CEFBBDE70DF12D035A46514624
:109320002046FFF7B9FDBBE74FF4167005F12602A2
:10933000009004F5087010440246204601F0B9FB85
:10934000DCE7000037B5044601F048F9D4F8E41032
:10935000002965D0204600F03DFD002860D0204661
:10936000FFF736F9024600286ED123682046D3F86D
:10937000A030984723682046D3F89C30984704F5DE
:109380000055D5F8C41391B1204600F023FD70B10B
:109390000023C5F8C43395F8D533009395F8D4333A
:1093A000D5F8D023D5F8CC132E48FEF7F0FBD5F82E
:1093B000C81391B1204600F00DFD70B10023C5F82F
:1093C000C83394F86131009394F86031D4F8642183
:1093D000D4F838112348FEF7DAFB04F58055D5F8A8
:1093E000201B69B1204600F0F5FC48B1D4F8CC1040
:1093F000002204F5087002F0F1F90023C5F8203BC3
:1094000014F0D6FBD4E93631D4F8D020C4F8D0001B
:10941000821A9B1841F10001C4E9363103B030BD16
:10942000D4F8E0100029AAD0204600F0D3FC002890
:10943000A5D02046FFF7CCF8014600289AD000229C
:10944000204601F023FE95E794F819320133DBB290
:1094500004F5D75100930C3100232046FFF704FC9C
:1094600083E700BF202F0020C06C08B503685B694C
:1094700098470028D4BF0020012008BD10B5C8B00F
:10948000D0F8CC100E4A684600230CF042F968462A
:109490000CF0A7FA60B10B4C68460CF09EF920B1B5
:1094A00068460CF02BFA011E04DA68460CF051FAFB
:1094B00048B010BDC9B2204613F0EEFEECE700BF85
:1094C000823C0208C0350020A0F1C800FFF7D6BFDB
:1094D00038B50C468D18AC4200D138BD4FF48071C0
:1094E000002014F012F904F8010BF4E714F060BB4B
:1094F00037B504460846694601F021FE251D04F2F1
:10950000045408222946684617F0E9FF18B9286074
:10951000686003B030BD0835A542F2D1F9E7F7B570
:109520000E4604466946304601F009FE251D04F248
:10953000045708222946684617F0D1FF98B93378B6
:1095400003F00303023B012B07D9D4F80C35013398
:10955000C4F80C35012003B0F0BDD4F80835013350
:10956000C4F80835F6E70835AF42E2D1D4F804254F
:109570006B4603CB04EBC20250609160D4F8043513
:10958000A022013393FBF2F102FB1133C4F804353E
:109590000020E0E770B506229AB04FF4E13131487F
:1095A00013F006FE4FF47A7014F006FB2E4B0020E9
:1095B0000121187114F0B2F90121084614F0AEF936
:1095C00000F062FA00B9FEE7284C294805F0E0F9FE
:1095D00014F08CF8204605F021FB264B264A27493B
:1095E000189418A8199304F017FA00BB684600F005
:1095F00091FA2148224D6022694618F0DAF80A24CF
:1096000005F1680695F86830013BDBB2FD2B09D9FE
:10961000684600F07FFA60226946304618F0C9F8C3
:10962000013CEFD1144A154918A804F01DFA154958
:109630000C4813F02DFE20220F490A4801F0EAFDE4
:10964000084813F02DFE104B08490D4800241C70EB
:10965000FFF7C0FA0A4822464FF47A51FFF7F9FBA8
:109660001AB070BDC0350020043100203431002014
:10967000202F002042DB0208100600207C3C02085C
:10968000A805002030400208040500201FB5114C39
:10969000114B20464FF4A062002140F8043B17F024
:1096A00048FF00230420C4F80435C4F80C35C4F87E
:1096B0000835FCF70AF9094A0260094A0192094A89
:1096C00000920346084A094902940948FFF74CF9F9
:1096D00004B010BDD0290020644002084C400208AC
:1096E000002F002020010020202F00200431002026
:1096F000A8050020044A054B13600548E833C2F86A
:10970000C8300BF000BF00BFA8050020DC3E0208F7
:10971000642900202DE9F0433A483B4E394FA9B067
:10972000F7F766FD4FF000090446304613F0B8FB2A
:1097300068B19F2C0DD0A046304613F077FDC5B21E
:109740000A2D29D1304613F0ABFB0028F4D19F2C11
:1097500030D12C4B0D2283F89F209F24294D013CB2
:109760002B5D0D2B28D10A21274813F095FD0021F0
:109770006B46264829552A46FFF78EFB9DF8003098
:109780003BB12349204813F083FD1F48694613F07D
:1097900099FD00232B700FE001342946304607F86D
:1097A000085007F8049013F077FD0D2DBDD19F2CC4
:1097B000D4D1CEE7002CD1D1144C2046FFF7C2FD06
:1097C00014F0F6F9134BD3E9042599699861411A0D
:1097D000521845F10005C3E9042594F88D3173B1A1
:1097E0002046FFF741FE50B90B4B1B684FF47A71CE
:1097F0005943204629B0BDE8F04300F0EBBA29B048
:10980000BDE8F08304050020C0350020A805002035
:109810003E400208002F00201C0100200048704735
:109820000000C07F002070470020704770477047DD
:1098300070474FF0FF30704770470020704700209E
:1098400070470020704700207047000000487047B4
:109850006C40020800207047004870476C400208C6
:1098600040680368DB681847B0F918007047017753
:10987000704770470020704700797047BFF34F8FE3
:109880000549064BCA6802F4E0621343CB60BFF39C
:109890004F8F00BFFDE700BF00ED00E00400FA05B8
:1098A00000207047406808B50368D3F884309847B3
:1098B00010F0140F14BF0120002008BD436893F876
:1098C0006001704710B54FF47A7204460023D0E966
:1098D0000401F7F769FCA368184410BD0020704725
:1098E000002070477047002070470020704700201C
:1098F0007047002070470020704700000048704704
:109900007A4002087047F8B507460C468E18B442F4
:1099100000D1F8BD78680368D3F8A43098474FF4B5
:1099200080710546002013F0F0FE454004F8015B0D
:10993000EDE708B5034600201871012113F0EEFF92
:109940000121BDE80840084613F0E8BF10B500202B
:109950000C4601F0010114F04BF8C4F34001012062
:10996000BDE8104014F044B810B5012014F07AF8A6
:109970000446002014F076F840EA440010BD08B513
:10998000F9F736FB72B6BDE80840F9F739BB10B5F8
:109990004FF4DE710446FBF79CFF204610BD406883
:1099A000002107F0FFB810B5044614F001F9D4E91E
:1099B0000431A269A061821A9B1841F10001C4E937
:1099C000043110BD10B500220023C0E904238160DA
:1099D000044614F0EDF8A06110BD036810B51B6CCF
:1099E0000446984720B92046BDE8104005F012B85B
:1099F00010BD10B44468134694F8602110BC05F003
:109A000037B830B5012185B0044608F0CDF9012200
:109A10000021204608F0EDF97F238DF80F30002259
:109A20000123CDE9003289210DF10F02D4F85C0148
:109A300005F047FED4F85C31186803680521DB693E
:109A4000984714F0B5F80546D4F85C311868D96A1F
:109A500002681269904720B114F0AAF8401B32281E
:109A600006D9D4F85411204607F071F905B030BD7D
:109A7000D4F85C31186803685B6D9847E4E708B573
:109A80004068FFF7BEFF08BD30B51B4A1B491C48A4
:109A900087B009F028FA0023049310221623CDE999
:109AA0000232122105230024CDE90031154A16495E
:109AB00013480594082306F043F8054658B11349A6
:109AC000134813F0E5FB12480A22294613F05AFC0A
:109AD000204607B030BD012211460124084809F094
:109AE00093F8009441F2210341F60F5221460448B5
:109AF00009F034F9ECE700BFC44202083C43020815
:109B0000482F002000007A428D67594483400208A4
:109B1000C035002013B5054B00936946044B0193F3
:109B2000044600F037FC204602B010BDA8400208F1
:109B3000482F002070B5194E194B33604820FBF7B1
:109B4000C4FE184C054606F0C1F82946204606F02A
:109B500063F8154B2360154B154919600022C3E9C2
:109B60000146144C83F82420C3E90322124B2360DE
:109B7000124B6260A36000220023C4E9042314F0A6
:109B800017F80F4B0F4AA06100210020C3E9020122
:109B9000C3E90401C3E906011A6070BD0431002065
:109BA00064420208482F0020B4400208202F002001
:109BB000BC410208002F002028420208EF934466AF
:109BC000E02E00203C420208704770477047704703
:109BD0000048704742DB02080020704700207047B1
:109BE000002070474FF07E507047C82070474FF4F8
:109BF0007A60704770B50F481646F6F7A9FFF6F77A
:109C000003FC02460B4600200B4914F0F3FC0B4BFF
:109C10000022F6F799FA044630460D46F6F7D2FBD5
:109C200002460B4620462946F6F746FCF6F7F4FEB8
:109C300070BD00BF9A99593F000024400000F03FDA
:109C4000002370B50446C0E90C33C0E90E33A0F818
:109C50005830406D03681B689847236820625B6B2F
:109C6000204698472368A0649B692046984706468B
:109C7000A06CF7F71FF84FF07E5105463046F6F717
:109C800069FF01464FF07E50F7F720F9014628465C
:109C9000F7F768F8F7F768FA2064606D03681B68E7
:109CA00098476064206D03681B689847206D0368BF
:109CB0001B6B984784F82C0070BD2DE9F0410446D9
:109CC000406D03681B689847656C2368451B9B695A
:109CD0000646204698474FF07E51F6F73BFF014677
:109CE0004FF07E50F7F7F2F8236807465B6B20468B
:109CF000984780462846F6F7DDFF3946F7F732F8F1
:109D0000F7F732FA054670B14046F6F7D3FF394609
:109D1000F7F728F8F7F728FA236C66641D44A84281
:109D200094BF20642564BDE8F081F8B51E46137821
:109D30000B7017469A090D4601D00020F8BD03F0BC
:109D400003020923D34013F0010319BFB7F8013010
:109D5000EB800B81CB801BBFB7F803302B81012137
:109D600005217C5CAC80A209032AE6D004F03F0404
:109D700002FB0444E2B2402ADFD801315418B44255
:109D8000DBDC394405F10A0017F013FD321B92B2F7
:109D9000B82A6A80D1D8391905F14A0017F009FDAF
:109DA0000120CBE710B50446C06C03681B689847D8
:109DB00030B9B4F8583043F00103A4F8583010BD5E
:109DC00000238380438080F80231F8E7C06C036889
:109DD0005B681847406D036810B51B680C469847D0
:109DE000001B0028D4BF0020012010BD406D036877
:109DF00010B51B680C469847204410BD03682DE938
:109E0000F0411B6805460E469847044630B9E86C99
:109E1000036831465B68BDE8F0411847012812D05D
:109E2000EF6C3B6820F07F412846D3F80880FFF7AD
:109E3000DDFF220E013A034631463846C446D2B20F
:109E4000BDE8F0416047BDE8F0812DE9F0410446EE
:109E5000006D0368C2B05B68FF2202A99847061E26
:109E600072DD2368206D5F680368DB6B98470546E9
:109E7000206D03689B6B98472946024602AB20463B
:109E80000096B847E06C03681B68984705460028B1
:109E90005AD00146334602AA2046FFF746FF002863
:109EA0004DD0206D0368DB6B98474FF08141F6F78A
:109EB00059FFF7F733F985F80201276D3B683846FB
:109EC000D3F80C80DB6B9847324601463846C047D2
:109ED0000746206D036831469B68984763690344D1
:109EE0006361236806462846D3F8088001F011F91B
:109EF0003B46024629462046C0472B789B0726D47E
:109F0000A36B0133A36323683946DB6932462046DD
:109F10009847312801461DDDE66CB0F5FA4F3368ED
:109F2000A8BF4FF4FA4120465F6AFFF75FFF29465A
:109F300002463B46304642B0BDE8F0411847E06C6F
:109F4000036829465B68984742B0BDE8F081E36B3F
:109F50000133E3632946204642B0BDE8F041FFF7F4
:109F60004DBFF0B5C56C04462B68406D1E69036893
:109F7000C1B01B68984701462846B04760B32046E9
:109F8000FFF79BFE206D0368FF219B689847236CB9
:109F9000B3EB500F4FEA500520D2236820469B694F
:109FA00098470646206C281AF6F784FE4FF07E513B
:109FB00005463046F6F7CEFD01464FF07E50F6F7E7
:109FC00085FF01462846F6F781FFF7F7CDF80146F1
:109FD0002046FFF70BFFA06141B0F0BDA16920460C
:109FE000FFF7F8FE0028F7D0206D03685B6B9847F9
:109FF000C0B1E36923B9606D03681B689847E061ED
:10A00000606D03681B689847E369C51A236820469A
:10A010005B6A9847854240D9B4F8583043F0020350
:10A02000A4F85830E56C606D0023E3612B68DE68AE
:10A0300003681B68984701462846B04760600028BF
:10A04000CAD003788DF80030092203F0030322FA06
:10A0500003F3DB0741BFC388ADF801300389ADF8D6
:10A06000033054BF0123052382880DF803205D1CB3
:10A07000027900F10A010DEB050001F035F8666880
:10A08000728805445319FF2B0CDDE06C03683146E0
:10A090005B689847002363609EE7236820461B6A3D
:10A0A000984794E706F14A010DEB050017F081FB94
:10A0B000206D768803682E4431469B689847054694
:10A0C000606D03681B689847E060206D0368324646
:10A0D0001B6969469847064678B96568236828462B
:10A0E0001F6901F016F8294602462046B847616804
:10A0F0002046FFF76BFE66606EE705EB45056908D5
:10A100002046FFF773FEA06066E7F8B5416A044693
:10A11000FFF760FEC8B1256D2B685E6A2368204694
:10A120009B6A984701462846B047256D2B689E6A72
:10A1300023682046DB6A984701462846B0474FF41B
:10A14000FA612046FFF752FE6062206D0368DB690A
:10A150009847206D03681B6B984794F82C30834216
:10A1600017D084F82C00B0B9606D03681B6898475D
:10A170002062606D03681B689847236AC01AB0F5B7
:10A18000FA5F82BFB4F8583043F00403A4F85830A3
:10A1900001E0002BEDD06368002B64D0206D0368D4
:10A1A0005B699847002800F09880606D03681B6821
:10A1B0009847E5682369471B3B44236106462046D0
:10A1C000FFF77BFD236C9F427CD900232364236827
:10A1D00020469B6998470646206CC0F16400F6F75C
:10A1E00069FD4FF07E5105463046F6F7B3FC014657
:10A1F0004FF07E50F6F76AFE01462846F6F766FEF7
:10A20000F6F7B2FF01462046FFF7F0FDA061206D92
:10A2100003689B69984761688A884888930902F0B7
:10A220003F0203FB0222D2B223680232DB680244FF
:10A230002046984761680B789B0755BF236B636B7B
:10A240000133013354BF236363632046FFF7BEFD30
:10A2500000236360236820461B6B98470146204615
:10A26000FFF7C4FDA062236820461B6B98470028B7
:10A2700011DDA16A2046FFF7ADFD60B1206D0368D6
:10A28000DB6A9847236820461B6B984701462046A7
:10A29000FFF7ACFDA062E56C606D2B689E6A0368F9
:10A2A0001B68984701462846B047014610B1204632
:10A2B000FFF7A4FD2046FFF7C8FD2046BDE8F840A3
:10A2C000FFF74FBE1D44AD1B632D25647FF67FAFA6
:10A2D000606D03681B68984798E7A1682046FFF700
:10A2E00079FDA0B1206D03689B69984761688A88F1
:10A2F0004888930902F03F0203FB0222D2B223688E
:10A30000023202441B692046984761689DE7F8BD08
:10A310002DE9F047064608790C461746984600F0A6
:10A32000D3FEF56C88B16388B82B0ED82B684146F4
:10A330003046D3F80890FFF759FD3A4603462146C8
:10A340002846CC46BDE8F04760472B6821462846A2
:10A350005B68BDE8F04718470368DB69184710B52C
:10A3600020220446002117F0E4F8204610BD10B466
:10A3700004460846214610BC09F078BF10B50446D3
:10A38000FFF7EDFF4022002104F1200017F0D1F883
:10A39000204610BD30B50D4689B00446FFF7DFFFFB
:10A3A0002B6869461B6828462022984720466A4643
:10A3B00004F120010DF054F9204609B030BD000031
:10A3C000F0B5B1B00146044668460DF066F99DF857
:10A3D0000030013BDBB2FD2B30D81B4B20AA03F130
:10A3E0004007164618685968154603C50833BB422E
:10A3F0002A46F7D1154B08AA03F1200C1746186816
:10A400005968154603C5083363452A46F7D12246E5
:10A41000394610A80DF05AF83246694618A80DF0D2
:10A4200055F8202218A910A817F059F830B910AB28
:10A4300013F8012B2AB901302028F9D1002031B0BE
:10A44000F0BD0120FBE700BF90430208D1430208A2
:10A4500038B50C460546014620222046FFF77CFF12
:10A4600020280AD1402205F120012046FFF774FF81
:10A47000A0F140035842584138BD0020FCE738B5F0
:10A480000B680C465B68014605462022204698472B
:10A4900020280BD1236840225B6805F1200120466B
:10A4A0009847A0F140035842584138BD0020FCE7CE
:10A4B0003F2A70B51ED95F2A00F1200300F1600425
:10A4C00007D853F8042B41F8042BA342F9D14020BC
:10A4D00070BD1A460D4652F8046B45F8046BA24253
:10A4E000F9D1403150F8042B41F8042B9842F9D1AE
:10A4F0006020EDE70020EBE7602A30B40B4613D173
:10A500000A4603F1400400F1200152F8045B41F8CF
:10A51000045BA242F9D1603352F8041B40F8041BDB
:10A520009A42F9D130BC7047402AFBD100F120019A
:10A530000A4603F1400453F8045B42F8045BA3426B
:10A54000F9D130BC0DF0A9B813B504460846114640
:10A550001A4604F12003009323460DF0AFFE02B02B
:10A5600010BD0B46114600F1200218460CF0AEBF9C
:10A570000020704770477047002070477047704751
:10A58000704700207047002070470020704700206F
:10A5900070470020704770B5046D23680546084673
:10A5A0009E6800F0B6FD01462046B04705220446ED
:10A5B0000021286E00F002FE34235C436423B4FBC8
:10A5C000F3F4604370BD08B504220121006E00F071
:10A5D000F5FD7823584308BDFFF732BBFFF795BD63
:10A5E000F8B58B8803F03F04013CE4B223F03F034D
:10A5F0001C438C80A40901340D46E4B201F10A0623
:10A600000027AB8803F03F0313FB04F3BB4200DCDD
:10A61000F8BD3046264422463146274417F0C9F893
:10A62000EFE7F8B50A788B88920706460C4601D505
:10A630000020F8BD03F03F079B090133DBB207FBA5
:10A640000333402B07F10105F2DC0368DB6B98470D
:10A650000028EDD0A28892090132D2B207FB024055
:10A6600006F168010A3017F0A4F8A38823F03F032D
:10A670001D433368A5801B6C214630469847A3884C
:10A6800003F03F03013340EA0360D2E72DE9F043D2
:10A69000202B93B080460E4617461D4603D8FFF781
:10A6A00081FB044620B90024204613B0BDE8F083A6
:10A6B0000346102203F84A2B06F12009324652F8CD
:10A6C000041B43F8041B4A45F9D1D8F85C00036821
:10A6D0001B6898472A46C4F86A008046394604F148
:10A6E000AE0017F066F805F1640363800DF1040C09
:10A6F000334618685968624603C208334B4594468E
:10A70000F7D12A4639460AA8CDF8248017F051F827
:10A7100005F1240301AA04F16E013046FFF714FF8E
:10A72000C2E72DE9F04FAFB099469DF8E0A0DDF803
:10A73000EC804FEA9A130AF03F0403FB044408F14B
:10A7400005032344A62B06468B46174604D900254D
:10A7500028462FB0BDE8F08FFFF724FB0546002800
:10A76000F5D0202303709BF8003080F84A3096F82B
:10A77000683080F84B30494622460DF101008DF8D3
:10A7800000A004F1020917F014F804F1B9030DEB6D
:10A7900009006B44B8F1000F12D09DF8E42003F8D3
:10A7A000B82C3A99424617F004F808EB09036A46B8
:10A7B00005F14C01384600F006FE02306880C7E71C
:10A7C000FF2203F8B82C336E1A6801461668184643
:10A7D0000422B047A31DEAE77FB509788DF814106D
:10A7E0000B9903910A9902919DF8241001919DF80B
:10A7F0002010009105A9FFF794FF07B05DF804FB56
:10A800002DE9F8430229DDF8249007460D469046CD
:10A810001E4603D809F11103B82B03D900242046A2
:10A82000BDE8F883FFF7BEFA04460028F6D0AD0075
:10A83000057098F8003080F84A3097F8683080F852
:10A840004B3000F14C01089A4B46304600F0BBFDFE
:10A8500002306080E3E770B50E461546FFF7A2FAB6
:10A86000044638B10C2300F84A3B2A46314616F01C
:10A87000A0FF6580204670BDF8B50F4616461D4600
:10A88000FFF790FA044668B12D01282345F003052F
:10A89000037080F84A50324639464B30013616F084
:10A8A00088FF66802046F8BD2DE9F0470B78FF2B26
:10A8B00005460C4690464AD003689B6C984704F1C5
:10A8C0004A09064604F10A0AE6B9A278494628462A
:10A8D000FFF7C1FF0746002839D0227904F10A01A9
:10A8E0000A3000F010FC3B78B88023F0030343F0FB
:10A8F00002033B703246434639462846BDE8F047DE
:10A90000FFF706BD2B6821465B6C2846984700F58B
:10A910009670A2788044334649462846FFF7ACFF3C
:10A92000074688B1227951460A3000F0ECFB3B78AB
:10A93000B88023F0030343F002033B700022434638
:10A9400039462846FFF7E4FC013EF6B2BCE7BDE815
:10A95000F08770B591F84A6006F00F03032BC2B080
:10A9600005460C462FD14B88042B2CD901A800F0AA
:10A97000A6FB237822798DF8043004F10A010DF149
:10A980000E0000F0C0FB6288ADF80800013A92B2F8
:10A9900004F14B010DF14E00ADF8062016F009FF51
:10A9A000686E036801A91B68984760B901A9284629
:10A9B000FFF716FE36094FF4967206FB022201A934
:10A9C0002846FFF771FF002042B070BDB82A70B56D
:10A9D0000E46154603D8FFF7E5F9044610B90024E2
:10A9E000204670BD2C2300F84A3B2A46314616F01B
:10A9F000E0FE6580F4E72DE9F0410D781746C5F3D8
:10AA00008302092A06460C4620D0013BDAB2022A0C
:10AA10001CD825F0030545F001050D70406E9B0123
:10AA20008B8003681B6898472378C3F38303082B44
:10AA30000AD0042B14BF012203223B462146304694
:10AA4000BDE8F041FFF764BC0222F6E7BDE8F08103
:10AA50002DE9F0411F460B789DF818500646C3F3C8
:10AA6000830009280C4622D0013DE8B202281ED8F6
:10AA700023F003030B701388706ECB8053880B8117
:10AA80000368AD011B688D8098472278C2F383026A
:10AA9000082A0AD0042A14BF012203223B46214679
:10AAA0003046BDE8F041FFF733BC0222F6E7BDE8CF
:10AAB000F0812DE9F0410C46069F257825F003052D
:10AAC00045F002052570C5F38305092D064611469C
:10AAD000984618D160884A301A46204416F069FE1C
:10AAE0006388434463800023A3800525706E036858
:10AAF00021461B6898473B462A4621463046BDE81A
:10AB0000F041FFF705BC1A4604F10A0000F0FBFA19
:10AB10002578A080C5F38305A5F108035D425D415A
:10AB2000E4E700002DE9F04F0A7802F00303023B4E
:10AB3000012BF1B005460C4665D8C2F38303092BFF
:10AB40008E8854D13F2E1AD891F852E04F88D1F810
:10AB50004A20D1F84E300EF0030C093F06FA0CF6ED
:10AB6000FFB21FFA86F847450BD80A3405680397E9
:10AB7000CDE900E401F153060296AC6DA047002038
:10AB800032E05336012200F1680102FA0CF2A019FA
:10AB900016F0A5FC0028F2D12B682146DB6B284675
:10ABA00098470028EBD0686E036821461B689847D9
:10ABB0000028E4D194F90201F6F780F84FF07A51B9
:10ABC000F6F7D0F84FF08141F6F7CCF8F6F7A6FA91
:10ABD000A3885A1C2344A28098722B6821465B6C80
:10ABE0002846984740F0C06071B0BDE8F08F0B2B4D
:10ABF00006F03F063CD191F94A30002B32DB002EA3
:10AC000042D1930706D42B6821469B6B2846984770
:10AC10000028B4D12378C3F383020F2AAFD801A14F
:10AC200051F822F04BAD00084BAD00084BAD0008C9
:10AC300015AD000849AF0008CFAE0008CFAE000840
:10AC400055AE00084BAD00087FAB00081BB00008F4
:10AC50007FAB00087FAB00087FAB00087FAB00082C
:10AC6000F5AF0008002E8AD10368DB6E984786E7AF
:10AC7000002EC6D0032B07D14B88032B04D90368C1
:10AC8000D1F84A20DB6F9847A28892090132D2B2EC
:10AC900005F1680104F10A0016F021FC00287FF498
:10ACA0006EAF2B682146DB6B2846984700283FF49F
:10ACB00066AF2378C3F383030A2B06D121462846C7
:10ACC00071B0BDE8F04FFFF744BE686E0268032B19
:10ACD000126821460ED19047064600287FF44FAFF8
:10ACE00021462846FFF77CFC324621462846FFF7DE
:10ACF000DBFD44E7904700287FF441AF214628461A
:10AD0000FFF76EFC2B6821465B6C2846984740F0A5
:10AD1000807069E76388D4F84A60032B7FF62FAF11
:10AD2000686E036821461B68984700287FF427AFA8
:10AD30002B683246DB6F2146284698472146284635
:10AD400071B0BDE8F04FFFF76CBC94F84B308DF854
:10AD50001830638894F84A60042B7FF610AF686E51
:10AD6000036821461B689847814600287FF407AF97
:10AD700095F86830B3425CD12B6806A9DB6C284695
:10AD8000984704F14C0806460EAF0DF1BC0AB145D8
:10AD90004FDA2B684A461B6D394628469847638828
:10ADA0004246023B5146384600F031FB031E4EDD61
:10ADB00022782968C2F38302082A3FD19AF80080DA
:10ADC0004FEA981208F03F0602FB0666B21C9B1A77
:10ADD00056445244DBB203920493737803F00F039A
:10ADE000CDE901830DF1BD060096D1F85CA03B468C
:10ADF0004A4621462846D047C8B1237813F00203BB
:10AE000015D1CDE9023301932379009306A904F10A
:10AE10000A033A462846FFF784FC014638B14FF44E
:10AE2000FA730093324643462846FFF742FEFF235B
:10AE3000237021462846FFF7F4FBD5E6CDE901A3B0
:10AE400000974E6D4B4621462846B047EFE709F183
:10AE500001099CE7638894F84A60232B7FF68FAE44
:10AE6000686E036821461B68984700287FF487AE08
:10AE700095F86830B3427FF461AF04F14B0606AA3F
:10AE800004F16B0730687168134603C30836BE428D
:10AE90001A46F7D106AA0EA905F16800FFF761FB73
:10AEA00063882FAF213B324639460EA800F0AFFA37
:10AEB00000287FF743AF2B68CDE900700EAA5E6EC5
:10AEC000214606AB2846B047FF23237036E794F8A7
:10AED0004A308DF818306388032B7FF650AE686EC9
:10AEE000036821461B689847064600287FF447AE52
:10AEF0002B680EAA5F6F06A904232846B84704F101
:10AF00004B0A80460DF139090DF1BC0B464590DA2C
:10AF100063884846013B5246594600F078FA0028BB
:10AF200009F121090EDD2B682278CDE900B006EB8E
:10AF300046169F6F0EAB3344C2F383022146284668
:10AF4000B84776E70136E1E70EA8FFF708FA0EAE3C
:10AF500004F14A0304F16A0718685968324603C2CB
:10AF60000833BB421646F7D16388D4F86A90632B46
:10AF70007FF605AE20220EA905F1680016F0AFFAA3
:10AF800000283FF4FCAD686E036821461B689847B3
:10AF900000287FF4F4AD0EAF0FCF2FAE0FC6B4F87C
:10AFA000028097E80F00A8F16408B8F1200FA8BF4D
:10AFB0004FF0200804F1AE0A86E80F0042465146E1
:10AFC00038A8CDF8DC9016F0F4FB08F124032FAA82
:10AFD00004F16E010EA8FFF7CAF900283FF4CFADC7
:10AFE0002B68CDE900A80EAA1E6E21464B462846C6
:10AFF000B0471EE703F00303023B012B3FF6BFAD52
:10B00000686E036821461B68984700287FF4B7AD37
:10B010002B6821461B6F284628E66288022A7FF6A5
:10B02000AEAD94F84A3003F00F03032B7FF4A7ADC5
:10B03000042A7FF6A4AD2FA800F041F823782279E6
:10B040008DF8BC3004F10A010DF1C60000F05BF888
:10B050006288ADF8C000013A92B204F14B010DF5DF
:10B060008370ADF8BE2016F0A4FB686E03682FA9AC
:10B070001B68984700287FF482AD2B68DDF8062115
:10B08000DB6F2FA92846984779E500BF2DE9F041ED
:10B090000D7825F0030545F002050D700646406E5B
:10B0A0000368002517460C468D801B6898473B4671
:10B0B0002A4621463046BDE8F041FFF729B9002273
:10B0C000027082804280704700F03F0380090328AD
:10B0D00000F1010206D013FB02F04028CCBF002093
:10B0E000012070470020704710B5930902F03F041B
:10B0F00003FB0444402C04DC224616F05AFB204695
:10B1000010BD0024FBE710B51446FFF7EDFF204605
:10B1100010BD83889A0903F03F0302FB0333428882
:10B120000078DBB2023310F00300134405D0C21ED6
:10B13000504250418000184470470420FBE730B56E
:10B140000446A1B002A80D4609F06CF9237801224B
:10B15000C3F383030DF1070102A88DF8073009F04E
:10B1600049FA9DF80730092B04D10222211D02A8BB
:10B1700009F040FA628804F14A0102A809F03AFA9B
:10B1800008220DEB0200294609F066FA02A809F030
:10B190002FF921B030BDA0F14103052B02D837387B
:10B1A000C0B27047A0F16103052B01D85738F7E70B
:10B1B0003038C0B20A2828BF0020704737B503686E
:10B1C000144604220D461B680DEB020198470198B6
:10B1D000621BB0FBF2F302FB1300284403B030BD46
:10B1E000F0B50B4D03468E18B14203F1020303D1B3
:10B1F000002300F81230F0BD11F8014B270904F0CC
:10B200000F04EF5D2C5D03F8027C03F8014CEBE7C3
:10B210007C4402082DE9F041DFF8308005460C46F9
:10B220008F18BC4201D1BDE8F08114F8016B3309DD
:10B2300006F00F0618F80310284612F02DF818F83B
:10B240000610284612F028F8EBE700BF7C440208FD
:10B25000F8B5064610460D461446F5F7C9FFB0EBA3
:10B26000450F17D1224631468B1BAB4202F1020239
:10B2700001DB0120F8BD12F8020C12F8017CFFF787
:10B280008AFF04463846FFF786FF40EA041001F8BB
:10B29000010BE9E70020EDE7F0B504460020074682
:10B2A00025780DB1904208DB214614F8012B1AB124
:10B2B0009A42F9D100230B70F0BD41F82040254699
:10B2C0002E782C4601351EB19E42F9D127702C46AE
:10B2D0000130E5E7F0B59FB01F46164604466846C4
:10B2E0000D4609F09FF83A463146684609F082F962
:10B2F000DDE92412684609F07DF92A4621466846B0
:10B3000009F0AAF9684609F073F81FB0F0BD2DE9FD
:10B31000F041B0B0064601A815460C461F4608F09D
:10B320004BFA3146102201A808F0F6F92E46A6EB9A
:10B330000508B84506DB01A808F0D4F9404630B04E
:10B34000BDE8F0813246214601A808F025FC103402
:10B350001036ECE72DE9F043B5B0064605A81C46CB
:10B360000F46154608F028FA3146102205A808F0C5
:10B37000D3F907EB04092E190F2CA9EB0405A6EB52
:10B38000040819DC002C0FDD1022002101A816F0A2
:10B39000D0F82246414601A816F00BFA294601AA28
:10B3A00005A808F0E5FA103505A808F09BF9ED1B93
:10B3B000284635B0BDE8F0834246294605A808F086
:10B3C000D7FA103CD8E7F0B58F1CA1B00E4639462D
:10B3D0000546FFF7BFFF044602A809F023F82946F7
:10B3E00002A8202209F085F92246394602A809F070
:10B3F00001F90223009320223346294602A809F0CE
:10B4000090F902A808F0F4FFA01C21B0F0BD2DE9CE
:10B41000F043022BA3B005460F4616461C4603DC3C
:10B42000002023B0BDE8F08304A808F0FBFF06F17C
:10B4300002082022294604A8023C09F05AF94FF0DC
:10B4400002092246414604A809F0D4F820222946E0
:10B4500003AB04A8CDF8009009F063F904A808F044
:10B46000C7FF4A46314603A816F039F80028D7D15D
:10B470002346424639462846FFF749FFD1E703787D
:10B480000B70427862B343F010030B708368C1F80D
:10B490000130C368C1F805300923028A32B10A7845
:10B4A00042F020020A70028ACA520233428A32B142
:10B4B0000A7842F040020A70428ACA520233426855
:10B4C00062B1127852B10A7862F07F020A70426863
:10B4D000013A12F8010F08B1202B03D1D8B27047FE
:10B4E0000123DAE7C8540133F3E738B5002383704A
:10B4F00004460878E362C4E909336370C30641BFB8
:10B50000D1F801306362D1F80530A3624CBF092342
:10B510000123850642BFCD5AA5850233450642BFA9
:10B52000CD5AE58502339A4220700DDB000609D51D
:10B53000D51A07D02A461944A01C16F03AF9621908
:10B540000023937001236370204638BD014809F041
:10B55000CDBF00BF0C3100202DE9F0430746002489
:10B56000ADF5037D08463960C7F8844C3E499046E6
:10B570000AF0D9F800284DD03AA83B4A396823464A
:10B580000AF0C7F83AA80AF02CFA002842D04FF087
:10B59000A00912A8FEF7E3FEA022002112A815F0D0
:10B5A000C8FF202202A93AA80AF099F920280446E7
:10B5B0002DD101221AA93AA80AF091F901280546CD
:10B5C00025D1042235A93AA80AF089F904281ED108
:10B5D000022201A93AA80AF082F9022817D12A46C4
:10B5E0000DF169013AA80AF07AF901280FD1402239
:10B5F0000DF16A013AA80AF072F9402807D12246F3
:10B600000DF1AA013AA80AF06AF9202806D03AA852
:10B610000AF09FF90DF5037DBDE8F08302AD0FCD73
:10B620000AAC0FC495E80F0084E80F000AAE0FCEF5
:10B6300012AD0FC594E80F0085E80F00404602AA3E
:10B640000DF1AA01FEF78DFFD7F8840C1328DEDC7C
:10B65000431C09FB0070C7F8843CA02212A90430E7
:10B6600016F0A7F895E700BF8D4402082DE9F843CE
:10B67000D0F8849C0E461746041D0025A94504DC1D
:10B680004FF000084046BDE8F88321463A46304670
:10B6900015F025FFA046A0340028F3D00135EDE7D2
:10B6A0002DE9F74FD0F8848C05460C46914600F6FC
:10B6B000E436071D4FF0000A4FF0FF3BD04525DC74
:10B6C000B8F1140F07D008F10103C5F8843CA0239A
:10B6D00003FB08552E1DA0220021304615F029FF3E
:10B6E000234686F82090344603F1200518685968EF
:10B6F000224603C20833AB421446F7D1FF2386F833
:10B7000021303346184603B0BDE8F08F2022394679
:10B710002046019715F0E3FE3B460028F2D097F84B
:10B72000203003F00303032B05D0D7F888305B45A6
:10B730003CBF3E469B460AF1010AA037BEE7000027
:10B740002DE9F04188B015469DF8388018F0030FB8
:10B7500004460F461A461FD12946FFF787FFE8B176
:10B76000D4F8845C1C4A6B1EC4F8843C231DC31AA5
:10B77000581150432A1AA0214A43A03A03F1A401C8
:10B7800004338542D8BF00222144E01815F0B7FEEB
:10B79000012008B0BDE8F0811F2B01DC0020F8E794
:10B7A0006A462B4605F1200E9446186859681646DD
:10B7B00003C6083373453246F7D16146002220465E
:10B7C000FFF76EFF2A4680F8208000F162013846BC
:10B7D000FEF7C7FEDCE700BFCDCCCCCC2DE9F043B3
:10B7E0000C46CBB00160064631492046174609F0A9
:10B7F000A6FF02A82E4A0123214609F08AFF02A8CB
:10B800000AF0EFF8E0B10025ADF8045006F1660447
:10B81000D6F8843CAB4210DD14F8423C13B9013534
:10B82000A034F5E7A4F162086FB94146202202A8CE
:10B8300009F099FF202880460AD002A80AF089F86A
:10B840004BB0BDE8F0834046B8470028EDD1E6E7AD
:10B850000122A4F1420102A809F085FF01288146D6
:10B86000EBD1042204F12A0102A809F07CFF04288C
:10B87000E3D1022201A902A809F075FF0228DCD158
:10B880004A46A4F1410102A809F06DFF0128D4D174
:10B890004022A4F1400102A809F065FF4028CCD164
:10B8A0004246214602A809F05EFF2028B7D0C4E72F
:10B8B0008D44020810B5421E0A24002012F8013FF0
:10B8C000303BD9B2092900D910BD04FB0030F5E79F
:10B8D00010B50446F5F78CFC00212318A34203D9C8
:10B8E00013F8012C202A00D010BD03F8011DF5E744
:10B8F00070B5CAB00446002302A809F00AFF02A8E6
:10B900000AF06FF8002800F021826168042202A882
:10B9100009F0E5FF61682022043102A809F0DFFF89
:10B920000422694602A809F0DAFF6168082228317A
:10B930000DEB020009F0D3FF6168082230310DEBF6
:10B94000020009F0CCFF61681022383102A809F02A
:10B95000C6FF61680422483102A809F0C0FF61688F
:10B9600001224C3102A809F0BAFF616801224D3171
:10B9700002A809F0B4FF616801224E3102A809F063
:10B98000AEFF0122694602A809F0A9FF61680422FE
:10B99000503102A809F0A3FF61680422543102A8C3
:10B9A00009F09DFF61681022583102A809F097FF45
:10B9B00061680422683102A809F091FF04226946F7
:10B9C00002A809F08CFF61680122703102A809F019
:10B9D00086FF61680122713102A809F080FF616869
:10B9E0000122723102A809F07AFF616801227331E5
:10B9F00002A809F074FF61680422743102A809F0FA
:10BA00006EFF616801227F3102A809F068FF61685A
:10BA1000012201F2291102A809F061FF61680122E7
:10BA200001F5957102A809F05AFF0122694602A8A2
:10BA300009F055FF61680122783102A809F04FFF33
:10BA4000616801224F3102A809F049FF61680122B3
:10BA50007E3102A809F043FF61680122803102A80B
:10BA600009F03DFF61680222823102A809F037FF28
:10BA700061680122843102A809F031FF6168042263
:10BA8000883102A809F02BFF616801228C3102A8DD
:10BA900009F025FF616810228D3102A809F01FFF0F
:10BAA000616801229D3102A809F019FF032269464D
:10BAB00002A809F014FF616801229E3102A809F072
:10BAC0000EFF61680422A03102A809F008FF616836
:10BAD0000122A43102A809F002FF61680422A83102
:10BAE00002A809F0FCFE61680422AC3102A809F04A
:10BAF000F6FE61687822B03102A809F0F0FE6168B4
:10BB0000012201F5947102A809F0E9FE61680122A1
:10BB1000793102A809F0E3FE616801227A3102A8B6
:10BB200009F0DDFE6168012201F22B1102A809F083
:10BB3000D6FE616801227B3102A809F0D0FE61685F
:10BB400001227C3102A809F0CAFE616801227D3120
:10BB500002A809F0C4FE65682E6D00213046F5F795
:10BB60009FFA002840F0F48080493046F5F7B6FA95
:10BB700000B17E4E2E656E6D00213046F5F790FACD
:10BB8000002840F0E7804FF080413046F5F7A6FAF4
:10BB900008B14FF080466E65AE6E00213046F5F775
:10BBA0007FFA002840F0D8804FF080413046F5F70A
:10BBB00095FA08B14FF08046AE662E6800213046F7
:10BBC000F5F76EFA002840F0C98069493046F5F76C
:10BBD00085FA00B1664E2E60AE6C66493046F5F7C8
:10BBE0005FFA002840F0BC8063493046F5F776FAEA
:10BBF00000B1614EAE646E6F60493046F5F750FAA1
:10BC0000002840F0AF805E493046F5F767FA00B192
:10BC10005B4E95F870306E670C2B28BF0C23052BFC
:10BC200038BF052385F87030626892F87130082BB0
:10BC300028BF0823052B38BF052382F871306268BE
:10BC400092F94C301E2BA8BF1E236FF008018B42C7
:10BC5000B8BF0B4682F84C30626892F87330012B03
:10BC600028BF012382F873306668D6F8AC500021F3
:10BC70002846F5F715FA002876D142492846F5F707
:10BC80002DFA00B13F4D96F82931C6F8AC50022B81
:10BC900028BF022386F82931626892F88030012B90
:10BCA00028BF012382F880306368B3F8822042F213
:10BCB00010718A4228BF0A46A3F8822093F8842094
:10BCC000012A28BF012283F884206268D2F88830D4
:10BCD000B3F5E13F28BF4FF4E133B3F5165F38BF4A
:10BCE0004FF41653C2F8883092F88C300E2B28BFD0
:10BCF0000E2382F88C30626892F89D30012B28BFA9
:10BD0000012382F89D30626892F89E30012B28BF93
:10BD1000012382F89E30626892F8A430022B28BF7B
:10BD2000022382F8A430626892F82831012B28BFE0
:10BD3000012382F82831626892F82B31012B28BF49
:10BD4000012382F82B3102A809F003FE4AB070BD2E
:10BD500000260FE700261EE700262DE700263AE71B
:10BD6000044E47E7054E54E700258CE70000A0414C
:10BD7000000010410000164300401C459A99F9400C
:10BD80000000FA4300002041426892F84E305B0008
:10BD90003B2BDCBF002382F84E30806803681B68B1
:10BDA00018470000000000002DE9F04314464268E7
:10BDB00092F8A43087B0151D63B98DF804108DF882
:10BDC00005300295214601A80593FFF758FB07B0FF
:10BDD000BDE8F083012B1FD10269D2E90289D2E9C3
:10BDE00004678DF804108DF8053040460EA3D3E9A2
:10BDF000002349460295F4F75FFBF4F70DFE0AA312
:10BE0000D3E90023039039463046F4F755FBF4F7A5
:10BE100003FE00230490D5E7D2E90A89D2E90C6732
:10BE200001238DF80410DEE70000000080842E411D
:10BE30002DE9F047171DA8B0044689461646AD49BE
:10BE40000A2238461D4615F04AFB00284AD106F161
:10BE50000E0014F01AF9F4F727FE4FF07E51064653
:10BE6000F5F71EF920B9A4493046F5F737F930B196
:10BE7000A249284628B0BDE8F04715F092BC3146EB
:10BE80009D486768F5F722F84FF07E51F4F760FEA1
:10BE900038602046FFF778FF63684FF07E511868DE
:10BEA000F4F758FE01469448F5F710F80646F5F702
:10BEB00035F90446F4F702FF01463046F4F748FE30
:10BEC0008F49F4F74FFF4FF07C51F4F743FEF5F73D
:10BED00025F98C4903462246284628B0BDE8F0479C
:10BEE00015F03CBA88490322384615F0F8FA50B9E3
:10BEF000F01D14F0CAF8F4F7D7FD666830602046EC
:10BF0000FFF742FF1FE381490B22384615F0E7FA9D
:10BF100038B906F10F0014F0BBF8636883F87E00AF
:10BF2000EDE77B490422384615F0D9FA60B9794922
:10BF3000022206F1080015F0D2FA6368B0FA80F028
:10BF4000400983F82B01DAE773491322384615F0CC
:10BF5000C6FAC0B906F1170014F09AF80028636811
:10BF6000B8BF0330801083F87F002046FFF70CFF36
:10BF700063686A4993F87F209200284628B0BDE89C
:10BF8000F04715F0EBB966490B22384615F0A7FAD1
:10BF900038B906F10F0014F07BF8636883F873007A
:10BFA000ADE760491022384615F099FA60B9594951
:10BFB000022206F1140015F092FA6368B0FA80F0DC
:10BFC000400983F872009AE757491622384615F05F
:10BFD00086FA90B906F11A00FFF76CFC431E012B9C
:10BFE00001D9A82801DD514943E7636883F84F0070
:10BFF000A0680368DB69984781E74D4910223846FD
:10C0000015F06DFAA8B906F11400FFF753FC431EB2
:10C010003A2B01D9F02802DD46493C22ADE763689E
:10C0200000EBD070401083F84E00A06803689B6955
:10C03000E1E741490F22384615F051FA38B96068F6
:10C04000102206F11301583002F088FA57E73B49F5
:10C050000822384615F043FA38BB06F10C0240219D
:10C060006846FFF7F5F8F0B16846FEF7A9F9D0B1D8
:10C0700010A8FEF783F940220DEB02006946FEF797
:10C080003BFAA068036810A99B6C98472C49284686
:10C0900015F087FB202210A905F12100FFF7A0F879
:10C0A00028B0BDE8F0872749E3E62749052238464E
:10C0B00015F015FA00284DD1244906F1080212F8AE
:10C0C000013F2BB96068202206F109010430BBE76B
:10C0D0003A2B09D8292BF2D92A3BDBB221FA03F3F8
:10C0E000DB07ECD51A49C4E63F2BFBD05B3B022BA8
:10C0F000E5D8F7E7C64402080000C842D144020868
:10C1000000002041F0440208FD44020801450208F5
:10C110000D450208B54E02081245020826450208E0
:10C12000424502084E4502085F450208764502086E
:10C13000654502089B450208C3450208D34502082D
:10C14000DC450208FE4502080D4602080500010014
:10C15000144802089D490722384615F0C0F9C0B9B5
:10C160009B49032206F10B0015F0B9F96368B0FA98
:10C1700080F0400983F84D002046FFF705FE636814
:10C18000944A93F84D10944B00290CBF1146194660
:10C190006FE692490622384615F0A1F9804600283C
:10C1A00057D104F11C0306F10A0118461E4615F08A
:10C1B000F8FA2C23042210A93046FFF76DF8071E69
:10C1C00045DD1098414614F0F3FE012F82463ED023
:10C1D0001198414614F0ECFE022F814637D0129898
:10C1E00013F056FF032F064604D0139813F050FFA8
:10C1F0005FFA80F87A495046F4F766FF38B3794918
:10C200005046F4F757FF10B3F6B2731F072B1ED832
:10C21000A8F10503032B1AD873494846F4F754FFD5
:10C22000A8B172494846F4F745FF80B1636883F8C6
:10C230007060636883F871806368A068C3F848A081
:10C24000C3F8749003681B689847694911E6694907
:10C250000FE669490422384615F041F938B906F16C
:10C260000800676813F011FFC7E90A0147E6634950
:10C270000422384615F033F938B906F1080067682A
:10C2800013F003FFC7E90C0139E65D49082238467F
:10C2900015F025F9A0B906F10C0013F0F6FEF4F73D
:10C2A00003FC00210646F4F70FFF38B1554930462C
:10C2B000F4F700FF10B163681E6520E65249D8E527
:10C2C00052490822384615F00AF9A8B906F10C00BF
:10C2D00013F0DBFEF4F7E8FB00210646F4F7F4FE6A
:10C2E00040B14FF080413046F4F7E4FE10B163688E
:10C2F0005E6504E64649BCE546491322384615F01A
:10C30000EEF860B906F1170013F0C2FEC0B2402883
:10C3100003D8636883F87900F1E53F49A9E53F490F
:10C320001122384615F0DBF850B906F1150013F06C
:10C33000AFFEC0B24028F0D8636883F87A00DEE52B
:10C3400037491222384615F0CAF850B906F11600DE
:10C3500013F09EFEC0B24028DFD8636883F87B00EC
:10C36000CDE530491722384615F0B9F850B906F135
:10C370001B0013F08DFEC0B24028CED8636883F84E
:10C380007C00BCE528491322384615F0A8F850B9BE
:10C3900006F1160013F07CFEC0B24028BDD86368D9
:10C3A00083F87D00ABE521490A22384615F097F85D
:10C3B00000283DD106F10E0013F06AFEC0B24028FD
:10C3C000ABD8636883F8780099E500BF134602088C
:10C3D00076490208B0440208994402086D4D0208EB
:10C3E0000000164300401C450000E0400000FA43F6
:10C3F0001B460208304602084C4602085146020815
:10C40000564602080000A0415F4602080B4702089A
:10C4100073460208864602089A460208A8460208A1
:10C42000BA460208CD460208E5460208F946020867
:10C4300071490F22384615F052F8B8B906F11300C9
:10C4400013F023FEF4F730FB00210646F4F73CFE20
:10C4500000283FF44FAF4FF080413046F4F72AFEFA
:10C4600000283FF447AF63689E6648E563490B22A6
:10C47000384615F034F898B963680E36B03316F8BC
:10C48000011F21B16268B0329A1A762A02D90022BD
:10C490001A7034E57C2908BF0A2103F8011BEEE776
:10C4A00057490F22384615F01AF860B906F1130003
:10C4B00013F0EEFDC0B2022803D8636883F82901A7
:10C4C0001DE55049D5E450490C22384615F007F8CF
:10C4D00018BB10364D490322304615F000F8A0B1C4
:10C4E0004B490722304614F0FAFF68B14949082247
:10C4F000304614F0F4FF60B147490622304614F08C
:10C50000EEFF40B14549B4E40120636883F82A0195
:10C51000F5E40220F9E70320F7E741490322384612
:10C5200014F0DDFF88B9F01D13F0B2FD636883F8E5
:10C530004C002046FFF728FCD4E90120036892F95B
:10C540004C10DB6A9847374993E4B9F1000F11D1D9
:10C5500035490522384614F0C2FF58B906F10900E2
:10C5600013F093FDF4F7A0FA6668B0642046FFF775
:10C570000BFC6AE62D490F22384614F0B0FF68BB69
:10C5800006F1130013F081FDF4F78EFA636801469B
:10C59000C3F8AC00E06803689B689847C0B12046C8
:10C5A000FFF7F2FB6368D3F8AC4000212046F4F7B4
:10C5B0006DFD08B11E495CE42046F3F725FF0B46EC
:10C5C0001C490246284628B0BDE8F04714F0C6BE14
:10C5D000636819490022C3F8AC204AE41749284689
:10C5E00015F0DFF88F22394605F1100028B0BDE8BC
:10C5F000F04701F0B3BF00BF044702081447020828
:10C6000020470208304702084947020876490208D5
:10C610007C490208864902089149020856470208E7
:10C62000884702084A3E02088C47020892470208DF
:10C63000A2470208C6470208E24702080348020868
:10C640002DE9F04102F1040896B005460F46164662
:10C65000A349092240461C4614F041FF28BB6B68E1
:10C660004FF07E511868F4F775FA01469D48F4F7CB
:10C670002DFC0646F4F752FD0546F4F71FFB014674
:10C680003046F4F765FA9849F4F76CFB4FF07C51AB
:10C69000F4F760FAF4F742FD944903462A4620462F
:10C6A00016B0BDE8F04114F059BE9149022240464F
:10C6B00014F015FF28B96B68186801F069FF02468D
:10C6C00018E08C490A22404614F009FF20B96B6833
:10C6D00093F87E2088490EE088490322404614F0F2
:10C6E000FEFE70B96B6893F82B11854A854B0029C3
:10C6F00018BF1A468449204616B0BDE8F04114F030
:10C700002DBE82491222404614F0E9FE20B96B6822
:10C7100093F87F209200DDE77D490A22404614F01D
:10C72000DEFE18B96B6893F87320D3E779490F22BE
:10C73000404614F0D4FE18B96B6893F87210D4E731
:10C7400075491522404614F0CAFE18B96B6893F873
:10C750004F20BFE771490F22404614F0C0FE20B9B8
:10C760006B6893F84E205200B4E76D490E224046A4
:10C7700014F0B5FE10B96A685832BBE7DFB96949F1
:10C780000722404614F0ABFEA8B9A86803685B6CAA
:10C790009847402206A9FDF78BFE1C35024606A9E4
:10C7A0002846FEF71DFD58492A46204614F0D6FDBE
:10C7B00016B0BDE8F0815C490422404614F08FFEBB
:10C7C00010B96A68043295E758490622404614F0C9
:10C7D00086FE28B96B684B4A93F84D10484B86E7A4
:10C7E00053490322404614F07AFE28B96B68D3E916
:10C7F0000A01F4F759F960E74E490322404614F064
:10C800006EFE18B96B68D3E90C01F2E74A490522BC
:10C81000404614F064FEE8B96B68986C01F0B8FE0D
:10C82000014602A814F0BDFF6B68586F01F026FFA7
:10C83000014606A814F0B5FF6B68404993F87120D3
:10C84000019293F87030009302AA06AB204614F0D0
:10C8500085FDADE73A490722404614F040FE10B985
:10C860006B68186D29E737490722404614F037FEF8
:10C8700010B96B68586D20E733491022404614F018
:10C880002EFE18B96B6893F87A2023E72F491222FD
:10C89000404614F024FE18B96B6893F8792019E724
:10C8A0002B490922404614F01AFE18B96B6893F818
:10C8B00078200FE727491122404614F010FE18B9DE
:10C8C0006B6893F87B2005E723491622404614F055
:10C8D00006FE002842D16B6893F87C20FAE600BF80
:10C8E000254802080000C842000020412F480208E5
:10C8F00039480208414802084C48020851480208D9
:10C9000076490208B54E02083C480208554802081C
:10C9100068480208734802088348020889480208E8
:10C9200099480208A8480208AC4A0208B048020820
:10C93000B7480208BB480208034F0208BF48020874
:10C94000CD48020846490208D5480208E6480208D0
:10C95000F948020803490208154902086C491222E5
:10C96000404614F0BCFD18B96B6893F87D20B1E621
:10C9700068490E22404614F0B2FD10B96B68986EFB
:10C980009BE665490A22404614F0A9FDB0B923464A
:10C990003E2203F8022B202262706968AF3111F841
:10C9A000012F12B900221A7002E7181B9E28F9DC29
:10C9B0000A2A08BF7C2203F8012BF0E757490E2210
:10C9C000404614F08CFD18B96B6893F8292181E674
:10C9D00053490B22404614F082FD98B96B6893F8D6
:10C9E0002A3133B94F49204616B0BDE8F04114F062
:10C9F000D8BE012B01D14C49F5E7022B0CBF4B49A6
:10CA00004B49F0E74B490222404614F068FD38B923
:10CA1000B37913F0DF0F03D16B6893F94C2059E61B
:10CA200045490422404614F05AFD10B96B68986CD1
:10CA300043E642490A22404614F051FD78B9404984
:10CA4000204614F0AEFEA86803685B6C984720226D
:10CA50000146A01C16B0BDE8F041FEF7C1BB394944
:10CA60000422404614F03BFD20B9A8680368DB6847
:10CA7000984724E634490B22404614F030FD08B9AB
:10CA8000324A37E632490E22404614F028FD08B9F2
:10CA90003049A8E730490E22404614F020FDB0B9D5
:10CAA000E8680368DB68984700210546F4F7EEFA6A
:10CAB00008B12A4997E72846F3F7A6FC0B46284910
:10CAC0000246204616B0BDE8F04114F047BC2549A7
:10CAD0000E22404614F003FD08B9234983E7234999
:10CAE0000D22404614F0FBFC08B921497BE721499F
:10CAF0001122404614F0F3FC0028F6D01E490D2206
:10CB0000404614F0ECFC0028EFD01C494246F2E508
:10CB10002C4902083F4902084E49020859490208B7
:10CB200068490208744902087A49020884490208DF
:10CB30008F490208984902089B490208A049020847
:10CB400041400208AB490208B0490208BC4902084A
:10CB5000C1490208D0490208E3490208E247020835
:10CB6000F2490208F9490208084A0208164A02086E
:10CB7000244A02084A4A02085C4A02086A4A020831
:10CB80002DE9F04F0023137089B005460F46144677
:10CB90000B461E4601333278202AFAD096490A22E3
:10CBA000304614F0ECFC002878D1B37A13F0DF0F94
:10CBB00074D106F10A031E4601333278202AFAD0D6
:10CBC0003046FEF785FE337833B98C49204609B0EC
:10CBD000BDE8F04F14F0E5BD6B694FF0000903F2BA
:10CBE0008C483378202BB34606F10106F9D0002B90
:10CBF0004CD05B461A781E46013322B1202AF9D167
:10CC000086F800901E46D5F814A05B461A4613F825
:10CC1000017B6FB17C2F01D02C2FF7D182F80090CF
:10CC20001F4613F8012B202AFAD03846FEF750FE93
:10CC300059461BF8013B202BFAD00BB97049C5E7C8
:10CC40001FB13B780BB96F49C0E7B8F800200391DA
:10CC50000023504601F094F80399804640B96A4A8F
:10CC60000B46A021204609B0BDE8F04F14F042BBAE
:10CC700080F80490002FB4D03946504601F0CEF829
:10CC800080460028ADD1614A3B46EAE76869A022A8
:10CC9000214609B0BDE8F04F01F0ACB93846202379
:10CCA000042204A9FEF7F8FA0128074607D16869AB
:10CCB000A022214601F09EF909B0BDE8F08F40F3B3
:10CCC0006481059E52493046F4F788FA20B9A86875
:10CCD00003685B6D9847EFE74E493046F4F77EFAFC
:10CCE00098B9D5E9000603681B689847C6F8A800FC
:10CCF0002846FFF749F8A86803689B6D9847464A9D
:10CD00004649002808BF114660E7022F64D0444915
:10CD10003046F4F763FA60B90699686901F07EF865
:10CD200028B1037923F0010303713C494EE73D49E3
:10CD30004CE73D493046F4F751FA48B9069968691D
:10CD400001F06CF80028F2D0037943F00103EBE71F
:10CD500036493046F4F742FA38BB0699686901F063
:10CD60005DF806460028E2D04188686901F094F831
:10CD70003379721D70B1018861B12D4913F0010F33
:10CD80002C4B18BF0B4600932B49431D204614F033
:10CD9000E5FA91E7274913F0010F2046244B08BF1D
:10CDA0000B46264914F0DAFA86E725493046F4F7AF
:10CDB00015FA00284CD10699686901F02FF806464B
:10CDC0000028B4D00146686901F081F81D49721D40
:10CDD000204614F0C3FA6FE719493046F4F7FEF91C
:10CDE000002872D1686901F06FF810B1421D164930
:10CDF000EEE7164AFBE700BF854A0208904A0208A0
:10CE0000A04A0208B14A0208C24A0208D74A0208E8
:10CE1000EE4A0208F34A0208714A02084A3E020832
:10CE2000F84A0208FF4A0208144B02081A4B02088B
:10CE300042DB020898DF02081E4B02082A4B020858
:10CE4000314B0208364B0208464B0208834A02085F
:10CE50004F493046F4F7C2F9002845D1069F4D49A5
:10CE60003846F4F7BBF9064668696EB9314601F0F9
:10CE700038F8A86803683146DB6D9847A8680368EE
:10CE80009B6D98474449A1E6394600F0C7FF064626
:10CE900038B9034602460699686900F071FF0646F4
:10CEA00088B1002333716869314601F01AF8A86827
:10CEB00003683146DB6D9847A86803689B6D984707
:10CEC0003649721D84E7364980E631493046F4F729
:10CED00085F9002859D1686900F0FDFF10B1421DA5
:10CEE000304975E72B4AFBE72F493046F4F776F9CE
:10CEF000B8B9032F686905D0079900F08FFF18B9FA
:10CF00002A4963E600F28C4002880699686900238A
:10CF100000F036FF08B9264958E600232549037179
:10CF200054E625493046F4F759F978B90699686905
:10CF300000F0F6FE014638B1686900F0D6FF00281F
:10CF40007FF4F3AE1D4941E61D493FE61D493046D9
:10CF5000F4F744F9C8B9069E1B493046F4F73EF988
:10CF600038B11A493046F4F739F908B118492DE6B5
:10CF70000120009068690123A022214601F054F8A5
:10CF800000287FF499AE134920E613491EE600BF3E
:10CF9000524B0208704B02085A4B0208774B0208AA
:10CFA000904B0208A84B0208E24B0208BD4B020856
:10CFB000D24B0208E64B0208FB4B0208024C020867
:10CFC000124C0208324E0208224C02082A4C020877
:10CFD000314C0208973C0208514C02082DE9F04FF1
:10CFE00014468DB00546884608227A4920461E46DA
:10CFF00014F075FA28B178490822204614F06FFA27
:10D0000030B9E86803681B6A0DB0BDE8F04F1847F7
:10D0100072490622204614F062FA18B9E8680368DB
:10D02000DB69F1E76E490922204614F058FA28B965
:10D0300028686C4903685B689847EFE76A490E22E5
:10D04000204614F04CFA80B9A27B12F0DF020CD11A
:10D05000A868036840F2DC515B6998476349304631
:10D060000DB0BDE8F04F14F09CBB6149062220468C
:10D0700014F035FA40B9A868036840F2DC515B69E6
:10D08000012298475B49EAE75B490A22204614F0EF
:10D0900026FA30BB286803681B68984780451ED96C
:10D0A000286803685B6808F10101984728680368ED
:10D0B0001B689847014604A808F0CEF99DF8103087
:10D0C0009DF813204D4903F5FA6302939DF8113042
:10D0D00001939DF8123000939DF814302FE04849D9
:10D0E000BDE748490922204614F0F9F948B9E86833
:10D0F0006968036832461B6C0431984710BB42498B
:10D10000ADE742490522204614F0E9F9E8B928685C
:10D1100003681B689847014604A808F09DF99DF82C
:10D1200010309DF813203A4903F5FA6302939DF8F5
:10D13000113001939DF8123000939DF81430304661
:10D1400014F00CF90DB0BDE8F08F324905222046ED
:10D1500014F0C5F980B9601DFEF7ACFB04462868E1
:10D1600003681B689847844204D9286803682146ED
:10D170005B689AE7284972E728490922204614F09B
:10D18000AEF938B9A86803681B6B31460DB0BDE82D
:10D19000F04F184722491022204614F0A0F9002829
:10D1A00044D110342046F4F723F8402828BF40200B
:10D1B00047102246394604A8FEF74AF838B1A86855
:10D1C000036804A95B6B3A469847164947E7164936
:10D1D00045E700BF634C02086C4C0208784C02081B
:10D1E000754C0208EF9344667F4C02088E4C02088F
:10D1F000DF480208A74C0208B84C0208C34C0208DA
:10D20000EC4C02080B4D0208154D02081B4D02089C
:10D21000D34C0208214D0208274D02088F3E020818
:10D22000484D02084A3E0208594D0208A2490A2206
:10D23000204614F054F9074600286BD105F11C0371
:10D2400004F10A0118461C4614F0ABFA2C230522FF
:10D2500004A92046FEF720F8B0F1000858DD049834
:10D26000394613F0A5FEB8F1010F834646D0059864
:10D27000002113F09DFEB8F1020F814643D00698BD
:10D2800012F006FFB8F1030F5FFA80FA3ED007985C
:10D2900012F0FEFEB8F1040FC4B203D0089812F0E9
:10D2A000F7FE074685495846F3F70EFF80B38449D9
:10D2B0005846F3F7FFFE58B3AAF10503072B27D80A
:10D2C000631F032B24D87F494846F3F7FDFEF8B1CE
:10D2D0007D494846F3F7EEFED0B1002F18DDA8686F
:10D2E0000368CDE900474A461C6D59465346A0479E
:10D2F00076493A46304614F031F823E70024A24636
:10D300004FF00009CEE70024A246CBE70024C9E78E
:10D310006F49A4E66F490922204614F0E0F8B8B935
:10D320006868102204F10901383001F017F9284625
:10D33000FEF72AFD6849304614F033FA69689122F5
:10D34000383106F10E000DB0BDE8F04F01F006B91E
:10D3500062490B22204614F0C2F828B9A868036875
:10D36000DB6C98475E497AE65E490422204614F059
:10D37000B6F840B933462246414628460DB0BDE8CE
:10D38000F04FFFF75DB958490422204614F0A7F882
:10D3900040B933462246414628460DB0BDE8F04F1D
:10D3A000FEF746BDB8F1000F14D150492046F3F7FF
:10D3B00015FF78B9A86803681B6998474C4A4D4B1C
:10D3C0004D49002818BF1A4630460DB0BDE8F04F51
:10D3D00013F0C4BF49490322204614F080F888B9ED
:10D3E000A86803685B6898470446A86803689B6858
:10D3F000984743490346224630460DB0BDE8F04FFA
:10D4000013F0ACBF3F490522204614F068F828B954
:10D41000E86803681B699847014620E63A490B22F1
:10D42000204614F05CF80746F8B904F10B082C69A3
:10D4300023682046DB6898470546BD420FDD236818
:10D4400039461B69204698474146F3F7C7FE40B965
:10D45000236839465B6920469847024618B92B492C
:10D46000FDE50137E9E72A49AEE72A490B222046C4
:10D4700014F035F8002855D105F11C0304F10B0117
:10D4800018461C4614F08DF92023022204A92046D8
:10D49000FDF702FF00280ADD0128049908D0059A4B
:10D4A000286903689B69984720B11B49D7E51B4948
:10D4B000164AF5E71A49D2E5694D020800001643FD
:10D4C00000401C450000E0400000FA43744D020893
:10D4D000914D0208C9450208A74D0208B64D020841
:10D4E000C24D0208014E02080D4E0208D44E020839
:10D4F0005A4C02084A3E0208D54D0208CC4902089F
:10D50000EB4D0208FD470208FA4D02085E4C020886
:10D510003C480208064E0208124E020842DB02088E
:10D52000154E02086E490B22204613F0D8FF07461D
:10D53000002842D128690368DB6898478046204666
:10D54000F3F756FE0B2804D904F10C00FEF7B2F9EC
:10D550000746474501DB634981E56349DFF88C9164
:10D560004246304613F0FAFE3046F3F741FE3418D7
:10D57000A31B852B05DDB8451BDD5D493A462046DA
:10D5800023E72869036839461B699847824628695A
:10D59000036839465B699847524603464946204628
:10D5A00013F0DCFE2046F3F723FE0137B8450444B0
:10D5B000DED1002304F8013CC4E54E490622204692
:10D5C00013F08DFF38B93246214628460DB0BDE82C
:10D5D000F04FFFF7D5BA48490E22204613F07FFFDF
:10D5E00008B946493BE546490F22204613F077FF2C
:10D5F00038B96B6883F89D002846FEF7C5FB4149A2
:10D600002DE541490B22204613F069FF30B96B68C4
:10D6100093F89D30002BF2D03C4920E53C4909228B
:10D62000204613F05CFF30B9A868036801211B6A2B
:10D630009847384913E538490822204613F04FFF30
:10D64000014628B9A86803681B6A9847334906E56C
:10D6500033490922204613F042FF28B9A86803681D
:10D660005B6A98472F49FAE4B8F1000F35D12E498B
:10D670000322204613F033FF28B9A86803689B6A89
:10D6800098472A49EBE42A490D22204613F027FF48
:10D6900038B9637B13F0DF0F03D1A86803681B6CF4
:10D6A00073E524490B22204613F019FF38B9E37AB9
:10D6B00013F0DF0F03D1A8680368DB6B65E51E4933
:10D6C0000A22204613F00BFF38B9A37A13F0DF0FBC
:10D6D00003D1A86803689B6B57E51849BFE400BFF6
:10D6E0002B4E0208374E0208454E02084E4E0208E5
:10D6F000554E02080D4B0208614E0208704E02089A
:10D70000844E020876490208944E0208B54E02087B
:10D71000A04E0208AA4E0208B84E0208C14E0208E6
:10D72000D04E0208DA4E02088A3C0208E84E02088F
:10D73000EF4E0208FD4E0208094F0208144F02087E
:10D7400030B50D46CBB09F490446284607F0F7FF99
:10D7500002A89C4A0123294607F0DBFF02A808F033
:10D7600040F9002800F02C8100236168042202A8FF
:10D77000CDE9003307F0F7FF61682022043102A8E9
:10D7800007F0F1FF0422694602A807F0ECFF616888
:10D79000082228310DEB020007F0E5FF616808223E
:10D7A00030310DEB020007F0DEFF616810223831E6
:10D7B00002A807F0D8FF61680422483102A807F0E8
:10D7C000D2FF616801224C3102A807F0CCFF6168EA
:10D7D00001224D3102A807F0C6FF616801224E31D7
:10D7E00002A807F0C0FF0122694602A807F0BBFFAC
:10D7F00061680422503102A807F0B5FF6168042275
:10D80000543102A807F0AFFF61681022583102A816
:10D8100007F0A9FF61680422683102A807F0A3FF9E
:10D820000422694602A807F09EFF61680122703158
:10D8300002A807F098FF61680122713102A807F081
:10D8400092FF61680122723102A807F08CFF6168C3
:10D850000122733102A807F086FF61680422743147
:10D8600002A807F080FF616801227F3102A807F05B
:10D870007AFF6168012201F2291102A807F073FF03
:10D880006168012201F5957102A807F06CFF012281
:10D89000694602A807F067FF61680122783102A893
:10D8A00007F061FF616801224F3102A807F05BFFBA
:10D8B000616801227E3102A807F055FF61680122EC
:10D8C000803102A807F04FFF61680222823102A86E
:10D8D00007F049FF61680122843102A807F043FF85
:10D8E00061680422883102A807F03DFF61680122C7
:10D8F0008C3102A807F037FF616810228D3102A831
:10D9000007F031FF616801229D3102A807F02BFF6B
:10D910000322694602A807F026FF616801229E31B2
:10D9200002A807F020FF61680422A03102A807F0D6
:10D930001AFF61680122A43102A807F014FF616890
:10D940000422A83102A807F00EFF61680422AC315E
:10D9500002A807F008FF61687822B03102A807F03A
:10D9600002FF6168012201F5947102A807F0FBFE35
:10D9700061680122793102A807F0F5FE6168012291
:10D980007A3102A807F0EFFE6168012201F22B1143
:10D9900002A807F0E8FE616801227B3102A807F0C7
:10D9A000E2FE616801227C3102A807F0DCFE6168BA
:10D9B00001227D3102A807F0D6FE02A807F0C9FFB8
:10D9C0004BB030BD244F020838B50C46054610490F
:10D9D000204607F0A8FE30B1214628460C4ABDE893
:10D9E0003840FDF785BF0B49204607F09CFE70B11B
:10D9F00021462846074AFDF77BFF21462846FFF7C8
:10DA00009FFE20460349BDE8384007F098BE38BD68
:10DA1000244F02082F4F020870B50546D2B00B46BE
:10DA2000164610494268684613F098FC2868694613
:10DA300007F079FE044690B1296800236A460AA8D7
:10DA400007F067FE0AA807F0CCFF044638B10AA920
:10DA50003046FCF7FDFC04460AA807F07AFF204692
:10DA600052B070BD3B4F020830B50446D3B00B46F0
:10DA700015460F494268684613F070FC20686946F5
:10DA800007F05DFE216801236A460AA807F041FEFF
:10DA90000AA807F0A6FF044630B10AA92846FCF7F9
:10DAA000EEFC0AA807F055FF204653B030BD00BF7A
:10DAB0003B4F020800207047836910B544695A1C27
:10DAC000A24208D204698261E1540269836900219B
:10DAD000D154012010BD0020FCE7F8B505460F46E3
:10DAE00016460024B44201D12046F8BD2B68395DAA
:10DAF0001B68284698470028F6D00134F2E700203A
:10DB000070474FF0FF3070474FF0FF30704770475D
:10DB100010B500230122C0E9012304460160C0F8CA
:10DB20008C3480F89034034900F2914013F039FEB0
:10DB3000204610BD834A0208A0F12303DBB2162B56
:10DB400004D8064A42FA03F3DB0704D5402894BF01
:10DB50000020012070470120704700BFFC1B80FFA0
:10DB6000F0B5434B0D46002A14BF16461E46E9B0D9
:10DB700004463146284607F0D6FD18B9002630463F
:10DB800069B0F0BD32460023294620A807F0C1FD48
:10DB900020A807F026FF06460028EFD00023012723
:10DBA000C4E901730322694620A807F098FE032800
:10DBB00003D020A807F0CDFEE1E7022204F108011E
:10DBC00020A807F08CFE02280246F2D1A11D20A851
:10DBD00007F085FE02280546EBD13A4604F592612E
:10DBE00020A807F07CFE0128E3D12A46211D20A8A9
:10DBF00007F075FE0228DCD1242765891F2DD8D8AF
:10DC00007D4305F10C010222214420A807F067FEA4
:10DC100002280246CDD105F10E01214420A807F0CB
:10DC20005EFE0228C5D105F111011F22214420A862
:10DC300007F055FE1F28BCD105F110010122214437
:10DC400020A807F04CFE0128B3D1802269460DEBD5
:10DC5000020007F044FE8028ABD12544A288AB899E
:10DC60009A429CBF0133A380638901336381C4E777
:10DC7000444F020870B50C464979242988B00546FE
:10DC8000164606D12188006808B0BDE8704000F053
:10DC9000C3BB232904F1050207D133462868218834
:10DCA00000F01FFC012008B070BD232311460DF1C8
:10DCB00001008DF8003013F074FD33466A46EDE73D
:10DCC0002DE9F04F054691B00F46904600F10C0645
:10DCD0004FF000096B894B4505DC4FF0000A5046B8
:10DCE00011B0BDE8F08F347918EA0404B24608D1C7
:10DCF00004236A4631462846FFF7BCFF83465C454D
:10DD000003DB09F101092436E4E739460DEB041081
:10DD100000F0AAFBFB888342E1D00134EFE700006A
:10DD20002DE9F0410D46064614492846F3F756FA08
:10DD300018B906F28C40BDE8F0812B78B6F80A805D
:10DD4000232B08BF013506F112070024444501DBEF
:10DD50000020F0E717F8013C232B3946284618BF6E
:10DD600007F1FF31F3F73AFA243720B9242303FBF4
:10DD700004600C30DFE70134E8E700BF834A0208A3
:10DD80002DE9F8438846054617461E46013911F825
:10DD9000019FB9F1000F0AD141462846FFF7C0FFA5
:10DDA000044668B10388BB4235D0478005E0484649
:10DDB000FFF7C2FE04460028E9D12046BDE8F883FB
:10DDC0006889C6B1431C6B812423434303F10C04CF
:10DDD0002B4401222C441A742423584305EB0009D8
:10DDE0001130A9F80C601F224146284400F0B6FB10
:10DDF000A9F80E70E1E71F28DFD8431C6B812423AC
:10DE0000434303F10C042B4401221A74AE88B31867
:10DE10002C44AB80E0E74C46CFE700002DE9F0470B
:10DE20000D4604461B492846F3F7D8F920B904F2F9
:10DE30008C442046BDE8F0872B78B4F80AA0232B49
:10DE40004FF0000708BF013504F10C06B846BA458B
:10DE500001DC4446EDE77379232B14BF06F1050975
:10DE600006F10609494628463446F3F7B7F9002873
:10DE7000DFD02846F3F7BCF949460246284613F09E
:10DE80002EFB00280CBF3446444601372436A046FA
:10DE9000DDE700BF834A0208F0B541B144890023A1
:10DEA000242500F10C06A34204DB002001E000F26F
:10DEB0008C40F0BD05FB03F2B75A8F4202D10C3201
:10DEC0001044F6E70133EEE7C188FFF7E5BF01B183
:10DED0000988C1807047018909B1FFF7DDBF084695
:10DEE000704701B1098801817047F8B50B8863B1AB
:10DEF0004189002200F10E042425914207DC002410
:10DF000000F10C022426A14208DC00201DE005FBE4
:10DF100002F6A65B9E42F8D00132EEE706FB04F55E
:10DF2000575B9F4201D00134EDE74B1E9BB21A1B99
:10DF300005F1300172430C35438101449C42C8BF56
:10DF40000022284413F0DBFA0120F8BD2DE9F84344
:10DF50000546884614461E46002747451DDB2179A5
:10DF60006379208811F0010F04F10502E9881AD0C5
:10DF7000232B194F194B08BFA21D884218BF3B46DF
:10DF8000174930460FF0B1F905F10C074FF00009C1
:10DF90006B894B4511DCBDE8F883202130460FF03A
:10DFA0007BF90137D9E7232B0B4F0C4B08BFA21D80
:10DFB000884218BF3B460B49E3E77A8823889A4298
:10DFC00006D133463A4608F101012846FFF7BEFF65
:10DFD00009F101092437DBE742DB02084E4F020852
:10DFE0006DDD0208504F02080B4600F28C42002102
:10DFF000FFF7ACBF10B588B091B172B100234FF4F8
:10E000007A74CDE90512CDE902340B70054C019408
:10E0100001A90793FFF7E8FF079A104608B010BD63
:10E020000A46FAE7604F02082DE9F74F98469DF837
:10E0300030A090F89034009207460D4608EA03039A
:10E04000BAF1000F02D01BB92C4607E0002BFBD120
:10E050002C462A2304F8023B2C236B7007F112068E
:10E060004FF000094FF02C0B7A894A4509DCAC428D
:10E0700088BF04F1FF340023601B237003B0BDE8A8
:10E08000F08F16F8022C314608EA0202BAF1000FAE
:10E0900004D02AB909F101092436E5E7002AF9D1AB
:10E0A00016F8012C232A18BF06F1FF31084601910A
:10E0B000F3F79EF80246601B009B01991044023062
:10E0C0009842E7DA2046019213F073FB019A144458
:10E0D00004F801BBDEE70000F0B53B4B0D46002A1B
:10E0E00014BF16461E46E9B031460446284607F0DE
:10E0F00026FB32460123294620A807F00AFB20A868
:10E1000007F06FFC064670B180220021684613F0CC
:10E1100010FA0322694620A807F025FB032805D042
:10E1200020A807F016FC304669B0F0BD022204F1C9
:10E13000080120A807F017FB02280246F0D1A11D14
:10E1400020A807F010FB02280546E9D1012204F5BA
:10E15000926120A807F007FB0128E1D12A46211D82
:10E1600020A807F000FB0228DAD104F110050027EF
:10E170006389BB42D4DD0222291F20A807F0F3FAED
:10E1800002280246CCD1A91E20A807F0ECFA0228EA
:10E19000C6D11F22691C20A807F0E5FA1F28BFD1AD
:10E1A0000122294620A807F0DEFA0128B8D18022F2
:10E1B00069460DEB020007F0D6FA802805F1240528
:10E1C000AED10137D4E700BF444F0208806A7047E0
:10E1D00040697047836953F8210070476FF06043CE
:10E1E000994270B534BF8E004FF0FF36044630467A
:10E1F0000D46F7F76CFB20602846F7F768FB606078
:10E200003046F7F764FB0023C4E90205236120468A
:10E2100070BD4B1C30B5024605690DD00023184671
:10E22000AB4200DB30BD946854F82340641A002CE4
:10E23000D8BF01300133F3E72846F3E71830FFF782
:10E24000E8BF70B5024604694FF0FF330020FF2598
:10E2500084420ADC002B26DB1168013C51F82300C4
:10E260001461116999420EDC70BD966856F8206001
:10E27000761A002E05DC5668365CAE423CBF03467B
:10E2800035460130E4E7990014680431655844F8D4
:10E2900023505468E5186D78E5549468615844F843
:10E2A00023100133DDE70020DEE71830FFF7C9BF98
:10E2B0002C30FFF7C6BF02698A4230B5034618DD2D
:10E2C0000068013A50F821001A611A698A4200DC9C
:10E2D00030BD8A001C680432A55844F821505C689F
:10E2E00065186D7865549C68A25844F82120013166
:10E2F000EBE70020ECE700210430FFF7DCBF18302B
:10E30000FFF7D9BF30B5D0E90354AC420CD0056853
:10E3100045F8241041680A550269816841F82230A5
:10E3200001320261012030BD0020FCE700231A46C3
:10E330000430FFF7E7BF70B5044618300D46FFF70D
:10E34000E1FF30B92368294620465B68BDE870408C
:10E35000184770BD70B51346044600222C300D4698
:10E36000FFF7D0FF30B92368294620465B68BDE837
:10E370007040184770BD00002DE9F0410646134B70
:10E3800046F8043B04460D463046FFF727FF294672
:10E3900004F11800FFF722FF294604F12C00FFF7D3
:10E3A0001DFF0027AF4202DB2046BDE8F0814FF49D
:10E3B0008270F7F78AFA8046FCF781FE00231A463E
:10E3C00041463046FFF79EFF0137EBE78C4F0208CE
:10E3D000431E0F3013F8012F1AB98342FAD10120DE
:10E3E000704700207047F0B5D0F820510F2D04463B
:10E3F00011DCAB1C20F8151000EB031302F1100721
:10E40000106851681E4603C60832BA423346F7D137
:10E410000135C4F82051F0BD2DE9F047064600252E
:10E420008E46284606F12008D6F82011A94201DDC3
:10E43000984201DBBDE8F08736F81510714511D11F
:10E4400008EB051C00F1010902EB00140CF1100AA5
:10E45000674603CF574520606160BC4604F108045D
:10E46000F6D148460135DFE730B5A3B0054604A82C
:10E470000C4605F0D7FF10220DEB0200294606F0EE
:10E4800038F923780122C3F383030DF10D0104A8A9
:10E490008DF80D3006F0AEF8628804F14A0104A848
:10E4A00006F0A8F802231022009329460DF10E036E
:10E4B0000DEB020006F035F9BDF80E3053B901231B
:10E4C000ADF80E3004A8BDF80E4005F091FF2046CF
:10E4D00023B030BD4FF6FF729342F3D14FF6FE7377
:10E4E000EEE72DE9F0419846D0F820319EB0054680
:10E4F0000E4617460024A34218DC684605F092FF3A
:10E500003846F2F775FE39460246684606F072F85C
:10E5100041466846102206F09FF82846424631469A
:10E52000FFF761FF684605F063FF12E035F814203D
:10E53000B24211D1023405EB0414424604F1100337
:10E54000254603CD9D42106051602C4602F1080221
:10E55000F6D11EB0BDE8F0810134CCE701390244A8
:10E56000131A012B02D800230370704711F8013FE2
:10E57000002BF8D000F8013BF2E7013810F8013F1A
:10E580000BB901207047202BF8D000207047000005
:10E5900070B500210646F2F779FD374C054640B1CB
:10E5A000302323702E22A37000236270E370324860
:10E5B00070BDC6F3C7537F3B1E2B99B257DC13F1D6
:10E5C000170F54DBC6F31602162B42F4000216DDB9
:10E5D000173902FA01F0002E40DB0A2221460FF023
:10E5E0009FF8237822460134002BFAD12E23137092
:10E5F000EDB93021931C517000221A70D7E7002B1F
:10E6000008DBC1F11700013142FA00F08A4022F024
:10E610007F45E0E7DB43002E42FA03F54FF030037D
:10E6200020DA63702D222E232270A3700334E11DA3
:10E6300023460A2045432A16303203F8012B8B4229
:10E6400025F07F45F6D106342278302A234603D1BF
:10E6500014F8012D2E2AF7D10133CDE72D2304F82C
:10E66000013BBAE723702E2363700234DFE73023C7
:10E670002370002363709AE72031002037B52049CA
:10E680000546F2F76FFB002104462846F2F71CFD11
:10E6900070B34FF07C512046F2F75CFAF2F73EFD82
:10E6A0004FF47A7290FBF2F302FB13000028154C32
:10E6B000154AB8BF404210210090204612F01AFEC1
:10E6C0002046F2F795FD0021431E2044002B03DD78
:10E6D00010F8012C302A0ED00A48F2F789FD0138D3
:10E6E000235C2E2B04BF00232354064803B030BD07
:10E6F0004FF03F41CFE700F8011D013BE6E700BFC7
:10E7000000007A4410310020B84F0208024A137802
:10E7100043F01003137070473031002038B50446C1
:10E72000406812490368D3F8B03098472368204600
:10E730005B6D9847034684F8240060680268082BE4
:10E740008CBF10212021126E9047094BA068002534
:10E750001D7003689B6B9847012801D1FFF7D6FF16
:10E76000A5612577E583256238BD00BF0DE7000868
:10E7700030310020C38B41833F2B82BF0023C383F2
:10E7800003627047034B187800F0EF00431E5842B5
:10E7900058417047303100202DE9F041174E347850
:10E7A00014F0100405460F46904616D040680368E2
:10E7B0000121DB6E9847041E0DDD6868444503683F
:10E7C000A8BF44461B6B22463946984790B16B69F7
:10E7D00001336B610024002333703378012B06D0A2
:10E7E000686803689B69984708B90123337020461D
:10E7F000BDE8F081EB680133EB60ECE730310020DD
:10E80000406808B50368DB6F98474FF47A73B0FB34
:10E81000F3F008BD10B50446406803689B6A98474A
:10E82000A06803689B699847014B00221A7010BDCD
:10E830003031002040680368D3F89C30184700004E
:10E8400070B5094E3378DB0604460CD403681B6CA4
:10E850009847054638B9236820465B6C9847357061
:10E860002583E583256270BD3031002010B5174B3C
:10E870001A78C38B012A044617D13F2B17D8036897
:10E880001B6C984780B9236820461B6D9847F2F7A8
:10E8900045FCB4F918300D33984205DCE38B0133A5
:10E8A000E383236A0344236210BD3F2BFCD9236A10
:10E8B000002BF9D0B8BF3F3343F38F136FF07702CB
:10E8C0009342B8BF134623830023ECE73031002086
:10E8D00006490B78024613F0100005D000230B7098
:10E8E0001369013313610120704700BF30310020EC
:10E8F0000739234B2DE9F04153F8218004460146A6
:10E9000040461546F2F7EAFBC0BB2846F1F76AFD20
:10E910001C4B0022F1F7D0FD02460B4600201A499D
:10E92000F1F712FC06460F4620464146F2F710F971
:10E93000F1F76AFD154B0022F1F7E8FE02460B469F
:10E9400030463946F1F7B8FD0F4B002204460D461C
:10E95000F2F724F860B10022002320462946F2F79E
:10E960003BF840B120462946F2F79EF8BDE8F08119
:10E97000054D0024F6E700240025F3E70020F5E725
:10E98000C04F02080000703F0000F03F000024402C
:10E9900040686FF0004104F028BD406803685B6D7B
:10E9A00018470000406808B503681B699847024B88
:10E9B00000221A7008BD00BF30310020F8B50446AF
:10E9C000806803685B690D4616469847606803686F
:10E9D00032465F6A29460023B84720B9064B032216
:10E9E0001A700120F8BD2046FFF7DCFFA06803681D
:10E9F0009B6998470020F5E730310020406808B552
:10EA000003689B69984710B9014B01221A7008BD31
:10EA10003031002038B5B0F91A30044613B9207FE0
:10EA200098B938BD03681B6D9847B4F91A3005468C
:10EA3000B4F918001844F2F741F901462846F2F7F4
:10EA40004DFB0028EBD00120EBE7236820469B6DAF
:10EA50009847064B0546002220461A70FFF7CEFF66
:10EA600015F10F0018BF0120DBE700BF3031002097
:10EA70000846114606291A4601DDFFF739BF002076
:10EA80007047002070470000F0B51D4F1D4CD7F8AF
:10EA9000E03585B0002200921B4A04EA832303EB91
:10EAA000C12307CA01AD85E80700D7F8E02504EACD
:10EAB000822203F1FF6602F1FF6106F5F02601F5FF
:10EAC000F021B14218D802F10062013AB24213D3E8
:10EAD000A3F50043DB0A0293F3F754FA694628468C
:10EAE000F3F7E2FA0446F3F75FFA002C14BF6FF075
:10EAF0000400002005B0F0BD6FF01500FAE700BF7C
:10EB00000070FF1F00FCFF038C3502082DE9F04761
:10EB1000204E214FD6F8E04507EA842404F1FF6433
:10EB200004F5F02414441D4604EBC124F3F72AFA3B
:10EB3000804678B9089B23F0070303EB04096FF0C4
:10EB4000784AA1450AD1F3F72FFA40EA080010F0FD
:10EB5000FF0001D06FF00400BDE8F087D6F8E03583
:10EB600007EA832303F1FF6202F5F022A24202D8F2
:10EB70005344A34204D2F3F717FA6FF01500EBE702
:10EB80002146F5E802230120F3F748FA08348046CD
:10EB9000D7E700BF0070FF1F00FCFF0338B5184621
:10EBA0001546049A8BB182B1094B0A4CD3F8E03573
:10EBB00004EA83242C4404F1FF6404F5F02404EBFC
:10EBC000C12112F0F6FD002038BD6FF01500FBE703
:10EBD0000070FF1F00FCFF0310B5034B03600446E9
:10EBE00006F047FD204610BDE04F020810B5044670
:10EBF000FFF7F2FF20465021F6F76BFE204610BDCE
:10EC000010B50449044606F03DFD034B2360204641
:10EC100010BD00BF24010020E04F020813B50023FF
:10EC20008DF807309DF80730044603F0FF014BB123
:10EC3000204606F04AFD0021204602B0BDE8104003
:10EC400006F032BD06F030FD0028F1D002B010BD54
:10EC50000148FFF7D5BF00BF3431002008B5024896
:10EC6000FFF7BAFF08BD00BF34310020028BC08A15
:10EC7000101A7047C28A018B914288BF016903460E
:10EC800083BF885C0132DA824FF0FF307047028B1D
:10EC9000C38A9A4286BF0269D05C4FF0FF3070474A
:10ECA00070B54FF47A730E460021C0E90113034694
:10ECB00015462B4A43F8C42B0446C0F8C4109C22C6
:10ECC000C3E90111C0E93411C0E93611C0F8E01000
:10ECD000283012F02EFCF3B2192B19D8214A52F821
:10ECE000233006F4E0661E43EBB2192BC4F88460AF
:10ECF00022D81C4A52F8233005F4E0651D43002356
:10ED0000C4F88850E36123842361A382204670BD48
:10ED100006F0C002C02A0CD1C82B0AD8124B06F04C
:10ED20003F0206F4E06653F822200E4B53F82230DF
:10ED3000D9E74FF0FF36D7E705F0C002C02A0CD163
:10ED4000C82B0AD8084B05F03F0205F4E06553F8DC
:10ED50002220044B53F82230D0E74FF0FF35CEE7A6
:10ED6000F04F0208D4390208B039020838B5044619
:10ED7000283000F0A9F8E06918B111F095F90023E6
:10ED8000E36120690025258410B111F08DF925611A
:10ED9000A58238BD38B50546074B45F8D43B044637
:10EDA000FFF7E4FF2846F6F7A0FA04F1C400F6F7EF
:10EDB0009CFA204638BD00BFF04F0208B1F5806FC5
:10EDC00070B505460C4610D8038C99420AD9202903
:10EDD0000E4638BF2026C069314611F087FA18B1B7
:10EDE000E8612E84204670BDFEE70024FAE713B5E3
:10EDF00090F824308DF8071004467BB1418C013126
:10EE0000FFF7DCFF40B1638CE2699DF80710D15435
:10EE1000638C01336384012002B010BD01220DF127
:10EE20000701283000F0A0F8B0FA80F04009F3E7BD
:10EE300070B590F8243004460E46154693B1418CC7
:10EE40001144FFF7BBFF10B90025284670BD638C45
:10EE5000E0692A461844314612F0ABFC638C2B441F
:10EE60006384F2E792B2283000F07EF80028EBD1FC
:10EE7000EBE70346006918B19A8A002112F059BBEA
:10EE800070470346C06918B11A8C002112F051BBBB
:10EE9000704738B504460025C5820583FFF7E9FFB2
:10EEA00065842046FFF7EDFF38BD00000248C82208
:10EEB000C721FFF7F5BE00BF843100200148FFF7EE
:10EEC00069BF00BF8431002010B5044690F964008A
:10EED000F2F708FF94F96500F2F704FF201DF3F73D
:10EEE0007FFA206E0321F7F743F9E06D0321F7F76E
:10EEF0003FF92368194A93420ED14FF0B0439A6B01
:10EF000042F400129A639A6B22F400129A639A6D8B
:10EF100022F400129A6510BD114A93420DD14FF0B0
:10EF2000B0439A6B42F480029A639A6B22F4800297
:10EF30009A639A6D22F48002ECE70A4A9342EAD17E
:10EF40004FF0B0439A6B42F400029A639A6B22F43A
:10EF500000029A639A6D22F40002DBE7005400403D
:10EF600000580040005C0040202A30B514D800232F
:10EF70009CB2A24207D890F894301344DBB280F8D8
:10EF80009430002030BD90F89440CD5C1C44044483
:10EF9000013384F87450EBE70120F3E770B590F883
:10EFA0009130012B04460E46A0F1040509D1436EB1
:10EFB0003BB1836E28469847022384F891300023A2
:10EFC0006366012E4FF0000312D1E26E84F8913097
:10EFD0001AB184F890302846904794F8902004F1B4
:10EFE000700120464FF00073BDE87040F3F712BA8D
:10EFF0000122636684F89120616E743129442046B1
:10F000004FF08073BDE87040F3F766BA10B590F822
:10F010009130012B044604D1436E13B1836E043842
:10F020009847022384F89130002363662046BDE8A8
:10F030001040F3F7B3BA436E1F2BDEBF436E0133AC
:10F04000436690F89130012BDAB206D1416E7031EF
:10F050004FF080730144F3F73FBA7047002380F804
:10F060009030704790F892300BB9F3F797BA704729
:10F07000014B1868F3F7A6BA68320020014B1868F4
:10F08000F3F79BBD68320020014B5868F3F79ABA3A
:10F0900068320020014B5868F3F78FBD68320020BA
:10F0A000014B9868F3F78EBA68320020014B9868DC
:10F0B000F3F783BD683200202DE9F041104D2F4653
:10F0C00004468C4690469E46061D0FCF0FC697E815
:10F0D0000700069B86E807001C35A362079BE362D6
:10F0E0000FCD04F13006C4E9088E0FC62B683360DB
:10F0F000002363642046C4F800C0BDE8F08100BF6F
:10F100009835020810B50446006803685B6C9847A0
:10F110002068216A036882689B6898472068216A92
:10F1200003680269DB68BDE810401847006803689F
:10F130009B6C18472DE9F0410D461946037C0446A7
:10F14000407CADF5007DDE08082B5FFA85FC06EB00
:10F15000D0066389879FD0B295BF40EA0C004CEA85
:10F16000122C8DF800008DF8010092BF0DF1010006
:10F170008DF800C00DF10200AB423E443A462CD15E
:10F1800012F017FB206803685B6B98472068216AC0
:10F190000368C268DB689847206803683246D3F882
:10F1A0003880694640ABC0472068216A036802691D
:10F1B000DB68984720680368DB6B98472389AB427C
:10F1C00007D1217C869840AB3A4603EBD10112F07F
:10F1D000F0FA0DF5007DBDE8F081A18912F0A9F9E2
:10F1E000D0E72DE9F04FADF5017D04468C9F9DF8E9
:10F1F00034A21646D5199946002B55D0684612F010
:10F20000D8FA8A993A460DEB060012F0D2FA206835
:10F210000368BAF1000F05D0E26A013254D1DB690C
:10F2200032219847206803685B6B98472068216A01
:10F230000368C268DB689847206803680DF580782A
:10F24000D3F838B02A4643466946D8472068216A31
:10F2500003680269DB68984720680368DB6B98479E
:10F26000BAF1000F07D0E26A20680132036845D185
:10F27000DB6901219847656935B1002F5CD0E37CDB
:10F2800018F80300A8470546B9F1000F07D1A37C81
:10F290008B9806EBD3013A46414412F08AFA28468D
:10F2A0000DF5017DBDE8F08F837C68464FEAD308F9
:10F2B00005EBD30512F07DFAA18908EB07020DEBEF
:10F2C000060012F036F9A2E75B6A9847804620688C
:10F2D000E16A03681B6998470028A3D02068036887
:10F2E0005B6D9847206803685B6A9847E369A0EB09
:10F2F00008009842EBD36FF43075D0E71B6A012108
:10F300009847206803685B6A984705462068E16A69
:10F3100003681B6998470028ADD0206803685B6DBF
:10F320009847206803685B6A9847E369401B9842E6
:10F33000ECD36FF43075A7E73D46A5E7F0B51E4660
:10F34000037987B005460F463BB9CDE900620A460E
:10F350000189FFF7EFFE07B0F0BD90F9114090F87A
:10F3600011C0002CB8BF0734E410013C64B204ABF8
:10F37000E0001946002C12DA2C7CE408601E40B232
:10F38000B0F1FF3F15D10123CDE9022300230196FF
:10F39000009304EBDC022846FFF723FFDBE7B5F818
:10F3A00008E0013C4EFA00FE03F801EB64B20838B5
:10F3B000E0E74FEAC00E27FA0EFE03F801EB013832
:10F3C000DDE7F0B589B000238DF8173003790446E6
:10F3D0000A465BB9012101910DF1170100910189E4
:10F3E000FFF7A8FE9DF8170009B0F0BD90F91130A5
:10F3F000467C002BB8BF0733DB10013B5BB206A88D
:10F40000DD000146002B13DA257CED086B1E5BB294
:10F410005F1C15D10123CDE902330DF117030193D0
:10F420000023009305EBD6022046FFF7DAFED9E76A
:10F430002789013B2F4100F8017B5BB2083DE1E7E2
:10F44000DF0022FA07F700F8017B013BDFE7F0B5A8
:10F4500016461A46037987B005460F4643B9CDE9EB
:10F4600000320A4633464189FFF764FE07B0F0BD1B
:10F4700090F9114090F811C0002CB8BF0734E41087
:10F48000013C64B204ABE0001946002C12DA2C7C7B
:10F49000E408601E40B2B0F1FF3F15D10123CDE971
:10F4A00002230022CDE90062284604EBDC02FFF7CC
:10F4B00098FEDBE7B5F80AE0013C4EFA00FE03F8DF
:10F4C00001EB64B20838E0E74FEAC00E27FA0EFEFF
:10F4D00003F801EB0138DDE7F0B5037989B00446A4
:10F4E0000D468DF8172053B90122CDE900320A46A6
:10F4F0000DF117034189FFF71DFE09B0F0BD90F92A
:10F500001130467C002BB8BF0733DB10013B5BB2E8
:10F5100006A8DA000146002B13DA227CD208531E1B
:10F520005BB25F1C15D10020012301900DF1170083
:10F530000090CDE9023302EBD6022046FFF751FEE0
:10F54000DBE76789013B174100F8017B5BB2083AB2
:10F55000E1E7DF0025FA07F700F8017B013BDFE771
:10F560002DE9F0479DF820A09DF828709DF82C907B
:10F570001C4643EA0A03072B05460E46904642D82E
:10F58000544540D3FFF71DFF631CFF22DBB2CAF1D5
:10F59000080A02FA03F342FA0AF21343DB43DBB22E
:10F5A00080EA0802134205D1B9F1000F02D1002010
:10F5B000BDE8F08720EA030403EA08031C43E4B231
:10F5C000224631462846FFF787FF286803689B6A72
:10F5D00098479DF824804FF47A73814603FB08F81E
:10F5E000286803689B6A9847A0EB0903434502D348
:10F5F0006FF00F00DCE731462846FFF7E2FE60407F
:10F600000742EDD1D3E76FF00A00D1E77FB59DF84F
:10F6100024600396089E9DF82850CDE9013600230A
:10F6200000930446FFF7DDFD38B935B1A36923B176
:10F63000204604B0BDE87040184704B070BDF0B576
:10F6400090F9114090F811C0002CB8BF0734E410B5
:10F6500087B0013C64B205AD0F46E6002946002C98
:10F660000DDA9DF8344002949DF83040CDE9003425
:10F6700013464FEADC02FFF7C9FF07B0F0BD47FAB7
:10F6800006FE013C05F801EB64B2083EE7E77FB5F2
:10F690009DF824600396089E02960026CDE9003668
:10F6A00001239DF828500446FFF79BFD38B935B17A
:10F6B000A36923B1204604B0BDE87040184704B0E8
:10F6C00070BDF0B590F9114090F811C0002CB8BF92
:10F6D0000734E41087B0013C64B205AD0F46E60084
:10F6E0002946002C0DDA9DF8344002949DF83040F4
:10F6F000CDE9003413464FEADC02FFF7C8FF07B03C
:10F70000F0BD47FA06FE013C05F801EB64B2083E85
:10F71000E7E770B586B000238DF8133090F911300B
:10F72000427C002BB8BF0733DB10013B04465BB2C1
:10F7300005A8DD000146002B16DA0123CDE90233CE
:10F740000DF11303019300230093D2082046FFF725
:10F7500048FD054628B963691BB19DF81300984719
:10F76000E080284606B070BDE689013B2E4100F8D6
:10F77000016B5BB2083DDEE770B50B46054601F153
:10F780001404303053F8046B40F8046BA342F9D1F1
:10F790006A640E1F01F11004286856F8041F0368FC
:10F7A00082689B689847A642F6D170BD406C18B934
:10F7B00070478B4204D018300378002BF9D11846DB
:10F7C0007047F8B50546FFF7F1FF88B1041D05F154
:10F7D0002C0605F1400756F8041F002904DB2868B1
:10F7E00022680368DB689847BE4204F10404F2D142
:10F7F000F8BD00000648074B074A1B68B3FBF2F34D
:10F8000010B544684B434268121B9342FBDC10BDA9
:10F81000001000E04000002040420F00CBB2192B46
:10F8200009D80F4A52F8233001F4E0601843431C12
:10F8300018BF0846704701F0C002C02A0CD1C82B7F
:10F840000AD8084B01F03F0201F4E06053F822208F
:10F85000034B53F82230E9E74FF0FF30704700BF09
:10F86000D4390208B0390208704790F8282008B54A
:10F8700012B103681B6B9847BDE80840F6F7C4BA9D
:10F88000C0690EF0C1BBC0690EF0F0BBF8B5074609
:10F890000C465D1E8E18B44200D1F8BD14F8011B51
:10F8A000F86900220EF0E4FB05F8010FF3E70DF014
:10F8B00036BF4B1C084603D00021C0B20DF054BE29
:10F8C0007047084611461A46431C02D0C0B20DF0DC
:10F8D000CBBD7047C0690EF0C8BBD0E90812C06943
:10F8E0000EF0A2BB084611461A46431C01D00EF08A
:10F8F000F7B8002070470EF05DB90EF059B9084610
:10F900000EF05AB94B1C084601D00DF06FBE70477F
:10F910001FB5084611461A46431C13D00024CDE9F2
:10F920000044CDE9024421B1074B0393074B0091FA
:10F93000029369460DF08CFE029B1BB169460322BF
:10F940000846984704B010BD895E0008695E00084B
:10F950004B1C084601D00EF085B8002070470846C1
:10F96000431C114601D00EF043B870470846431CB3
:10F97000114601D00DF0D2BF704710B52C210446BE
:10F98000F5F7A7FF204610BD90F8282012B10368B4
:10F990001B6C18477047000070B586B004AD85E851
:10F9A0000C0004230322CDE90132012200230E467C
:10F9B00000921946044603F07DFE95E80300064BCD
:10F9C000236004F12003E66183E80300002320465E
:10F9D00084F8283006B070BD1C5002080368D3F8C4
:10F9E000DC3018470368D3F8E030184770472DE93A
:10F9F000F04385B00F464FF0000801230DF10F02D0
:10FA000040F6E70106468DF80F8002F0B4FA04468E
:10FA1000002855D133683046D3F8D83098470421B0
:10FA20008146FFF7C3FE032105464846FFF7BEFEA9
:10FA300028B165B90E2F47DD6FF00C0440E017F1D7
:10FA4000090FF9DB002DF7D007F1090303E00E2FB2
:10FA5000FBB20EDD0933DBB21F2BEDD801250723E6
:10FA6000224600950421304602F066FA042304463B
:10FA70000DE01133DBB21F2BDED8012223460092AA
:10FA80000421304602F058FA45460446032386F81E
:10FA90005831ACB92946304601F0E7FA044678B946
:10FAA0000422F9B2304602F0FCFA044640B90123C0
:10FAB0000DF10F0240F6E701304602F055FA044618
:10FAC000204605B0BDE8F08307F11103DBB21F2B20
:10FAD000B2D80122234600920421304602F02CFACB
:10FAE00003230446D3E7000010B502F098FA044659
:10FAF00005480EF020FD04480EF011FD10B102483B
:10FB00000EF013FD204610BDB837002010B5044696
:10FB100003480EF00DFD2368BDE81040184700BFF4
:10FB2000B837002001480EF0E9BC00BFB83700200C
:10FB300010B54FF4DE710446F5F7CBFE204610BD3C
:10FB4000F0B587B004469DF844E09DF830509DF82C
:10FB500034609DF93870BDF83CC0CDF814E0DDF894
:10FB600040E0CDF810E0CDE9027CCDE9005600F090
:10FB700030F9014628B9204607B0BDE8F04003F04F
:10FB80008FBA07B0F0BD012A02D101600020704792
:10FB9000022A05D0032AF9D0002AF7D10260F5E73E
:10FBA0000B680360F2E700001FB50023CDE90013E6
:10FBB000084B03930848094B029369460EF064FC16
:10FBC000029B1BB1694603220846984705B05DF8C1
:10FBD00004FB00BF0DFB0008B837002087FB0008BE
:10FBE000F0B587B004469DF93450BDF838609DF8F3
:10FBF00040700497CDE901560F9F0C9D0397009527
:10FC000000F021F9014628B9204607B0BDE8F040D0
:10FC100003F046BA07B0F0BD10B5044600F088F90D
:10FC2000014B2360204610BD84500208704700003D
:10FC300008B5A1F11A030846032B16D8DFE803F034
:10FC40000A0206110B480EF0ADFC08BD09480EF083
:10FC500075FCFAE707480EF087FC80F00100C0B29F
:10FC6000F3E704480EF097FCF7E7BDE808400DF015
:10FC7000F9BE00BFB83700200846A0F11A03032BD5
:10FC8000114601D90DF04ABE704710B52C2104462B
:10FC9000F5F71FFE204610BD08461C28114604D863
:10FCA0001A2810D809D00DF0A3BE1D28FBD1B2FA36
:10FCB00082F1054849090EF061BCB2FA82F10248AE
:10FCC00049090EF043BC7047B837002037B50446E9
:10FCD0002C20F5F7FAFD0A4B0A4905460CCBFFF735
:10FCE0005BFE094B2B601B221D23CDE90032294608
:10FCF0001C231A222046FFF7DFF9204603B030BD4F
:10FD0000EC510208B83700208C5102084AB116297C
:10FD10000B466FF00800A8BF16238342B8BF034606
:10FD200013700931C9B21F298CBF6FF00C0000207D
:10FD30007047000010B5012986B006D002292BD0EB
:10FD4000C9B16FF0130006B010BD00220368059220
:10FD5000194A04924FF0080C0A22CDE9022C4FF008
:10FD6000120E0722CDE9002E1449D3F8F040144AB0
:10FD70000923A047E7E7104A0368039210240A22E8
:10FD8000CDE901240F4A04910092D3F8F4400E4AC1
:10FD90000E4B0A49A047D6E7002302680393064B9F
:10FDA00002930A210123CDE900310449D2F8FC4035
:10FDB0000622A047C7E700BFCDCCCC3F0000D94307
:10FDC0000000FA4233331C439A9999400000A04046
:10FDD00070472DE9F34198469DF8343001930C9B10
:10FDE00000930E461746BDF82C309DF824209DF850
:10FDF00020109DF92850044601F0FEFA00BB23684C
:10FE00004146D3F8E83020469847C8B923683946B8
:10FE1000D3F8E4302046984790B923683146DB6B2D
:10FE20002046984760B90121204601F01EF938B9F3
:10FE300023685B6D2946204602B0BDE8F0411847B3
:10FE400002B0BDE8F081F0B585B00E469DF838707F
:10FE5000029711460D9F01971A46BDF83030009366
:10FE60000A9B9DF92C50044601F01CFB90B92368B5
:10FE70003146DB6B2046984760B90121204601F0EE
:10FE8000F4F838B923685B6D2946204605B0BDE813
:10FE9000F040184705B0F0BD70B50E461D4611463E
:10FEA0009DF81430049A044601F070FB88B9236869
:10FEB0003146DB6B2046984758B90121204601F0B6
:10FEC000D4F830B92368294620465B6DBDE8704000
:10FED000184770BD73B50E4611461A469DF824307A
:10FEE0000193089B00939DF818309DF91C5004461F
:10FEF00001F062FB90B923683146DB6B20469847DE
:10FF000060B90121204601F0B0F838B923685B6D73
:10FF10002946204602B0BDE87040184702B070BDC7
:10FF200010B54FF4DE710446F5F7D3FC204610BD42
:10FF300010B5044600F068FC034B2360034BC4F883
:10FF40004C31204610BD00BF04520208F451020893
:10FF500070B50C460546144920461646F1F7B4F82C
:10FF6000F0B112492046F1F7A5F8C8B12EB12146EB
:10FF70002846BDE8704003F0F7B8D5F85411204684
:10FF8000F0F7E6FD0A4920F00040F1F79DF800285F
:10FF9000EDD02146284600F0DAFE0028E7D070BDFB
:10FFA0006FF00B00FBE700BF000016430000704439
:10FFB0000000A0410022FFF7CBBF0000036873B52B
:10FFC0009B6D1646002205460C46984790B99EB197
:10FFD0000B4B04F1090203EB420113F8123091F9C3
:10FFE000014003F00F021B09002100912846214621
:10FFF00003F066F802B070BD04220723F4E700BFE7
:020000040801F1
:10000000045302080122FFF7D9BF000030B5074BA7
:1000100005460FCB85B06C4684E80F002B6821465F
:10002000D3F8A0302846984705B030BDC83502083F
:1000300013B5036800220092DC6940F272220223A9
:100040006FF07F41A04702B010BD000030B5074BF4
:1000500005460FCB85B06C4684E80F002B6821461F
:10006000D3F894302846984705B030BDC83502080B
:1000700082B02DE9F041012906A880E80C000B9C14
:100080009DF826609DF8277009D0022975D00029B7
:100090004BD06FF01300BDE8F04102B070479DF8FF
:1000A000188042F2107000FA08F0F0F703FE514990
:1000B00005460798F0F756FE01462846F0F706FF7A
:1000C000F1F752F8A8F10503DBB2012B9DF82830B7
:1000D00005468BBF08210021112019200BBB4FEAD8
:1000E000880304EB4707002EC8EB47020CBF142619
:1000F000002601EB8201DBB2314409B25A1E00290D
:10010000A8BF521892FBF3F3BDF824209DF82010ED
:100110009BB2083201FB032300EB83006843800895
:10012000B9E7A8F102039B00DBE7F800F0F7C6FD92
:1001300005463046F0F7C2FD01462846F0F70AFDB5
:100140000546BDF82400F0F7B9FD01462846F0F752
:1001500001FD0546E000F0F7ADFD01462846F0F749
:10016000F9FC254904460698F0F7B0FE0146204602
:10017000F0F7ACFEF0F7F8FF8DE79DF81930032B90
:1001800034D8DFE803F002282D300623634304331C
:100190000522B3FBF2F39CB23022B4FBF2F303EB83
:1001A000830000EB800002FB13444000A4B280B245
:1001B00014B10234204480B29DF82430C3EBC30252
:1001C00003EBC20300EB43000C4B80B25843F0F743
:1001D00071FD0B49CCE704EB4404C4F34F04DBE7A7
:1001E0006400A4B2D8E704EB4404FAE76FF0090016
:1001F00051E700BF0000204100007A4400127A005D
:100200001D24F44308B50846F0F754FD0249F0F701
:100210005DFEF0F7A9FF08BD00007A41036889B2CE
:10022000D3F8EC3018470368D3F8DC301847D0F81F
:100230005C01704700F00E03062B0BD0082B0CD08E
:100240000A2B0CD00138C0B2FD288CBF6FF0010022
:10025000002070476FF430707047024870470248C2
:10026000704700BF3EFDFFFF3DFDFFFF70470000F0
:100270002DE9F0428AB004460F4601F0FFFE05AEBC
:1002800000230DF11C090128C9E901330546079334
:100290000593B3803DD194F86131042B35D80433F4
:1002A000DBB28DF8243094F860318DF81C30D4F82E
:1002B00068310893B4F86631ADF8143094F86331BE
:1002C000003B18BF01238DF8173094F86431591E94
:1002D0004B424B418DF8163094F86231003B18BF09
:1002E00001238DF81830039796E80300099B0190CD
:1002F000ADF808100093216899E80C008E6F204635
:100300002946B0470AB0BDE8F082072B08BF082392
:10031000C7E730BBD4F87001F0F7CCFC01462148A8
:10032000F0F7D4FD0790D4F87401F0F7C3FC94F80B
:100330007B31089013F0FB0F11D0022B03D09A1FD2
:10034000534253415B00B4F88021ADF8142094F877
:100350007C218DF816208DF817300025C3E7012386
:10036000F1E703280ED1B4F89C315BBAADF81C302C
:1003700094F8A3318DF81E3094F89E318DF8143026
:100380000225B0E7022809D1D4F87001F0F792FCF9
:1003900001460448F0F79AFD0790DEE76FF013007E
:1003A000B0E700BF00007A4910B50C4659B101F022
:1003B00065FE012802D0032803D038B92070002040
:1003C00010BD0220FAE76FF00200F9E76FF01300AA
:1003D000F6E708B5D0F85C010221FFF7F2F94FF01B
:1003E000FF3008BD37B50D46044690F85811D0F8D7
:1003F0005C01FFF7E6F95DB90123CDE90033002385
:10040000D4F85C011A46D121FFF75BF903B030BD87
:100410002946204601F014FE0028EDD0F6E707B586
:1004200000238AB20093114601F0DCFD03B05DF8B1
:1004300004FB1FB50023ADF80C300123CDE90033D8
:1004400003AA02231221D0F85C01FFF7F8F8BDF8E7
:100450000C0040BA80B205B05DF804FB2DE9F04114
:10046000002486B0FF270226CDE90274CDE90046BC
:1004700005462346224640F6E201D0F85C01FFF72C
:100480006FF8CDE90274CDE900462346224640F6D6
:10049000E501D5F85C01FFF763F86FF07F4128466E
:1004A00001F0E5FCD5F85C31186803680A21DB69C6
:1004B00098472746264601230DF1170240F61901F9
:1004C00028468DF8176001F056FD9DF8170000F0E2
:1004D0000100A04001343843082CC7B2EBD12B688F
:1004E00002244FF0FF081B6928469847CDE90148D0
:1004F00003960096D5F85C010023012240F6E20144
:10050000FFF72EF8CDE90286CDE900640023D5F887
:100510005C01012240F6E501FFF722F8384606B0FB
:10052000BDE8F08190F83410022938B5044605D0B2
:10053000032911D06FF01805284638BDD0F85C01AA
:10054000FFF73FF9D4F89811204601F090FC0546DA
:10055000002384F83430EFE790F85811D0F85C01AC
:10056000FFF72FF90021204601F06BFC054600281B
:10057000E2D1D4F85C311868D96A026812699047F0
:100580000028E5D0D4F85C31186803685B6D9847A3
:10059000EFE7D0F85C3110B50446186803681B69B2
:1005A0009847C1B22046BDE8104002F03BBF10B5ED
:1005B0004FF4DE710446F5F78CF9204610BD036850
:1005C00010B5D3F8EC3044F2FF310446984728B90F
:1005D000236820461B69BDE81040184710BD000085
:1005E00010B5044601F04AFD01280ED123682046CB
:1005F000D3F884309847C3050AD410F0800F14BF95
:100600006FF00E004FF0FF3010BD6FF01300FBE7EE
:100610000048F9E742FDFFFFF7B505460E4601F039
:100620002DFD012833D12B6828461B6998470446C5
:1006300050BBD5F85C010221FFF7C3F8B16828462A
:1006400002F0C0FEF1680746284602F0BBFE0094A7
:10065000234682B2B9B2284601F0C4FC044698B9D8
:100660002B6844F2FF31D3F8EC3028469847044613
:1006700050B973680193F3780093B3787278317846
:10068000284601F00BFC0446204603B0F0BD6FF095
:100690001304F9E710B5044601F0F0FC012812D16B
:1006A000204601F023FE10F4004FC0F3072018BFCE
:1006B000A0F58070EFF796FE044B0022EFF7FCFEEA
:1006C000F0F7F2F910BD0248FCE700BF0000D03F90
:1006D0000000A0C12DE9F3411D4603681B690446D3
:1006E0000F4616469847002846D16DB92368002E5C
:1006F000DB6F14BF3146FF21204698474FF47A73D1
:1007000000EB8000B0FBF3F52846F0F7D3FA2D4953
:10071000F0F728FB2C49F0F7D9FBF0F725FD23680B
:1007200000220092D3F81C800146022340F272227C
:100730002046C04700BBD4F85C31186803685B6A88
:1007400098478046D4F85C311868596A0268126983
:100750009047A0B10025236820461B69984718B12F
:100760006FF43073984207D12368D5B123682046CF
:10077000DB6A98476FF0050002B0BDE8F081D4F85D
:100780005C31186803685B6D9847D4F85C31186871
:1007900003685B6A9847A0EB08008542D2D2012526
:1007A000D9E7D3F8843020469847236B1842DDD12F
:1007B00023681B6B32463946204602B0BDE8F04143
:1007C000184700BF00007A4400007A41036810B562
:1007D000D3F894300446984730B110BDD4F85C315A
:1007E000186803685B6D9847D4F85C311868596ADB
:1007F0000268126990470028F0D023682046D3F899
:100800009830BDE81040184738B504460D4602F050
:10081000B5FD0022C4F85421C4F86821C4F884212D
:1008200040F20162A4F89C212B4A2C4B12692360F0
:10083000032000230121C4F89F21294AC4F84C3128
:10084000C4E95C33C4E96933C4E96C3384F85031DA
:1008500084F85801C4F8603184F86431A4F8663132
:1008600084F86C11C4F87831A4F87C3184F87E31B6
:10087000A4F88031C4F8883184F88C31C4F8903100
:1008800084F89431C4F8983184F89E0184F8A33137
:10089000A4F8AC31C4F8B8316260FF22A26084F8D9
:1008A000493184F84A3102220423C4E90423E16077
:1008B00010230821C4E9061320204023C4E90803BB
:1008C000C4F85C514FF480738025C4E90A534FF497
:1008D00000732363204638BDC83502084C53020814
:1008E0000024743F10B5032ABDF8084011D8092927
:1008F00080F89C2110D85A1E032A80F89D110ED82A
:10090000B4F5007F80F89E310CD2A0F8AC410020F5
:1009100010BD6FF00900FBE76FF00700F8E76FF01C
:100920000A00F5E76FF06900F2E7D0F85C3170B5C6
:100930000446186802680D469668996A8268B0474E
:10094000D4F85C311868996A0268D668C268B04702
:10095000D4F85C31186803680121DB699847D4F842
:100960005C311868996A0268D6680269B047F5B1C7
:10097000D4F85C31186803685B6A984706462368B8
:1009800020461B699847054688B1D4F85C31186841
:1009900003685B6A9847801BB0F57A7F08D2D4F869
:1009A0005C31186803680A21DB699847E7E700258E
:1009B000284670BD036810B5D3F8843004469847C4
:1009C000430410D5D4F8B811204601F00F0101F00E
:1009D0006DF950B923682046D3F8EC30BDE81040DB
:1009E00044F2FF3118476FF0040010BD2DE9F047C5
:1009F000984603681B6904460F4616469847002828
:100A000041D194F86131042B3FD9072E5BD994F87A
:100A10006331012B39D1FD2E58D823683146DB6F65
:100A20002046984723680546D3F82490324643462B
:100A300039462046C84730BB20464FF47A7305EB51
:100A40008505B5FBF3F501F019FBD4F85C310646DA
:100A5000186803685B6A984705350746D4F85C3127
:100A6000186803685B6D9847D4F85C3118680368B0
:100A70005B6A9847C01B854209D2236820469B6A5F
:100A800098476FF00400BDE8F087FF2EC4E7D4F864
:100A90005C311868596A0268126990470028DDD0F5
:100AA000032E236809D1D3F8843020469847C30722
:100AB00003D42046FFF77EFFD0E7236820469B6AD9
:100AC000BDE8F04718476FF01D00DCE76FF003004A
:100AD000D9E72DE9F0411E46036886B01B6905463B
:100AE000884617469847044600283CD16FF07F435C
:100AF00098453946284618BF46F4007602F062FC55
:100B000031460446284602F05DFC002382B2A1B2C1
:100B10000093284601F066FA044620BB02460146CF
:100B2000284601F0C2FB0446E8B92B6844F2FF31C5
:100B3000D3F8EC30284698470446A0B9284601F07F
:100B40009DFA012813D195F89431019395F86431F9
:100B5000009395F8903195F86321B5F86611284611
:100B600001F028FB0446204606B0BDE8F081A8B994
:100B7000FF23049395F87E31039395F87D31CDE9F9
:100B8000014395F87C31009395F87B3195F87821F5
:100B9000B5F88011284601F033FBE3E74FF0FF344E
:100BA000E1E700001FB571B101F0A0FBC0B2EFF7A3
:100BB00019FC0F4B002201F10041EFF77DFCEFF72C
:100BC00073FF04B010BD0123CDE900338DF80F1081
:100BD0000DF10F021521D0F85C01FEF730FD9DF8F4
:100BE0000F00F0F767F84FF03F41F0F7BBF8E8E788
:100BF0000000E03F0121FFF7D5BF30B585B00546C5
:100C0000144601F03BFA012808D195F86431012B14
:100C100004D11CB9D5F8900105B030BD0023ADF862
:100C20000C300123CDE9003303AAD5F85C0102237F
:100C30001321FEF704FD14B19DF80D3023709DF8CB
:100C40000C00E9E72DE9F3410546D0F85C010F46B9
:100C50001646FEF75EFD2B680446D3F8843028461E
:100C600098476FF430739C4208D110F4007F18BF8E
:100C70006FF00504204602B0BDE8F081002CF9D1E8
:100C800043062CD400F03000202814BF4FF0000899
:100C90006FF0060800230DF10702012128468DF8A8
:100CA0000730FFF7AAFF16B1B04228BF3046C2B2E4
:100CB0009DF807303946284601F080F9044600289F
:100CC000D8D12B6844F2FF31D3F8EC30284698474E
:100CD000B8F1000F0CBF04466FF00604CAE76FF0CE
:100CE0000608D7E70022FFF788BF73B50546084618
:100CF0004FF07E511646EFF72BFF4FF07A51F0F789
:100D000031F80DF089FDF0F72FFA4FF07E51C4B2A3
:100D10003046EFF71FFF4FF07A51F0F723F80DF050
:100D200039FDF0F721FAE107C3B25CBF04F1FF34EB
:100D3000E4B2DA075CBF0133DBB201A928468DF8C3
:100D400004408DF8053001F08BF902B070BD73B529
:100D5000002305460846ADF804300C46F0F7DEF9EE
:100D6000A0F286331A2B21D9A0F25F33072B28D9A2
:100D7000A0F20B33082B27D9A0F5EB73282B26D92B
:100D8000A0F5D7730A2B25D94FF081412046EFF704
:100D9000E1FE4FF0814106462046EFF7D9FE32468C
:100DA00001462846FFF7A1FF02B070BDE122E9230A
:100DB00001A928468DF804208DF8053001F050F97E
:100DC000F2E7D722DB23F3E7C122C523F0E7752240
:100DD0008123EDE76B226F23EAE7000037B500239C
:100DE0008DF807300DF10702012340F68901044612
:100DF00001F0C1F8E8B9204601F040F901289DF85A
:100E0000075018D10D49D4F86801EFF7A1FE0C493D
:100E100020F00040F0F74EF968B105F0FB05012322
:100E20000DF1070240F6890120468DF8075001F0C8
:100E30009BF803B030BD45F00405F0E70000FA432D
:100E40006F12833A2DE9F0410229C8B005460E46DB
:100E5000174606D0032921D06FF0180048B0BDE82E
:100E6000F08190F86431012B03D1D3680BB1C0F845
:100E70009031D7E9012339682846FFF72AFE002878
:100E8000ECD13B68013304BF6FF07F433B603B68AC
:100E9000C5F8983185F834600020DFE75368FF2BF0
:100EA00000F2DD8001F0EAF80128044615D195F83A
:100EB0009431019395F8643100933B7995F863215F
:100EC000B5F86611284601F075F90028C6D100234F
:100ED0000093012240F2012139E0A8B93B79049343
:100EE00095F87E31039395F87D31CDE9010395F8AE
:100EF0007C31009395F87B3195F87821B5F8801115
:100F0000284601F07DF9E0E7022818D1D5F87031C4
:100F10007968642B4FEAC1039BB241F6705243F2E9
:100F20000F700093C9B240F2E14308BF134640F688
:100F30002F1208BF0246284601F08BF9C5E70328A7
:100F400040F09080002344F20102009311462846AD
:100F500001F048F8002881D102460146284601F0F8
:100F6000A4F900287FF47AAF032C19D003463A790C
:100F70003968284601F00EF800287FF46FAF2B681F
:100F800044F2FF31D3F8EC302846984700287FF42C
:100F900065AF2846FFF722FF00283FF47BAF5DE7EF
:100FA000284600F0D3FD00287FF458AF044695F89A
:100FB0009E31C3F10403A3424CDC0024FB222146F2
:100FC00009A8089410F0B5FA05F5DA73C5E96C4480
:100FD000C5F8B8410DF11C08029305F5D873CDE9A9
:100FE00000832846D7E9001208AB079400F030FBD5
:100FF00000287FF433AF03469DF81C2008A928463B
:1010000000F0C8FF00287FF429AF01238DF81830C5
:10101000079B8DF81930D5F8B4318DF81A3006AA2F
:10102000032340F28531284600F09EFF00287FF41C
:1010300015AF95F8B471102F28BF10270446A742AA
:101040009DD9E1B2284600F031FE00287FF406AFBA
:101050000134F4E7284600F00FFE0134A7E76FF0F3
:101060000300FBE64FF0FF30F8E637B500230D46EE
:101070008DF807300DF10702012340F6D801044630
:1010800000F079FF70B99DF807306DB143F01E0391
:101090008DF807300DF10702012340F6D8012046F4
:1010A00000F062FF03B030BD23F01E0343F00803DD
:1010B000EEE737B590F86431012B044602D00020EA
:1010C00003B030BD00F0DAFF01280546F7D1002358
:1010D0008DF806300DF10602034640F60211204657
:1010E00000F042FF0028EBD18DF807002B460DF1F0
:1010F000070240F64411204600F03DFF0028DFD1F2
:101100009DF8073043F002038DF807300DF1070218
:101110002B4640F64411204600F026FFD0E7036836
:1011200010B51B690446984760B92046FFF7C1FF18
:1011300040B923682046D3F8EC30BDE8104044F2B3
:10114000FF31184710BD37B500230D468DF8073025
:101150000DF10702012340F23671044600F00BFF47
:1011600088B99DF80730012D0CBF03F0FB0343F055
:1011700004038DF807300DF10702012340F23671A8
:10118000204600F0F1FE03B030BDF0B585B0044656
:1011900000F074FF0246002878D1D4F87031D4F8FA
:1011A0005C010392FF26B3F5966F029609D10221E6
:1011B0000423CDE9003140F6B801FEF7D1F905B0BE
:1011C000F0BDB3F5167F4FF002054FF00303CDE9F4
:1011D00000354FF004032ED1182240F2D161FEF702
:1011E000BFF90028EBD1CDE90260CDE90055042319
:1011F000D4F85C011A4640F69B01FEF7B1F90028CD
:10120000DDD1CDE9026004270195009702463B46F7
:10121000D4F85C0140F6B801FEF7A2F90028CED15F
:10122000CDE90260CDE9007506235022D4F85C01B7
:1012300040F2AC61C1E7082240F2D161FEF790F9BB
:101240000028BCD1CDE90260CDE900550246042357
:10125000D4F85C0140F69B01FEF782F90028AED17C
:10126000CDE90260042701950097D4F85C013B4664
:10127000102240F6B801FEF773F900289FD1CDE99E
:101280000260CDE9007506230246CFE7002096E70D
:10129000F0B5054685B00F460A24002601212846F0
:1012A000FFF743FBD5F85C0110224FF448716B4601
:1012B000CDE90066CDE90266FEF740F806226946F0
:1012C000384610F05CF910B9012005B0F0BDD5F832
:1012D0005C31186803680A21DB69013C984714F007
:1012E000FF04DBD12046F0E72DE9F0410446D0F8B9
:1012F0005C010D4617461E46FDF704FFD4F85C312D
:101300001868596A0268D2F808804268C047D4F861
:101310005C311868D96A0268D2F808804268C04710
:10132000D4F85C3131484FF401621A820122DA7438
:10133000D4F85C314FF440011A712D4A5A61C3E967
:101340000201D4F84C112046FFF7A2FF40B9D4F8AF
:101350005C01FDF7EBFE6FF001052846BDE8F0816A
:1013600094F8493163B13146204601F012FF054639
:10137000B0B9002F34D12046BDE8F04101F0A9BD3D
:1013800000212846EFF7AAFE0028ECD0294641F2BA
:101390008832204601F0C6FD05460028E3D0DCE790
:1013A000236820461B699847204600F0C1FF114B77
:1013B0009D42D2D18306D0D5002384F8493141F231
:1013C00088320021204601F0ADFD05460028C4D139
:1013D0003146204601F0DDFE05460028C9D0BCE7B5
:1013E0002046BDE8F04101F071BD00BF1D000D00B9
:1013F000350201083DFDFFFFF7B51D46264BC0F83D
:101400006831062380F8503100231646C0F8883131
:10141000224A80F86431FF230F46C0F86021C0F8EB
:1014200090319DF824200899A0F8665101230446C4
:10143000FFF75AFF70BB02463946204601F053F8C9
:1014400040BB44223146204601F07AF810BB2368A5
:1014500029461B6E20469847E0B91149204601F005
:101460008FF8B8B90121204601F01AFE90B9012386
:10147000009341F60F5241F221030221204601F070
:101480006DFC38B923681B6D0146204603B0BDE8EA
:10149000F040184703B0F0BD0000FA430903000113
:1014A000000070422DE9FF4117461E4645F25532B5
:1014B0004CF6CC43C0E95C23324BC0F884311A238C
:1014C000BDF8285080F8793140F209638846A0F8C9
:1014D0007A319DF830200B99A0F880510023044602
:1014E000FFF702FF002849D1236841461B6C2046C4
:1014F0009847002842D1236839465B6C20469847BC
:1015000000283BD13146204601F018FA002835D199
:101510001D49204601F034F880BB236829461B6E24
:101520002046984750BB4AF61253ADF80C3023685A
:101530000222DB6D03A920469847F8B923680146CB
:101540009B6C20469847C8B923680146DB6C20464F
:10155000984798B9FF21204601F002FE70B9012595
:10156000009541F2210341F60F520221204601F07D
:10157000F5FB18B92946204601F092FD04B0BDE8FC
:10158000F08100BF33331C430000704238B50D4674
:1015900011461A4602230446FFF7A6FE58B92368EF
:1015A00029461B6C2046984728B920460121BDE8F2
:1015B000384001F075BD38BD70B586B00D46164691
:1015C00080F8A3319DF82C200A9903230446FFF7E5
:1015D0008BFE88BB1C49204600F0D2FF60BB012176
:1015E000204601F05DFD38BBCDE90300CDE90100E7
:1015F0000090034602460146204600F001FED8B99D
:101600000B2384F87A31236884F87901C4F87401D3
:101610001B6C0E492046984770B9032E0ED8092D31
:1016200084F89C610DD8032384F89E314FF48073B5
:1016300084F89D51A4F8AC3106B070BD6FF009007C
:10164000FAE76FF00700F7E7000070420000FA3E8B
:101650002DE9F04F83469146ADF5297D1C460020CB
:10166000FF22484540F0CA80B0481023002603708E
:1016700047F25B574FF6FF734A462146C0E90173B4
:10168000C66001F015FFC0F3072304F8093004EB2E
:1016900009034FF41772587009F102033146E654FA
:1016A00009AD11A8059310960FF043FFA0482E60D6
:1016B000032101F058FF09F10203DA00063210ABF2
:1016C00021469B48009501F053FFFF2231462046FA
:1016D0000FF02FFF9BF89C71032F2ED0954B0CAA77
:1016E00003F1080C18685968164603C608336345A9
:1016F0003246F7D1186899889B79B371022F98BF49
:101700008D4B3060B18098BF13F807C02B680293EF
:101710004FF0000388BF4FF0000C1A4618460DF139
:1017200030084FF0010A029999427BD109920732A1
:10173000D208214610A810F03CF8099B0293002221
:1017400093B202985B438342114602F10102F7D340
:101750008BB25B009BB204939BF89E31BDF908509D
:10176000C1F34E020692C3EBC30203EBC203002196
:101770005B009BB28A460A46002D74DC9BF89E21D2
:101780006A4F8DF828906FF0710101FB02330993C5
:101790009BF8A3319BF89C219BF89D119B0043EA89
:1017A000C20343EAD10343F002038DF82930BBF8AA
:1017B000AC311A091B0142EA41128DF82B30082383
:1017C0008DF82A203B702F22FF23C7E90123002632
:1017D000FE6035469BF89E11B14200F2AF80059B3A
:1017E0009BF89C21DB0006339BB2032A00F27B812D
:1017F000DFE812F06D017501A001A2010B5C5340FE
:101800001D0145EA13132354130983EA521383EA93
:10181000D20303F0010383EAD2135200D2B21A4377
:1018200001301EE718F80010B9B110AFDE084FEA1A
:10183000D20EBE5D14F80E10DF43D54307F0070744
:1018400005F007053E41F6070AFA05F546BF2943AC
:10185000C9B2A94304F80E1001320130844508BF13
:10186000002001335FE7302D28464FEAD306A8BF9A
:1018700030200390D843A75D4FF0010C00F0070023
:101880000CFA00F027EA000703EB0C00A755C7107D
:10189000C043E65D00F007000CFA00F026EA0006FF
:1018A000E6554FF0000C9F1CFE434FF0010E06F072
:1018B00007060EFA06F60DF140084FEAD20EF810B0
:1018C00018F80EE007906FEA020808F00708205C9D
:1018D0004EFA08FE1EF0010F14BF3043B0434FEA2A
:1018E000E70618BFC0B2A05504980244029892B20D
:1018F00090420BD8069A0498524492B290429FBFED
:10190000013189B20A468A4688BF9246039E0CF18D
:10191000010C0FFA8CF0864207F10107C4DC304657
:101920000230303D18442DB283B225E774320020D6
:1019300088320020E0350208435402089DF82B301D
:101940000139891B23F00C0343EA810304220AA90D
:1019500038468DF82B3001F0ABFD0DF130084FF01B
:101960000009C8F800908DF82C0002217448CDF8C9
:101970003490ADF8389001F0F6FD28220DEB02010D
:1019800043466F48CDF8009001F0F2FD28220DEBA0
:10199000020143466A48CDF8009001F0E9FDEA08EB
:1019A000EB43A15C4FF0010E03F007030EFA03F3C3
:1019B00021EA0303A35405EB0E03DA10DB43A15C19
:1019C00003F007030EFA03F321EA0303A3545D4B6C
:1019D000029305F1020C05F12A00029B13F8011B8A
:1019E00002934FEAD1094FEADC0A18F8099014F87B
:1019F0000A30C9436FEA0C0201F0070102F0070246
:101A000049FA01F919F0010F0EFA02F218BF134357
:101A10000CF1010C14BFDBB29343604504F80A30AB
:101A2000DBD105F17203DFF82091029305F14A0C36
:101A30000DF1300A19F8011F6FEA0C024FF0010E88
:101A400002F007020EFA02F24FEAD10E4FEADC086A
:101A50001AF80EE014F80830C94301F007014EFAF5
:101A600001FE1EF0010F1ABF1343DBB2934304F8CB
:101A70000830029B0CF1010C6345DBD100214FF0D3
:101A800001090BEBD10C4FEAD0089CF89FC114F868
:101A900008306FEA010EC2430EF0070E02F0070293
:101AA0004CFA0EFC1CF0010F09FA02F218BF1343A6
:101AB00001F1010114BFDBB29343202904F808307F
:101AC00000F10100DDD17235ADB2013682E60622A9
:101AD000534304330522B3FBF2F39BB203E003EB61
:101AE0004303C3F34F03302003F12F02B2FBF0F2A4
:101AF0000A44B4990A60B3FBF0F101EB810202EBF6
:101B0000820200FB113352009BB292B213B1023336
:101B10001A4492B29BF89E11722313FB0123B39ACD
:101B20001360B29A0733DB08002013600DF5297D9E
:101B3000BDE8F08F5B00D0E703EB4303CDE700BFC8
:101B400088320020465402086D54020870B5464A97
:101B50008AB0034605AC02F11006106851682546AC
:101B600003C50832B2422C46F7D110683F4A2860BC
:101B700010689288ADF810203D4A029249F28E52C8
:101B8000ADF8042093F8A3210390002A93F89D2137
:101B90000AA800EB42020CBF3421082132F8142CB1
:101BA000B2FBF1F20621632AA3F8A421A3F8A6113F
:101BB0002AD037D83C2A53D022D81E2A19D8092A2D
:101BC0001BD92C4921FA02F2D20716D5B3F8AC2161
:101BD0000AA901EB9211B2F5C07F11F81C1CA3F801
:101BE000A81102F03F01A3F8AA1106D200200AB002
:101BF00070BD232AEAD02F2AE8D06FF06900F6E7FB
:101C00003E2A2DD0562AF8D1B3F8AC210AA901EB0F
